:100000000C94575A0C94835A0C94835A0C94835A28
:100010000C94835A0C94835A0C94835A0C94835AEC
:100020000C94835A0C94835A0C94835A0C94835ADC
:100030000C94835A0C9422600C94835A0C94835A27
:100040000C94835A0C94835A0C94835A0C94835ABC
:100050000C94835A0C94835A0C94835A0C94835AAC
:100060000C94835A0C94835A0C94835A0C94835A9C
:100070000000000000000000000000000000000080
:100080000000000000000000000000000000000070
:100090000000000000000000000000000000000060
:1000A0000000000000000000000000000000000050
:1000B0000000000000000000000000000000000040
:1000C00000000049000000495252000052525C2DCD
:1000D0000000000000000000000000000000000020
:1000E0000040000000494A52004952525B1C5253E2
:1000F0001C25241B2425251B0A0A2D1C12120A0A62
:100100000000000000000000404949494949525B95
:100110005B5B525B1C1C1312241C12090909120997
:100120000909090A0A0A0A0A0A13120A0A12130A10
:100130000000000000009252525252521312130952
:10014000001C0A1212401B65090A0009241B120038
:1001500000251C1C010025241C1C0024252424240B
:100160000000000000005249494000001B135249A2
:100170004900641C1C5B4A481C651C2552491C1C18
:10018000652464491C1C652564491C1C6D2E5C4952
:100190000000000000000000000000490000000016
:1001A000535200000053522500004A5225250000FA
:1001B0005B251300005B53000A1C095B1C657F373D
:1001C0004052522E2E1C525C2E251B1324251C1C23
:1001D00012002525120000121B0000132E37001BF1
:1001E00037372E2E37372E2E2E2E2E2E6E6E6E1C5D
:1001F0001313120009131200001213130012251C0E
:1002000013132E371C131313361C131B1B1B251320
:100210001C1C1B1B1B1C1C1C1C1C1C1C1C1C1C132A
:100220001312121313001313131C000913131C01D0
:100230000037131C13002E2E1C1C001C772E2500CB
:10024000137F251C010A37241C1C0A2E25250900B2
:10025000132E242525252E252525252525252D2E3E
:10026000251B2E2E251C1325251C1C1C1C011C1CAB
:100270001300011C0A000165775C016E7F6E521B42
:1002800025256D1C524925251C1353001C1C1C528E
:100290004A001B135B5B000009525C0000005B5CC2
:1002A000000000001B000000000000000000000033
:1002B000135B7F776E6E136577766E6E1B65777650
:1002C00076761B5BBF76B67609136DBFB7B6001B9B
:1002D000125C76BF0000121B125B00000000090ACE
:1002E0006E6E6E77241C6E6E77251C1C6E776E1CEE
:1002F0001C1C76761C1C2425B765646D6D1B766D01
:100300006D5B09125B5C5B125B641213131B1212B0
:100310001C1C1C1C1C241C1C242525242425251BDA
:1003200000002513000064BF00096EBFBF6D6EBFE3
:100330006D5B12135B12131209000901000000002B
:100340002E1C0900096E010009767F7F12777F7FDE
:100350006412BF775B121B095B121B0900001B09AB
:10036000000000000000000000000000000000008D
:100370007F7F5313130064121B0100001B12000047
:10038000000000000000000000000000000000006D
:10039000000000000000000000000000000000005D
:1003A0000000000000002600000026002F000000D2
:1003B0002F00370000003700FF000000FF00BF00E3
:1003C0000000BF00370000370000002626000000B4
:1003D000000000000000262626262600000000005F
:1003E0002F000000003700000000FF00000000BFE9
:1003F0000000000037000000000026262626260008
:100400000000000000002626262626002F000000FF
:100410000000370000000000FFFFFFFF0000BF00EA
:1004200000000000370000000000262626262600D7
:100430000000000000002626262600002F000000F5
:100440002F00370000003700FFFFFFFF0000BF0054
:100450000000BF00370000003700262626260000D7
:10046000000000000000000026262600002F0000EB
:100470002F00370000003700FF000000FF00BF0022
:100480000000BF00370000370000262626000000CD
:100490000000000000002600000026002F000000E1
:1004A0002F000037003700000000FF00000000BFF1
:1004B00000BF0000370000003700260000002600C3
:1004C000000000000000000000000000000000002C
:1004D000000000000000000000000000000000001C
:1004E0000000009B000000529BA400005B9B6D7706
:1004F00000000000000000000000000000000000FC
:10050000005B000000E4F6FF099BEDF6FFBFA4AD21
:10051000BFBFBFBF767F7FB7B7BF7F766EB7B7BFAE
:1005200000000000000000005BB6F6F6F6FFFFFFDB
:10053000FFBFFFFFFFBFBFAEFFFFFFB7AD65FFFF10
:10054000B7B6AD65FFFFBFB7AE6EFFFFBFB7B7650C
:10055000000000000000F6F6EDEDADA4B66D6D5C98
:10056000526E6565655265765C5C52536E246552C9
:10057000526E25255B52772D2525526E6E2D252531
:10058000000000000000A49B9B4900006564A49B40
:1005900092006D2525649349656E652E9B52242536
:1005A0006D25655225246D2D655225256E2E6452CC
:1005B00000000000000000000000004A00000000F1
:1005C0005B9B0000005B5B2D0000525B2E2E000148
:1005D0005B2D1C01005C5B014A654A5B1C6E7F77EA
:1005E000495B9B77776D5B65776E65656D2D25251E
:1005F0005C522E25130949641C09095C7F7F091C84
:100600007F7F777F777F77777F7F7776777F7F6E44
:10061000656E6EA4B6FF655BA4B7BFFF526DBFBF2A
:10062000BFFF7FBFBFBFBFFFBFBFB7BFFFFF7FB76A
:10063000BFBFFFFF6EB7BFBFFFFF77BFBFBFFFFFEB
:10064000FFFFBFBFB75BFFFFBFBFA464FFFFBFAD2E
:10065000A47FFFFFBFA4BF7FFFBFADBFBFBFFFB67B
:10066000BFBFBF77F7BFBFBF7777FFBFBFBF6452C2
:100670006D7F6E2E2D2D7F766E6E6E2E7777777650
:100680002E1C7F776E251C25776525251C096E6E2F
:100690001C0949255B494A6E7F645377BF775B5CD1
:1006A000256E6E255B4A25651C1B5B002524245B9B
:1006B00053001C1B5B5C00000A5B64000000646468
:1006C000000000005C0000000000000000000000CE
:1006D0005B5C7FBF77765C6D7FB777775C6D7FBF44
:1006E00077775C64BFBFBFBF0A5C6EBFBFBF0065EA
:1006F000646DBFBF00005B6D646D00000000125BA5
:100700007777777F6E6E77777F766D7677BF776D49
:100710006E76BF7F6D6E767FBF7676BFBF76BFBFCA
:10072000BFB664ADADB6B6ADBFFF646DADB6AD647A
:1007300077BFBFBFFFFF77BFBFBFFFFF7FBFBFBF99
:10074000FFF6BFB7ADF6FFFFA4ADFFFFFFFFFFFF52
:10075000FFFFFFFFFFFFFFF6A4005B520000000059
:10076000BFBFAD5B64BFB6ADADBFFFBFFFFFFFFF57
:10077000BF64FFFFBFB6765BFFBFBF5B0000FF5CDF
:100780000000000000000000000000000000000069
:10079000BFBF645C5C006E5C654900006D5B00007F
:1007A0000000000000000000000000000000000049
:1007B0000000000000000000000000000000000039
:1007C0000600040000000100020003000400050010
:1007D00006000700080009000A000B000C000D00CD
:1007E0000E000F0010000000110012001300140092
:1007F000150016000600030000001700180019007D
:100800001A001B001C001D001E001F0020002100FC
:10081000220023002400250026000000000002081A
:1008200000085504085A0000F8000990000A1E321A
:10083000050000FF1C080000000100020003000486
:10084000000501000101010201030104010502008C
:100850000201020202030204020503000301030273
:100860000303030403050400040104020403040455
:10087000040505000501050205030504050506003C
:100880000601060206030604060507000701070223
:100890000703070407050800080108020803080405
:1008A00008050900090109020903090409050A00EC
:1008B0000A010A020A030A040A050B000B010B02D3
:1008C0000B030B040B050C000C010C020C030C04B5
:1008D0000C050D000D010D020D030D040D050E009C
:1008E0000E010E020E030E040E050F000F010F0283
:1008F0000F030F040F051000100110021003100465
:10090000100511001101110211031104110512004B
:100910001201120212031204120513001301130232
:100920001303130413051400140114021403140414
:1009300014051500150115021503150415051600FB
:1009400016011602160316041605170017011702E2
:1009500017031704170518001801180218031804C4
:1009600018051900190119021903190419051A00AB
:100970001A011A021A031A041A051B001B011B0292
:100980001B031B041B051C001C011C021C031C0474
:100990001C051D001D011D021D031D041D051E005B
:1009A0001E011E021E031E041E051F001F011F0242
:1009B0001F031F041F0500C00300B0070000C00391
:1009C00000B0075800C10900B1070000C10900B11B
:1009D000077300C21000B2070000C21000B2076126
:1009E00000C30000B3077200C30000B307280190E2
:1009F000286D0091465E0093071D1391435E00939E
:100A0000073203B2074D1090236D0091465E0092AD
:100A10004764009307481491475E00924067009333
:100A200007351390286D0091435F009307211391C0
:100A3000425F0093073313902B6D0091406000924A
:100A4000436C0093074813072F1490276D009143C0
:100A50006000930720139142610093072C139023A9
:100A60006D00913F610092426D0093074813072E7D
:100A70001390286D009143610093071E1491426109
:100A80000093073013902B6D0091406100924370EA
:100A900000930748139143610093072C1390286D2E
:100AA000009146610093071D139143600093073244
:100AB0001490236D009146600092406C00930748AB
:100AC0001391476000924071009307351390286D91
:100AD0000091436000930721139142600093073314
:100AE00013902B6D009140600092476C0093074873
:100AF00014072F13902A6D00914260009307201372
:100B00009140600093072C1390276D00913F600087
:100B10009242700093074813072E1390236D0091A3
:100B20004062009243460093071E1407301390273B
:100B30006D009243540093074813072C1390286DBF
:100B40000093071D1307321490236D0092406C0030
:100B500093074813924070009307351390286D0057
:100B600093072113073313902B6D00924771009365
:100B7000074814072F1390276D0093072013072CA5
:100B80001390236D009247700093074813072E14AB
:100B900090286D00914F440093071E13914E44001E
:100BA00093073013902B6D00914C450092436C00DD
:100BB00093074813914E450093072C0A914F45091E
:100BC00090286D009152450093071D13914F4500E9
:100BD0009307321490236D009152450092476400B0
:100BE00093074813915345009240730093073513C0
:100BF00090286D00914F460093072113914E4700B6
:100C000093073313902B6D00914C47009243730070
:100C100093074814072F13902A6D00914E470093B5
:100C2000072013914C470093072C1390276D0091D8
:100C30004B47009242700093074813072E149023ED
:100C40006D00914C4F009247730093071E130730BD
:100C50001390276D0093074813072C1390286D00FD
:100C600093071D1407321390236D00924361009384
:100C7000074813924759009307351390286D009346
:100C8000072113073314902B6D0092426A009307DB
:100C90004813072F1390276D0093072013072C1379
:100CA00090236D009240710093074813072E149013
:100CB000286D0093071E13073013902B6D0092428E
:100CC0005900930748139243350093072C1390283B
:100CD0006D0093071D1407321390236D00924C5939
:100CE0000093074813924F64009307351390286DC3
:100CF0000093072113073314902B6D009247670070
:100D000093074813072F13902A6D009307201307AA
:100D10002C1390276D00924B3E0093074814072E2A
:100D20001390236D009243750093071E1307301331
:100D300090276D0093074813072C1490286D00939B
:100D4000071D1307321390236D0092435900930738
:100D50004813924061009307351390286D00930764
:100D60002113073314902B6D0092407100930748B4
:100D700013072F1390276D0093072013072C139050
:100D8000236D009242680093074814072E139028A1
:100D90006D0093071E13073013902B6D009243676D
:100DA000009307481392434A0093072C1490286D30
:100DB0000093071D1307321390236D00924F5300C9
:100DC0009307481392475E009307351390286D00F0
:100DD00093072114073313902B6D0092426D0093FB
:100DE000074813072F1390286D00924C6400930757
:100DF0002013072C13914C7D0093074814072E13E2
:100E0000914E7D0093071E13073013914F7E009380
:100E1000074813072C1490286D00914F6400930726
:100E20001D1307321390236D009247640093074807
:100E300013924067009307351390286D00914E641C
:100E40000093072114073313902B6D0092436C001D
:100E500093074813072F1390276D00914C6400935C
:100E6000072013072C1490236D00924B70009307FA
:100E70004813072E1390286D0093071E1307301395
:100E8000902B6D009243700093074814072C139029
:100E9000286D00914F640093071D130732139023B0
:100EA0006D0092406C0093074813924770009307BF
:100EB000351390286D00914E640093072114073379
:100EC00013902B6D00924C6C0093074813914C6467
:100ED0000093072F0A914E6409902A6D00914B648C
:100EE0000093072013072C1490276D009242700086
:100EF00093074813072E1390236D00924E4A0093D8
:100F0000071E1307301390276D00924F4C00930774
:100F10004814072C1390286D00914F640093071D0F
:100F20001307321390236D0092406C00930748130F
:100F3000924070009307351490286D00914E640024
:100F400093072113073313902B6D00924771009381
:100F5000074813072F1390276D00915364009307E0
:100F60002014072C1390236D00924B7000930748B8
:100F700013072E1390286D0093071E13073013904C
:100F80002B6D0092436C0093074814072C13902894
:100F90006D00914B640093071D13914C64009307FF
:100FA000321390236D00914B6400924073009307BD
:100FB0004813914C640092476400930735149028BD
:100FC0006D00914F640093072113073313902B6D2D
:100FD0000091476400924C6C0093074813072F134D
:100FE000902A6D00914C640093072014072C1390F5
:100FF000276D00914B6400924270009307481307DD
:101000002E1390236D00914C640092477300930758
:101010001E1307301490276D0093074813072C13F5
:1010200090286D00914F640093071D1307321390B1
:10103000236D00924061009307481492406700932B
:1010400007351390286D00914E6400930721130714
:101050003313902B6D009247640093074813072FBA
:101060001390276D00914C640093072014072C13F4
:1010700090236D0092426D0093074813072E139042
:10108000286D0093071E13073014902B6D009243B8
:10109000700093074813072C1390286D00914F643C
:1010A0000093071D1307321390236D0092406C00CC
:1010B0009307481492436C009307351390286D00F2
:1010C000914E640093072113073313902B6D009208
:1010D0004C6C0093074813914C640093072F0A91BE
:1010E0004E640A902A6D00914B6400930720130709
:1010F0002C1390276D00924B700093074813072E16
:101100001390236D00924E4A0093071E130730146C
:1011100090276D0092494B0093074813072C1390BA
:10112000286D00914F640093071D1307321390231D
:101130006D00924767009307481492407000930730
:10114000351390286D00914E6400930721130733E7
:1011500013902B6D00924C4A0093074813072F14ED
:1011600090276D009153640093072013072C139070
:10117000236D009242720093074813072E139028A4
:101180006D0093071E14073013902B6D0092436C73
:101190000093074813072C1390286D00914B6400AF
:1011A00093071D13914C64009307321490236D0034
:1011B000914B64009240730093074813914C640074
:1011C000924073009307351390286D00914F64008F
:1011D00093072113073313902B6D009147640092FE
:1011E00043730093074813072F14902A6D00914C06
:1011F000640093072013072C1390276D00914B6414
:10120000009242700093074813072E1390236D003D
:10121000914C64009240710093071E1407301390A4
:10122000276D0093074813072C1390236C00922F0F
:101230006C0093071D1307321490266700923267E3
:10124000009307481307351390256D0092316D0008
:101250009307211307331390236100922F610093AA
:10126000074814072F1390266700923267009307F0
:101270002013072C13902A6A0092366A00930748BD
:1012800013072E14902B6C0092376C0093071E13DB
:1012900007301390266400923264009307481307C6
:1012A0002C1390236400922F640093071D130732C0
:1012B0001490266C0092326C009307481307351384
:1012C00090256D0092316D00930721130733139021
:1012D000236400922F640093074814072F13902B68
:1012E00070009237700093072013072C13902A6D1B
:1012F0000092366D0093074813072E14902B6C0054
:1013000092376C0093071E130730139026700092DB
:1013100032700093074813072C1390236C00922F10
:101320006C0093071D1407321390267000923270E0
:10133000009307481307351390256D0092316D0017
:101340009307211307331390236C00922F6C0093A3
:10135000074814072F1390267000923270009307ED
:101360002013072C13902A6D0092366D00930748C6
:1013700013072E14902B6C0092376C0093071E13EA
:1013800007301390267000923270009307481307BD
:101390002C13902C6D0092386D0093071D140732AA
:1013A0001390276A0092336A009307481307351396
:1013B0009026700092327000930721130733149027
:1013C000237000922F700093074813072F13902764
:1013D0006D0092336D0093072013072C1390266C39
:1013E0000092326C0093074814072E13902C6A0069
:1013F00092386A0093071E130730139027700092EB
:1014000033700093074813072C1390236700922F23
:10141000670093071D14073213902664009232640C
:10142000009307481307351390256D0092316D0026
:101430009307211307331490236400922F640093C1
:10144000074813072F13902667009232670093070F
:101450002013072C13902A630092366300930748E9
:1014600014072E13902B6C0092376C0093071E13F9
:1014700007301390266400923264009307481307E4
:101480002C14902B67009237670093071D130732C7
:1014900013902664009232640093074813073513B3
:1014A00090226A00922E6A0093072114073313904A
:1014B000215900922D590093074813072F13902BA1
:1014C00067009237670093072013072C13902E5D57
:1014D00000923A5D0093074814072E13902664008B
:1014E0009232640093071E13073013902B71009201
:1014F00037710093074813072C1490236100922F33
:10150000610093071D130732139026640092326422
:10151000009307481307351390256D0092316D0035
:101520009307211407331390236400922F640093D0
:10153000074813072F13902667009232670093071E
:101540002013072C14902A6A0092366A00930748E9
:1015500013072E13902B67009237670093071E1313
:101560000730139026670092326700930748139163
:101570004E640093072C0A914F640A9023670091F0
:10158000526400922F670093071D139153640093D8
:1015900007321390266400915264009232640093E3
:1015A000074813915364009307351390256A0091FF
:1015B0004E640092316A0093072114914F640093A6
:1015C00007331390236400914E6400922F640093BC
:1015D000074813914F640093072F139023610091E4
:1015E0004B6400923B61003B61003B61009307202C
:1015F00013914C640093072C14901F5600914B6478
:1016000000923761003761003761009307481391FA
:101610004C640093072E1390235600914E64009261
:101620003B61003B61003B610093071E13073013D1
:1016300090225500914F6400923A61003A61003A5D
:1016400061009307481490235500923B61003B6171
:10165000003B610093072C1390286D00914F6400AC
:1016600093071D1307321390236D0092406100937E
:10167000074813924067009307351490286D009136
:101680004E640093072113073313902B6D00924390
:101690006C0093074813072F1390276D00914C643B
:1016A0000093072013072C1490236D0092426D00C5
:1016B00093074813072E1390286D0093071E1307F6
:1016C0003013902B6D009243700093074814072C41
:1016D0001390286D00914F640093071D1307321378
:1016E00090236D0092406C00930748139240710064
:1016F0009307351490286D00914E640093072113D1
:10170000073313902B6D0092436C0093074813919D
:101710004C640093072F0A914E6409902A6D009142
:101720004B640093072014072C1390276D009242FE
:10173000700093074813072E1390236D00924346C1
:101740000093071E1307301490276D009243540036
:1017500093074813072C1390286D00914F64009352
:10176000071D1307321390236D0092406C009307FE
:101770004813924070009307351490286D00914EE5
:10178000640093072113073313902B6D0092436C71
:101790000093074813072F1390276D00915364009F
:1017A00093072014072C1390236D0092427200932C
:1017B000074813072E1390286D0093071E13073058
:1017C00014902B6D0092436C0093074813072C1361
:1017D00090286D00914B640093071D13914C640099
:1017E0009307321390236D00914B64009240730075
:1017F00093074814914C640092407300930735138B
:1018000090286D00914F64009307211307331390C4
:101810002B6D0091476400924373009307481307B0
:101820002F13902A6D00914C640093072014072C0D
:101830001390276D00914B6400924270009307480B
:1018400013072E1390236D00914C64009240710099
:1018500093071E1307301490276D00930748130752
:101860002C1390286D0093071D1307321390236DDE
:101870000092406700930748149240670093073531
:101880001390286D0093072113073313902B6D00DD
:101890009240700093074813072F1490276D009310
:1018A000072013072C13901F640092494A009307E6
:1018B0004813924A470093072E13901E63009249E3
:1018C000440093071E14924A4B0093073013901F55
:1018D00064009249470093074813924A44009307D3
:1018E0002C13902364009249440093071D13924ADD
:1018F000470093073213901F640092494A009307F0
:101900004814924A4B009307351390236400924980
:101910004A0093072113924A4700930733139027F5
:10192000680092494F0093074813924A4700930773
:101930002F14902A6A00924E530093072013924F5F
:101940004B0093072C13902B6C00924A3F00930797
:10195000481392494F0093072E1390266C0092472C
:101960004D0093071E14924A4400930730139025AC
:101970006D00924940009307481392474B0093072C
:101980002C13902B6C009249440093071D13924A2C
:10199000440093073214901F590092494A0093075C
:1019A0004813924A470093073513902B6C009249D5
:1019B000470093072113924A470093073313902758
:1019C0005D009249470093074814924A4B009307E1
:1019D0002F13902B4F009249470093072013924AF0
:1019E000470093072C13901F530092494700930719
:1019F0004813924A4B0093072E13902B670092498D
:101A0000470093071E14924A470093073013901F14
:101A100056009249470093074813924A4B00930798
:101A20002C13902B67009249440093071D13924A90
:101A30004B0093073214901F5300924953009307B1
:101A40004813924A44009307351390266100924947
:101A5000470093072113924A4700930733139027B7
:101A600068009249470093074814924A4700930739
:101A70002F13902A5D00924E4F0093072013924F30
:101A80004D0093072C13902B6400924A4D0093074E
:101A9000481392494A0093072E14902664009252EC
:101AA0004A0093071E1392534B009307301390255F
:101AB0007000924F4D0093074813924E57009307C2
:101AC0002C13902364009249400093071D13924AFF
:101AD0003F0093073214901F59009249400093072A
:101AE0004813924A440093073513902361009249AA
:101AF0004F0093072113924A440093073313902712
:101B000068009249440093074814924A440093079E
:101B10002F13902367009249440093072013924AA1
:101B2000470093072C13901F640092494A009307C3
:101B30004813924A470093072E14901E630092495F
:101B4000440093071E13924A4B0093073013901FD3
:101B500064009249470093074813924A4400930750
:101B60002C13902364009249440093071D14924A59
:101B7000470093073213901F640092494A0093076D
:101B80004813924A4B0093073513902364009249FF
:101B90004A0093072113924A470093073314902772
:101BA000680092494F0093074813924A47009307F1
:101BB0002F13902A6A00924E530093072013924FDE
:101BC0004B0093072C13902B6C00924A3F00930715
:101BD000481392494F0093072E1490266C009247A9
:101BE0004D0093071E13924A44009307301390252B
:101BF0006D00924940009307481392474B009307AA
:101C00002C13902B6C009249440093071D14924AA8
:101C1000440093073213901F590092494A009307DA
:101C20004813924A470093073513902B6C00924952
:101C3000470093072113924A4700930733149027D4
:101C40005D009249470093074813924A4B0093075F
:101C50002F13902B4F009249470093072013924A6D
:101C6000470093072C13901F530092494700930796
:101C70004814924A4B0093072E13902B6700924909
:101C8000470093071E13924A470093073013901F93
:101C900056009249470093074813924A4B00930716
:101CA0002C14902B67009249440093071D13924A0D
:101CB0004B0093073213901F530092495300930730
:101CC0004813924A440093073513902661009249C5
:101CD000470093072113924A470093073314902734
:101CE00068009249470093074813924A47009307B8
:101CF0002F13902A5D00924E4F0093072013924FAE
:101D00004D0093072C13902B6400924A4D009307CB
:101D1000481492494A0093072E1390266400925269
:101D20004A0093071E1392534B00930730139025DC
:101D30007000924F4D0093074813924E570093073F
:101D40002C14902364009249400093071D13924A7B
:101D50003F0093073213901F5900924940009307A8
:101D60004813924A44009307351390236100924927
:101D70004F0093072114924A44009307331390278E
:101D800068009249440093074813924A440093071D
:101D90002F13902367009249440093072013924A1F
:101DA000470093072C13901F640092494A00930741
:101DB0004814924A470093072E13901E63009249DD
:101DC000440093071E13924A4B0093073013901F51
:101DD00064009249470093074813924A44009307CE
:101DE0002C14902364009249440093071D13924AD7
:101DF000470093073213901F640092494A009307EB
:101E00004813924A4B00930735139023640092497C
:101E10004A0093072114924A4700930733139027EF
:101E2000680092494F0093074813924A470093076E
:101E30002F13902A6A00924E530093072013924F5B
:101E40004B0093072C14902B6C00924A3F00930791
:101E5000481392494F0093072E1390266C00924727
:101E60004D0093071E13924A4400930730139025A8
:101E70006D00924940009307481492474B00930726
:101E80002C13902B6C009249440093071D13924A27
:101E9000440093073213901F590092494A00930758
:101EA0004813924A470093073513902B6C009249D0
:101EB000470093072114924A470093073313902752
:101EC0005D009249470093074813924A4B009307DD
:101ED0002F13902B4F009249470093072013924AEB
:101EE000470093072C14901F530092494700930713
:101EF0004813924A4B0093072E13902B6700924988
:101F0000470093071E13924A470093073013901F10
:101F100056009249470093074814924A4B00930792
:101F20002C13902B67009249440093071D13924A8B
:101F30004B0093073213901F5300924953009307AD
:101F40004813924A44009307351490266100924941
:101F5000470093072113924A4700930733139027B2
:101F600068009249470093074813924A4700930735
:101F70002F13902A5D00924E4F0093072014924F2A
:101F80004D0093072C13902B6400924A4D00930749
:101F9000481392494A0093072E13902664009252E8
:101FA0004A0093071E1392534B009307301390255A
:101FB0007000924F4D0093074814924E57009307BC
:101FC0002C13902364009249400093071D13924AFA
:101FD0003F0093073213901F590092494000930726
:101FE0004813924A440093073514902361009249A4
:101FF0004F0093072113924A44009307331390270D
:1020000068009249440093074813924A440093079A
:102010002F13902367009249440093072014924A9B
:10202000470093072C13901F640092494A009307BE
:102030004813924A470093072E13901E630092495B
:10204000440093071E13924A4B0093073014901FCD
:1020500064009249470093074813924A440093074B
:102060002C13902364009249440093071D13924A55
:10207000470093073213901F640092494A00930768
:102080004814924A4B0093073513902364009249F9
:102090004A0093072113924A47009307331390276E
:1020A000680092494F0093074813924A47009307EC
:1020B0002F13902A6A00924E530093072014924FD8
:1020C0004B0093072C13902B6C00924A3F00930710
:1020D000481392494F0093072E1390236C009247A8
:1020E0004D0093071E13073014074813072C139055
:1020F000286D0091465E0093071D1391435E009387
:10210000073203B2074D1090236D0091465E009296
:102110004061009307481491475E00924067009326
:1021200007351390286D0091435F009307211391A9
:10213000425F0093073313902B6D00914060009233
:10214000436C0093074813072F1490276D009143A9
:102150006000930720139142610093072C13902392
:102160006D00913F610092426D0093074813072E66
:102170001390286D009143610093071E13914261F3
:102180000093073014902B6D0091406100924370D2
:1021900000930748139143610093072C1390286D17
:1021A000009146610093071D13914360009307322D
:1021B0001390236D009146600092406C0093074895
:1021C0001491476000924071009307351390286D79
:1021D00000914360009307211391426000930733FD
:1021E00013902B6D009140600092436C0093074860
:1021F00013072F14902A6D0091426000930720135B
:102200009140600093072C1390276D00913F600070
:102210009242700093074813072E1390236D00918C
:102220004062009243460093071E14073013902724
:102230006D009243540093074813072C1390286DA8
:102240000093071D1307321490236D0092406C0019
:1022500093074813924070009307351390286D0040
:1022600093072113073313902B6D0092436C009357
:10227000074813072F1490276D0093072013072C8E
:102280001390236D009242720093074813072E1398
:1022900090286D00914F440093071E14914E440006
:1022A00093073013902B6D00914C450092436C00C6
:1022B00093074813914E450093072C0A914F450907
:1022C00090286D009152450093071D13914F4500D2
:1022D0009307321490236D00915245009240730091
:1022E00093074813915345009240730093073513A9
:1022F00090286D00914F460093072113914E47009F
:1023000093073313902B6D00914C47009243730059
:1023100093074814072F13902A6D00914E4700939E
:10232000072013914C470093072C1390276D0091C1
:102330004B47009242700093074813072E149023D6
:102340006D00914C4F009240710093071E130730AF
:102350001390276D0093074813072C1390286D00E6
:1023600093071D1307321490236D0092406700936A
:10237000074813924067009307351390286D009328
:10238000072113073313902B6D00924370009307BE
:102390004814072F1390276D0093072013072C1361
:1023A00090236D009240710093074813072E1490FC
:1023B000286D0093071E13073013902B6D00924376
:1023C0007300930748139243350093072C1390280A
:1023D0006D0093071D1407321390236D00924F5E1A
:1023E0000093074813924F64009307351390286DAC
:1023F0000093072113073313902B6D0092422D0099
:1024000093074814072F13902A6D00930720130792
:102410002C1390276D00924B3E0093074813072E14
:102420001490236D00924C4E0093071E1307301337
:1024300090276D0093074813072C1390286D009385
:10244000071D1407321390236D0092406C00930710
:102450004813924061009307351390286D0093074D
:102460002113073314902B6D0092426800930748A4
:1024700013072F1390276D0093072013072C139039
:10248000236D009240700093074814072E13902884
:102490006D0093071E13073013902B6D00930748B0
:1024A0001392434A0093072C1390286D0093071D45
:1024B0001407321390236D00924F53009307481373
:1024C000924F61009307351390286D0093072113F5
:1024D000073314902B6D0092426D00930748130749
:1024E0002F1390286D00924C640093072013072C43
:1024F00013914C7D0093074814072E13914E7D00D5
:1025000093071E13073013914F7E0093074813075C
:102510002C1490286D00914F640093071D1307320F
:102520001390236D00924764009307481392476C01
:10253000009307351390286D00914E640093072196
:1025400014073313902B6D00924C6C0093074813C3
:10255000072F1390276D00914C64009307201307F9
:102560002C1390236D0092426D0093074814072EA0
:102570001390286D0093071E13073013902B6D00E6
:102580009243700093074813072C1490286D009114
:102590004F640093071D1307321390236D00924779
:1025A0005E009307481392477000930735139028F5
:1025B0006D00914E640093072114073313902B6D27
:1025C00000924C6C0093074813914C640093072FC2
:1025D0000A914E6409902A6D00914B640093072084
:1025E00013072C1490276D00924270009307481334
:1025F000072E1390236D009243460093071E130786
:10260000301390276D009243540093074813072C12
:102610001490286D00914F640093071D1307321327
:1026200090236D00924767009307481392476C0010
:102630009307351390286D00914E64009307211481
:10264000073313902B6D0092436C009307481307D8
:102650002F1390276D009153640093072013072CCC
:102660001490236D009242720093074813072E13B3
:1026700090286D0093071E13073013902B6D009266
:10268000436C0093074814072C1390286D00914B5E
:10269000640093071D13914C640093073213902339
:1026A0006D00914B64009240730093074813914C66
:1026B0006400924073009307351490286D00914F89
:1026C000640093072113073313902B6D0091476427
:1026D000009243730093074813072F13902A6D004D
:1026E000914C640093072013072C1490276D0091E0
:1026F0004B64009242700093074813072E139023F7
:102700006D00914C64009240710093071E130730D6
:102710001390276D0093074814072C1390286D0021
:10272000914F640093071D1307321390236D00929D
:102730004061009307481392406700930735149057
:10274000286D00914E640093072113073313902BDB
:102750006D0092436C0093074813072F1390276D69
:1027600000914C640093072014072C1390236D00F4
:1027700092426D0093074813072E1390286D009323
:10278000071E13073014902B6D00924370009307BF
:102790004813072C1390286D00914F640093071D78
:1027A0001307321390236D0092406C009307481377
:1027B000924071009307351490286D00914E64008B
:1027C00093072113073313902B6D0092436C0093F2
:1027D000074813914C640093072F0A914E640990A7
:1027E0002A6D00914B640093072014072C13902747
:1027F0006D009242700093074813072E1390236DCB
:10280000009243460093071E1307301490276D0073
:102810009243540093074813072C1390286D00919E
:102820004F640093071D1307321390236D009240ED
:102830006C0093074814924070009307351390285A
:102840006D00914E640093072113073313902B6D95
:102850000092436C0093074813072F1390276D00D5
:102860009153640093072014072C1390236D00925A
:1028700042720093074813072E1390286D009307A8
:102880001E13073014902B6D0092436C0093074881
:1028900013072C1390286D00914B640093071D13B0
:1028A000914C64009307321390236D00914B6400A8
:1028B0009240730093074814914C64009240730057
:1028C0009307351390286D00914F640093072113EF
:1028D000073313902B6D009147640092437300936C
:1028E000074813072F14902A6D00914C640093073A
:1028F0002013072C1390276D00914B6400924270B7
:102900000093074813072E1390236D00914C640029
:102910009240710093071E1407301390276D0093A7
:10292000074813072C1390236C00922F6C00930719
:102930001D130732139026670092326700930748F1
:102940001407351390256D0092316D009307211304
:1029500007331390236100922F61009307481307F8
:102960002F14902667009232670093072013072CDC
:1029700013902A6A0092366A0093074813072E13B1
:10298000902B6C0092376C0093071E140730139045
:102990002664009232640093074813072C13902397
:1029A0006400922F640093071D1307321490266C65
:1029B0000092326C009307481307351390256D0081
:1029C00092316D0093072113073313902364009213
:1029D0002F640093074814072F13902B7000923731
:1029E000700093072013072C13902A6D0092366D08
:1029F0000093074813072E13902B6C0092376C003E
:102A000093071E14073013902670009232700093C3
:102A1000074813072C1390236C00922F6C00930728
:102A20001D130732149026700092327000930748ED
:102A30001307351390256D0092316D009307211314
:102A400007331390236C00922F6C009307481407F0
:102A50002F13902670009232700093072013072CDA
:102A600013902A6D0092366D0093074813072E14B9
:102A7000902B6C0092376C0093071E130730139055
:102A80002670009232700093074813072C13902C85
:102A90006D0092386D0093071D1307321490276A5A
:102AA0000092336A0093074813073513902670008D
:102AB0009232700093072113073313902370009212
:102AC0002F700093074814072F1390276D0092333F
:102AD0006D0093072013072C1390266C0092326C24
:102AE0000093074813072E14902C6A0092386A004E
:102AF00093071E13073013902770009233700093D2
:102B0000074813072C1390236700922F6700930741
:102B10001D14073213902664009232640093074814
:102B20001307351390256D0092316D009307211323
:102B300007331490236400922F640093074813070F
:102B40002F13902667009232670093072013072CFB
:102B500013902A63009236630093074813072E14DC
:102B6000902B6C0092376C0093071E130730139064
:102B70002664009232640093074813072C13902BAD
:102B800067009237670093071D140732139026647D
:102B900000923264009307481307351390226A00AD
:102BA000922E6A0093072113073314902159009243
:102BB0002D590093074813072F13902B6700923766
:102BC000670093072013072C13902E5D00923A5D47
:102BD0000093074814072E13902664009232640075
:102BE00093071E13073013902B71009237710093D7
:102BF000074813072C1490236100922F610093075C
:102C00001D13073213902664009232640093074824
:102C10001307351390256D0092316D009307211332
:102C200007331490236400922F640093074813071E
:102C30002F13902667009232670093072013072C0A
:102C400013902A6A0092366A0093074814072E13DD
:102C5000902B67009237670093071E13073013907D
:102C60002667009232670093074813914E640093E1
:102C7000072C0A914F640A902367009152640092D6
:102C80002F670093071D139153640093073213902D
:102C900026640091526400923264009307481391B5
:102CA0005364009307351390256A00914E64009297
:102CB000316A0093072114914F64009307331390F6
:102CC000236400914E6400922F640093074813918F
:102CD0004F640093072F1390236100914B6400927F
:102CE0003B61003B61003B610093072013914C6402
:102CF0000093072C13901F5600914B64009237618C
:102D00000037610037610093074814914C640093C9
:102D1000072E1390235600914E6400923B61003BB6
:102D200061003B610093071E13073013902255008A
:102D3000914F6400923A61003A61003A6100930752
:102D4000481390235500923B61003B61003B6100BA
:102D500093072C1490286D00914F640093071D1366
:102D600007321390236D009240610093074813923D
:102D70004067009307351390286D00914E640093CF
:102D8000072114073313902B6D0092436C009307B7
:102D90004813072F1390276D00914C640093072070
:102DA00013072C1490236D0092426D009307481373
:102DB000072E1390286D0093071E13073013902BD6
:102DC0006D009243700093074814072C1390286DF0
:102DD00000914F640093071D1307321390236D0079
:102DE00092406C009307481392407100930735138B
:102DF00090286D00914E64009307211407331390BF
:102E00002B6D0092436C0093074813914C64009320
:102E1000072F0A914E6409902A6D00914B6400932C
:102E2000072013072C1490276D009242700093071F
:102E30004813072E1390236D009243460093071EFC
:102E40001307301390276D009243540093074814E2
:102E5000072C1390286D00914F640093071D1307F2
:102E6000321390236D0092406C00930748139240F8
:102E700070009307351490286D00914E64009307FD
:102E80002113073313902B6D0092436C0093074876
:102E900013072F1390276D0091536400930720149C
:102EA000072C1390236D009242720093074813077A
:102EB0002E1390286D0093071E13073013902B6D6F
:102EC0000092436C0093074814072C1390286D0060
:102ED000914B640093071D13914C640093073213C8
:102EE00090236D00914B6400924073009307481348
:102EF000914C6400924073009307351490286D0044
:102F0000914F640093072113073313902B6D0091A9
:102F1000476400924C6C0093074813072F13902AC4
:102F20006D00914C640093072014072C1390276DBB
:102F300000914B64009242700093074813072E13D0
:102F400090236D00914C64009240710093071E1312
:102F500007301490276D0093074813072C1390280F
:102F60006D0093071D1307321390236D0092406785
:102F70000093074813924067009307351490286D1B
:102F80000093072113073313902B6D0092407000BC
:102F900093074813072F1390276D009307201407FA
:102FA0002C1390236D009240710093074813072E55
:102FB0001390286D0093071E13073014902B6D009B
:102FC000930748139243350093072C1390286D0004
:102FD00093071D1307321390236D00924719009336
:102FE00007481492471E009307351390286D0093ED
:102FF000072113073313902B6D0092422D00930786
:103000004813072F14902A6D0093072013072C13E1
:1030100090276D009243640093074813072E139086
:10302000236D0092476C0093071E130730149027FE
:103030006D0093074813072C1390286D0093071D0C
:103040001307321390236D009243590093074814DD
:1030500092475E009307351390286D009307211364
:10306000073313902B6D00924268009307481307B3
:103070002F1490276D0093072013072C1390236DB6
:10308000009240700093074813072E1390286D009C
:1030900093071E14073013902B6D0092407000931D
:1030A000074813072C1390286D0093071D13073250
:1030B0001490236D00924759009307481392475E7E
:1030C000009307351390286D0093072113073313DE
:1030D000902B6D0092426D0093074813072F1490B8
:1030E000286D0092406D0093074A26FF2F000000D4
:1030F00002060000FB00FF000000F405030C0504BD
:103100000C05030C05040C05050000FF0000FF0082
:103110000002090000F10400F900FF0100010A00AB
:1031200000E202010501010301010102050000FFA7
:10313000000000E702030C04050000FF000000F19E
:1031400000085A02040302040402040502040602F1
:10315000050000FF010001010007900000E20805E2
:103160000000FF000002080107C80106000100E797
:1031700000FF010001000007A00000EC0100FE00BC
:10318000010100FF010001030000E2030106040148
:103190000903050000FF000002010107C801060045
:1031A0000100EC00FF000002040000F10400F9003F
:1031B000FF000002010000F100FF010000ED00012E
:1031C0000602010100FF010000EC000102010700FE
:1031D0000207FF00010300FF00000208000764016E
:1031E00000140500F700FF000002090000F100FFD5
:1031F000000002040000F800085003084E030854C1
:1032000002084C02085802084A01085C0000FC034E
:10321000086003085A03086003085A03086003089B
:103220005A01050000FF000002040000FB00083EF8
:10323000010302010302010302010302010302016F
:10324000040A010302010302010302010302010354
:10325000020104020103020103020103020103024D
:1032600001030201040A0103020103020103020136
:103270000302010302010405010302010302010329
:10328000020103020103020104050103020103021A
:10329000010302010302010302010405010302010B
:1032A000030201030201030201030201050000FF02
:1032B0000000020300085602040A02040802040681
:1032C000020404020402000842020305020402028E
:1032D00003050203050204020203050000F80403CB
:1032E000050404050403050404050403050404059A
:1032F00004030501050000FF000002040000FB00BC
:10330000083401030201030401030601040A010356
:103310000201030401030601040A0103020103047C
:10332000010306010405010302010304010306026F
:10333000030202030402030603040503030203035A
:10334000040303060404050403020403040403063F
:1033500001050000FF000007000402040007FF0051
:103360000990000A3C0000FB010850030305030418
:10337000050303050304050303050304050303050F
:103380000304050303050304050303050304050300
:10339000030503050000FF00000700040204000706
:1033A000FF000990000A3C0000FB010853030305DD
:1033B00003040503030503040503030503040503D0
:1033C00003050304050303050304050303050304C0
:1033D0000503030503050000FF00000700040204C5
:1033E0000007FF000990000A3C0000FB010856039B
:1033F0000305030405030305030405030305030490
:10340000050303050304050303050304050303057E
:1034100003040503030503050000FF000007000483
:1034200002040007FF000990000A3C0000FB0108AD
:1034300059030305030405030305030405030305FA
:10344000030405030305030405030305030405033F
:10345000030503040503030503050000FF00000244
:10346000020106000100E000FF0000020101060069
:103470000100E000FF000002080106000100E0007A
:10348000FF000002050106000100E000FF0000024D
:10349000090106000100E000FFEE30F7300C310FAB
:1034A000311B3130313C31543163317231843196CA
:1034B00031A531B131BA31C631D831E731F03126D9
:1034C00032B032F83255339733D9331B345D346917
:1034D00034753481348D3400000000000000000099
:1034E00000000000000000000000000000000000DC
:1034F00000000000000000000000000000000000CC
:10350000000000000000004A4A4A4A4A4A4A4A4A21
:103510004A4A4A4A4A4A4A4A4A4A4A4A4A4A4A4A0B
:103520004A4A4A4A4A4A4A4A4A4A4A4A4A4A4A4AFB
:103530004A4A4A4A4A4A4A4A4A4A4A4A4A4A4A41F4
:103540004A4A4A414A4A4A4A4A4A01414A4A4A4A36
:1035500000014A4A4A4A01014A4A4A4A01014A418B
:103560004A4A01014A014A4A4A4A4A4A4A4A414A9F
:103570004A4A4A41014A4A4A4A41414A4A014A4161
:10358000414A01014A41014A004A4A4101410001C0
:10359000014A000100414A4A4A4A4A4A4A4A4A4ABA
:1035A0004A4A4A4A4A4A4A4A524A4A4A4A4A644A59
:1035B0004A4A4A0A6D4A4A4A4A5BAE4A4A4A4A65F8
:1035C000AE4A4A4A006DAE096DADADAEAE64AEAD69
:1035D000ADADAD6DAEAEADAEAEAEAEAEAEADAEAE51
:1035E000ADAEAEAEAEAEAEADAEB6AEAEADAEAEAEF6
:1035F000AEADAEAEAEAEAEAEAEAEB6B6B6AEAEB6CC
:10360000B6B6B6AEAEB6B6B6B6AEAEB6B6B6B6AE82
:10361000AEB6B6B6B6AEAEB6B6B6B6AEAEB6B6B672
:10362000B6AEAEAEB6B6B664004A4A4A4AB6AD4A7F
:103630004A4A4AB6B60A4A4A4AB6B6AD4A4A4AB6AB
:10364000B6B6004A4AB6B6B65B4A4AB6B6B6AE4A4F
:103650004AB6B6B6B64A4A4A4A4A4A4A4A4A4A4A1A
:103660004A4A4A4A4A4A4A4A4A4A4A4A4A4A4A4ABA
:103670004A4A4A4A4A4A4A4A4A4A004A4A4A4A013D
:10368000004A4A4A0000004A4A4A4A4A4A4A4A4AC2
:103690004A4A4A4A4A4A4A4A4A4A4A4A4A4A4A4A8A
:1036A0004A4A4A4A4A414A4A4A4A4A01004A4A4A16
:1036B0004A0000004A4A4A4A4A4A4A4A4A4A4A4A48
:1036C000414A4A4A4A4A4A4A4A4A4A4A014A4A00F6
:1036D0004A4A004A4A00014A01414A000041004169
:1036E00041010000004A014A00014A014A4A000122
:1036F0004A01414A00004A014A4A000041004A4A40
:10370000000000014A4A010000414A014100004115
:10371000410141000041414A00004A4A4A4A000032
:103720004A4A4A4A00004A4A4A4A000041414A413C
:10373000000000414A4100000101014100004A4AE5
:103740004A0100414A4A4A4A4A4A4A4A4A4A4A4A75
:103750004A4A4A4A4A4A4A4A4A4A4A4A4A4A4A4AC9
:103760004A4A4A4A4A4A4A4A4A4A524A4A4A4A53A8
:10377000534A4A4A5253534A4A4A4A4A4A4A4A4A86
:103780004A4A4A4A4A4A4A4A4A4A4A4A4A4A4A4A99
:103790004A4A4A4A4A535B5353524A535353535328
:1037A000525353535253534A4A4A4A4A4A4A4A4A3C
:1037B0004A4A4A4A4A4A4A4A4A4A4A4A4A4A4A4A69
:1037C0004A4A4A4A4A4A4A4A4A4A4A4A4A4A4A5251
:1037D000535352535353534A4A4A4A4A4A4A4A4A0B
:1037E0004A4A4A4A4A4A4A4A4A4A4A4A4A4A4A4A39
:1037F0004A4A4A4A4A4A4A4A4A4A4A5353535353FC
:10380000535353535353534A4A4A4A4A4A4A4A4AD9
:103810004A4A4A4A4A4A4A4A4A4A4A4A4A52534AF7
:103820004A4A53535352535353535353535353537B
:10383000535253535353534A4A4A4A4A4A4A4A4AAA
:103840004A4A4A4A52525252535B53535353535368
:10385000535353535352535353535353535253533A
:10386000535353005353534A4A4A4A4A4A52535BAA
:103870005353535353535353535353535353535318
:103880005353535353535353535353535353535308
:10389000535353525353534A4A4A4A4A4A53524A39
:1038A0004A4A4A5353524A4A4A53535B4A4A4A5332
:1038B00053535353535353535352525353535353DA
:1038C000535353535353524A4A4A0AADAE4A4A4A93
:1038D0005BADAE4A4A4A64AEAE4A4A4A64AEAE53A3
:1038E00053535B5C5C5353535B5C5C5353535B5C63
:1038F0005C5353535C5C5CAEAEAEAEAEAEAEAEAE41
:10390000AEAEAEAEADAEAEAE5CADAEAE5C5C5C5C73
:103910005C5C5C5C5C5CA45C5C5C5C5C5C5C5C5C9F
:103920005C5C5C5C5C5C5CAEAEADB6B6B6AEAEAEDE
:10393000B6B6B65C5C5C5C64B6645C5CA4646464EF
:103940005C5C5C5C645C5C5C5C5C5C5C5C5C5C5CAF
:103950005C5C5C5C5C5C5CB6B6B6B6094AB6B6B696
:10396000B6124AB6B6B6B65B4A5CB6B6B6654A5C3F
:1039700064B6B6AE4A64645CB6B64A64645CB6B615
:103980004A5C6464645C4A4A4A4A4A4A4A4A4A4A25
:103990004A4A4A4A4A4A4A4A4A4A4A4A4A4A4A4A87
:1039A0004A4A4A4A4A4A4A4A4A4A4A4A4A4A4A4A77
:1039B0004A4A01004A4A4A4A4A4A0000004A4A4AD8
:1039C0000041004A4A4A414A004A4A4A4A4A004A91
:1039D0004A4A4A01004A4A4A4A01004A4A4A4A01B6
:1039E000004A4A4A4A00000100004A4A4A4A410045
:1039F0004A4A4A014A4A4A4A4A00014A4A4A4A004D
:103A0000014A4A4A4A00004A4A4A4A0000414A4A90
:103A10004A0000004A4A000000000041010941003C
:103A200000414109410100000100000000000009BF
:103A3000010000000009414A00000009414A00411C
:103A400000090001004A00014100004A4101410013
:103A5000014A010001000101000000000000000017
:103A600000014A01000000414A000000000141003D
:103A7000000000010100000100414A4A4A000041E3
:103A80004A414A00004141014A00004A520952009D
:103A90004A53524909005252520109414A4A4A01C5
:103AA00001414A4A4A00004A52524A4A4A4A52533B
:103AB000534A5252525352535352525252535352E8
:103AC000495252524A5201495249094A0152524AF4
:103AD0000141014A4A01014A4A5353535353535334
:103AE00053535353535253535353535353535352A8
:103AF00053535353535253525252534A53525253A5
:103B000052524A414A4A4A535353535353535353BD
:103B10005353535352535253535353525353525379
:103B20005353535252535353535352525253524A74
:103B30004A41414A41414A535353535353535353B8
:103B40005352535353525353535353535352535348
:103B500053535252535253535353534A4A52524A55
:103B60005241414141414153535353535352535294
:103B70005352535353535353525353525353535318
:103B8000525253525353535353535A52524A4A5216
:103B90005241414141414153535353535353535263
:103BA00053535353535352525353535352525352EA
:103BB00052535353535352525352524A4A4A4A4A07
:103BC0004A41414A414141535300535353535300D7
:103BD00053535353530052535353530009535253A7
:103BE0005300005252525200005252414100004ACA
:103BF0004A4A010909414A535352525353535352AB
:103C00005353535353535353535252535353535287
:103C10005253535B535352525353534A4A41414AAE
:103C20004A414141414141535353535353535353D9
:103C30005353535353535353535353535353535354
:103C400053525253535253535353534A4A53535359
:103C5000534A414A4A4A4A5353535C5C5C53535358
:103C60005C5C5C5353535C5C5C5353535B5C5C53D4
:103C70005353535C5C535353525C5C5353534A5CF1
:103C80005C4A4A4A4A64B65C5C5C5C5C5C5C5C5C5A
:103C90005C5C5C5C5C5C5C64645C5C5C5C5C5C5C54
:103CA0005C5C5C5C5C5C5C5C5C5C5C5C5C5C5C5C54
:103CB0005CAEB6B6B6B65C5C5C5C5C5C5C5C5C5C8A
:103CC0005C5C5C645C5C5C5C5C64645C5C645C640C
:103CD000645C5C646464645C5C5C645C645C5C5BED
:103CE0005C5C5C5CAEADAE5C5C64645B4A5C5C641A
:103CF000645B535B5B5C645B535C5C5C5B52535C1E
:103D00005C5B5B4A52645C5C5B525264AE5B5B52D0
:103D10004AB6AEAE124141525252524A4A535352DF
:103D200052524A53535353524A535352535352527B
:103D3000525353525352535A535352525252525255
:103D40004A4A4A41414A4A4A4A4A4A4A4A4A4A4AE5
:103D50004A4A4A4A4A4A4A4A4A4A4A4A4A4A4A4AC3
:103D60004A4A4A4A4A4A4A4A4A4A4A4A4A4A4A4AB3
:103D70004A4A4A4A4A4A4A4A4A4A4A4A4A4A4A4AA3
:103D80004A4A4A4A4A4A4A4A4A4A4A4A4A4A4A4A93
:103D90004A4A4A4A4A4A4A4A4A4A414A4A4A4A4A8C
:103DA000414A4A414A4A004A0000014A4A41000049
:103DB00000004A010009000041000909000041001B
:103DC0000909090041000909090001090909090057
:103DD000010909090900004A4A4A0100094A4A4AF8
:103DE0000009094A4A4A0009094A4A4A0009094A97
:103DF0004A4A0009094A4A41000909414141090961
:103E0000090000000909090900004A4A00090001E7
:103E10004A41000900004A41000900014A01000925
:103E2000000041000009090000000009090000002D
:103E300000090909090909000009414A410900006E
:103E4000414A41090000414141000900004101008F
:103E5000090000010009004100000009004A0000BB
:103E60000009014100000000000000000000000007
:103E700000000000000000000109000000004109EE
:103E800000000000410900000000410000000000A7
:103E9000410000000000000041414100014101419A
:103EA00001004A0100010100410100000000414100
:103EB0000000000001010000000000000000000000
:103EC000000000000000004101414A010141014A97
:103ED00041410941014A0141014101010001410102
:103EE000000000004100000000004100000001004F
:103EF000000000014100004A41414141414141412E
:103F00004141414A4A41414A414A41414A41414174
:103F1000414A41414A414A414A41410141414141AD
:103F200041000141414141414141414A4141414AF0
:103F300041414A4141414A4141414A414141414156
:103F400041414A41414A414A414A4141414141413D
:103F50004141414101414A414141414141414A417F
:103F600041414141414141414A4A41414A41414126
:103F7000414A4141414141414A4141414A41414A0D
:103F80004141414141414141414141414141414121
:103F90004141414141414141414141414141414111
:103FA0004141414141414141414141414141414101
:103FB00041414141414141414141414141414141F1
:103FC00041410141414A4141014109414101004111
:103FD00000414A01000100414A01000100014A007C
:103FE000000000014A0000410923084A004A09373D
:103FF000004A004A0123004A004A0108004A004AD8
:1040000001000041004A0100004108414100004117
:1040100000414100084100410041004141000009C8
:1040200000414100000900414A08230900414100C4
:1040300037000041410037000041010823000041E2
:1040400000000000014100414A414141414A4141D3
:10405000414A4141414A4141414A41414A414A4123
:1040600041414141414A41414141414A414A414125
:10407000414141414141414A41414152B6414141A1
:104080004A00AE4A4141414164414A4141410041F7
:10409000414141414141414A414141414A414141FE
:1040A0004A4A41414A4141B6AEAEB6B6B6B6AEAEE8
:1040B000B6B6B6B6B6B6B6B6B6B6B6B6B6B6B65CFA
:1040C000B6B6B6B6B641ADB6B6B6B6410053B6B69C
:1040D000B6414A4109ADAEB6B6AEAEADB6B6B6B6AD
:1040E000AEB6B6B6B6B6B6B6B6B6B6B6B6B6B6B678
:1040F000B6B6B6B6B6B6B6B6B6B6ADB6B6B6B6AD72
:1041000000B6B6AD5C0041B6B6AE00414AB6B66583
:10411000414141B6B609414141B6AD4141414164D9
:10412000094A414141004A414A4A414141414141D4
:104130004A4141414141524141414A524A4A4A4A17
:104140004A4A41414141414A49414152525200414A
:104150005252530000414141414101525252524199
:10416000415A53535A4A41014A4A4A4101004A4A74
:104170004A41000001004A41000000004A010000DD
:10418000014A41000000414A410000004141410014
:10419000000041410000094A4A010001004A4A0169
:1041A000000000014A09000000014A010000090066
:1041B0000100090909000009090909090909090992
:1041C000090909090909090909090909090909095F
:1041D000090909090909090909090909090909094F
:1041E000090909090909090909090909090909093F
:1041F0000909090909090909410000000000010035
:10420000000000000000000000000000000041006D
:10421000000009090000000009000900000909095F
:104220005209000900090000000000000000000021
:1042300000000000000000000041010000000052EA
:1042400052000000000912000000000909090000E6
:104250000900090000010900010900000000525393
:104260000000000052530900000812520900090022
:1042700001090000490000090900000000000909C7
:104280000009000000090900000941010000005276
:104290004A01000000525200010000090900414992
:1042A000000000495201000000525200000052522A
:1042B000520000005209000041414101010041410A
:1042C000410100004141414100414141410100495A
:1042D00001090100004949010000000149000909E4
:1042E00000000100525200414141014A094141018F
:1042F0000952094141010909014949520100495244
:104300000953000953090952000952005252000092
:104310004900524900004941414A4A4141525252E2
:1043200052524A525353535352525352525253526F
:1043300052535253525352535253525B5A535A533D
:10434000525A525252525A4141414141004A4A4105
:104350004141415252524141415253524A414153CB
:10436000525252525252525252525252525252522D
:1043700052525252525252000000010000000000FE
:104380000000000000000000000900000800000913
:1043900000000000000900000000004900000000CB
:1043A000005209000000004101090041000900001D
:1043B000004100000000004A010008000041010027
:1043C00000000000000000000000000000000008E5
:1043D0000000000000000008000041410000000053
:1043E0004A01000000014A000008000141000000ED
:1043F00000010100000800000000090000000800A2
:10440000000008000000004A4A4141414141414149
:1044100041414A0141414141410041414141410045
:1044200041414141410141414141410041414141FD
:10443000410041414141410909004141414141415E
:1044400041414141414141414141414141414A4153
:1044500041414152524141414A52524141414149F7
:104460005241414141414141414A525252414A5ACD
:104470005353534152520949534953090000525270
:1044800052090000495252090900495252010900DB
:10449000094A4A000900095352525352525251528A
:1044A000525253520952535353520000535249002F
:1044B000000052090000000009090909090000096B
:1044C000000909090009090041000909090000095A
:1044D0000909090109090909090009090909090066
:1044E000090909090909090909090909090909093C
:1044F00009090909090909090009095209090009F5
:1045000000410009090900410009090900000909E1
:10451000090909090909090909090909090909090B
:104520000909090909000809090000090909090020
:10453000000009090900000009090900000909092A
:10454000000000090908010000090908000000092D
:104550000908090000000909000000524909090979
:1045600000014109000900010909010000000009DA
:1045700001000000000001010000000041010900ED
:1045800000000100000000000000494A0000000097
:1045900001010001000041000000000001000000D6
:1045A0000000010000000000000001000000000009
:1045B00000000000000000000000524A000000005F
:1045C000410900000000010100000000000100019D
:1045D0000000000000410001000000010001000097
:1045E0000000000000000000090900094900010066
:1045F0000041010101000001010100000041010131
:104600000000014101010000010101000001010160
:104610000000000001010009494909495201014116
:1046200001410101010141010101010101010101FA
:10463000010101010101010101010101010101016A
:104640000101010101010149094149090901010172
:10465000010101010101010101010101010101014A
:10466000010101010101010101010101010101013A
:1046700001010101010101090900000000410100DF
:1046800000000001010000000001010000082301FA
:10469000010000093701010000083701010000088E
:1046A00023010100000000000000000000000000E5
:1046B00000000000000000000008000000000008EA
:1046C000000000002309000000003708000000007F
:1046D000370000000000080000000000000000009B
:1046E0000000010000000000410000000000410047
:1046F00000000000410000230000410000370000DE
:10470000410000370009414141414141414141419E
:104710004141414141414141414141414141414189
:1047200041414141414141414101014141010100BA
:1047300000410101000909414900090001415201FC
:104740000900004149000900004141000900004101
:104750004100090009414100090909000100090956
:1047600009090000090909000909090008000909E7
:1047700009090000090909080000090908080900D9
:1047800009090808080009090800080809090008BB
:1047900000080909000909090909000900080900B8
:1047A00000000009090800090909090900090909A7
:1047B0000908000909000900090809080909090888
:1047C000000909090909080900090101000909008E
:1047D0000100000909014100000900010000090968
:1047E0000001000909090001000909090001000987
:1047F0000909000809090900000000000100000083
:10480000000000000000000900000009000900008D
:104810000000010000000009000000000809000974
:104820000008090909090000000900000001000052
:104830000101000100000000000100000000000074
:104840000000000000000000000000000000010166
:104850000000000000000000000100010000000155
:104860000000000001000000000000000000000047
:104870000000000100000000010100000000010133
:1048800000000000000952010100000101000000C9
:104890000001010000000001010000010000010012
:1048A0000001010000010101090100000012525243
:1048B000090909525252520101010101010101018C
:1048C00001010101010101010101010101000001DA
:1048D0000101010000090949520100125252520916
:1048E00009495209520900010100000000010100BC
:1048F00000000001010000000001000000000001B4
:104900000900000000490900000000120800000032
:10491000000900000000000000000000000000008E
:104920000000000000000000000000000000000087
:104930000000000000000000000000000000000077
:10494000000000000000000000090000010000005D
:1049500000000900000000005200000000095200A1
:10496000000000095A000000000052000000000092
:104970005200000000001201014141414141090182
:104980004101415B520909090952525252520952DE
:104990005252525209525252521249525252525289
:1049A00012525252525252414141414141414141C0
:1049B00041414141414141414101014141414101A7
:1049C00001414141410901010909491212090952F4
:1049D0005252525252525241414141414141414150
:1049E0004141014141414141014141414141014177
:1049F000414141090009495252090052525252099B
:104A0000005252525209000101010009090101013D
:104A1000000909000101000909000101000909005C
:104A20004952010909000052000909000009000962
:104A30000900090000090908090908090908090904
:104A40000009090009090008000909000800000917
:104A500009090901000909090808000909000808ED
:104A600008090808000900090909080800090908D7
:104A700000090008090008090908090800090900D7
:104A800009000009090809000009090809000008CF
:104A900009090908090809090000090008090009AD
:104AA000090808090009090000090909000808099E
:104AB0000909080800090909080808090909080876
:104AC0000009090008080809080908000008090980
:104AD0000908000800080800000808080808090874
:104AE0000909080800010909090900090909090952
:104AF0000009090909090000000000000000000188
:104B0000000000000001000000090000000000009B
:104B1000000000000000000900000000000909007A
:104B20000000090909090000000000091200000046
:104B30000000000000000000010001000000000073
:104B40000000000000000900000100000900000052
:104B5000000000090000004909094909000000009F
:104B60000000000000010000010000000001000042
:104B70000000010009000000000909000000000910
:104B800000000000000909000909490900000000AF
:104B900009000000000000000009000009000009F1
:104BA00000000000090909000000090909090000C6
:104BB00000000909000000090000000000000000DA
:104BC00000000000000000000009000008000000D4
:104BD0000009090909000009090909000909090969
:104BE0000909090909090900000000000000000086
:104BF00000000000000000000800000000000009A4
:104C00000909090909090909090909090909090914
:104C1000090909090909090000000000090000004C
:104C20000000090000000000090000080008000959
:104C300009090909090909090909090909090909E4
:104C4000090909090909095252525252520909091E
:104C5000090909010100000100000001010100092A
:104C600009000000000909090001000909090900FB
:104C70000009090909000052525252525209090909
:104C80000909090100010001000100010001000003
:104C90000000000000000000010000000000000013
:104CA0000000000000000052525252000009091298
:104CB00009000001000000000000000000000000EA
:104CC00000000000090000000000090000000000D2
:104CD0000900000000000908080808080808000882
:104CE0000808080808080808080808080808080844
:104CF0000808080808080808080808080808080834
:104D0000080808080808080809080009090009082F
:104D10000808000809090808080009080808080820
:104D20000909080808080908080808000909080806
:104D300008080909080808090908080800090908F5
:104D400008080808000009080808080808080908F1
:104D500008080008090800000808080808090800F1
:104D600009080909080809090909090900090909BF
:104D700009090009090909090009090909090909B5
:104D8000090909080909090909010909090909099C
:104D900008090909090908090900090900090900A0
:104DA00000090009000000000009000000000009DF
:104DB00009000000090009000000000009000000CF
:104DC00008000000000000000000000000000000DB
:104DD00000000000000000000009000000000008C2
:104DE000090000000011110000000009110000007E
:104DF0000009110800080000000000090900000077
:104E0000000909000000000009000000000009007E
:104E10000000000009000000000909000000090965
:104E20000000000009090909090909090009090028
:104E30000000000909000000000909090900000933
:104E400009090909090909090909090909090909D2
:104E50000909090909090900000000000000000013
:104E60000000000000000000000000000000000939
:104E700009000000000909090909090909090909C6
:104E800009090909090909000000000909000000D1
:104E900000090900000000090900000000090900DC
:104EA000000000090909090909090909090909098D
:104EB000090909090909090808080808080808086B
:104EC0000808080808080808080808080808080862
:104ED0000808080808080808080808080808080852
:104EE0000808080808080800090808080808090947
:104EF0000808080808080808080808080808080832
:104F00000808080808080808080808080808080821
:104F10000808080808080808090808000908090915
:104F2000080809080908080809080800080009080D
:104F30000808080809080808000008080808080800
:104F400009080808080808090909090808090909D9
:104F500009010909090909080909090909090909CA
:104F600009090908080808090901090909090808BF
:104F700008090909090808080900090008080809BA
:104F80000009090808080809090908080911110891
:104F9000080808090908080808090908080808088D
:104FA000000808080808080911080000000911098C
:104FB0000809001109091111080909091111090944
:104FC000090911110911090909080809110900083D
:104FD0000809111108080000090009090900090958
:104FE0000909000800090909000800090909B608AB
:104FF00009090909B60809090909B60809090909C9
:10500000B60009090964B609090909090909090964
:10501000090909B60909090909B61111110009B6EA
:105020001112120909B61111120909B61112111142
:1050300009B6111112110909090909090909090912
:1050400009090909090909090909090909090909D0
:1050500009090909090909090909090900090909C9
:1050600009000908090909090909090909090909BA
:1050700009090909090909090909090909090909A0
:105080000909090909090909090909090909090990
:10509000090908080909000909090909090909098B
:1050A0000909090909090909090909090808090972
:1050B0000909090909090908111109090909111141
:1050C0001109080911111109090909090909090931
:1050D0000909090909090909090909090909090940
:1050E0000909090909090909090909090909090930
:1050F000000909090900000909090909090909093B
:10510000090909090909090909090909090909090F
:105110000909090909090909090909090A0A0A0005
:10512000090A0909090009090909090909090909F7
:1051300009090909090909090909090909090909DF
:1051400009090909090909090909090909090909CF
:1051500009090809090909080808080808080808C9
:1051600008080808080808080808080808080808BF
:1051700008080808090808080808080808080800B6
:1051800009080808000909080808080808080808A4
:1051900008080808080909090809090900121B0973
:1051A00008095B5B1B09095B521B1B0852525252D8
:1051B0001B095B52525252080808080808080808E0
:1051C00008080808080808080852080808080852CB
:1051D00012080808081B52080808081B23120008B8
:1051E000081B1B23121108080808080808080808EB
:1051F0000808080808080008080808000008080847
:10520000080808080808080800080808080808002E
:1052100008080808080808091212080908091212E3
:1052200008080911121208080809121208080809CA
:1052300012120808080912120908080912120908AE
:1052400008091112090808090900006D6D0800001D
:10525000006DB60908006D6DB60808646D6DB6087E
:10526000086DF6FF6D08A4F6FFFFB6A4F6FFFFFF7A
:10527000FFF6F6FFFFFFFFB66411121109B66D11BC
:105280001209096D6D641209096D6D6D640909F6E5
:10529000F66D6D0909FFFFFF6D5209FFFFFFF65222
:1052A00000FFFFFFF6A452090909090909090909C4
:1052B0000909090909090909000909090909090967
:1052C0000909090909090909090900000009090969
:1052D0000900000009090908120909090900120951
:1052E0000909090011110809091112111200091206
:1052F00012111208090911110909090811110909E6
:1053000009001111090909080911120908081111E8
:1053100012110909111111120909111211120909A9
:105320001112121209111251111109111111111139
:1053300009091111121209090909090909090909BB
:1053400009090909090909090909090909090909CD
:1053500009090909090909090909090909090909BD
:1053600009090909090900090909090909090909B6
:1053700009090909090909090909090900080009B0
:105380000909110911090809111111080909111157
:105390001109090912111109090911110909091144
:1053A000111109000911111111001112121111002E
:1053B00009111111110911121111111109091211FB
:1053C0001109090911110909090909090911000936
:1053D0000909091208090909081208090908091226
:1053E0000009090912090809090912090809090827
:1053F000090908080808090808090909091109091B
:1054000009090912120909090912120809090912E0
:105410001B12090909121B1B0909091212090808A4
:1054200008121208080908090909090909090909DE
:1054300009090909090909090909090909090009E5
:10544000090909090009090909000A000808000AF0
:105450001608080001161F090909090909090900A8
:1054600000000000000909090A090A0A0A0A1414BE
:10547000141414140A161416140B0A16140B14140C
:1054800014140B14161F1609090909000A00000953
:105490000909140A0100000B14140A090914140A5A
:1054A0000A090B14140009001414140A00000A1449
:1054B000140B0A09090B0B0B09000009001400006A
:1054C000090A00160A00090A0016140A0A0A00143A
:1054D00016140A0008140B0A0008080B0A09000039
:1054E000080A000900000008080008510908080817
:1054F0000951090808005109090808085109090853
:105500000008510911080808510911080809510932
:105510001108080951091212525252525252525253
:10552000525252525252525252525252525252525B
:10553000525252521252525252125252525212520B
:1055400052525212525B5B521B1B231B09521B1BF4
:105550001B1B1252521B1B1B125252521B1B12526C
:105560001252521B52525B5B5B1B235B5B5B5B5BB0
:105570001B5B5B5B5B5B23080808080808080808DE
:105580000808080808080808080808090809110890
:1055900008125212110908525B51081108525208A0
:1055A00008120809510808080808080008080951E5
:1055B0000808080912510808085B5B120808080966
:1055C000525B0908080808090808090808080808BB
:1055D0000808080808080809121209080809121220
:1055E0000908080911120908080809121108080019
:1055F0000909080808080808080808080808080928
:1056000009080809091112F6F6FFFFFFFFA4F6FFCB
:10561000FFFFFFA4F6F6FFF6A452A4F6FF5200081F
:10562000A4F6FFA4000809A4F6F6FF095252F6FFFB
:10563000FF1211A400A4F6FFFFFFFFA452FFFFFF1B
:1056400052A408FFFFA400005200FFF600F652A487
:10565000FFFFFFFFA4FFFF00F6F652F6F600FFA4DF
:1056600052A4FFFFFF0052080800000909080808BB
:1056700008080908080808080808080808080808A9
:105680000808080808080808080808090908090996
:105690000811111111090900111100090900111156
:1056A0000009090811110900090809110909080868
:1056B0000909080808080909090808090808080864
:1056C0000809090909080809090909090909000956
:1056D000000909090900000909080800090008086B
:1056E0000808080808080808080808080809090937
:1056F00009090908090808091112111209111111E3
:1057000011120909111111120909111111110909B7
:105710001111111109091111111109091211111198
:105720000909090909090809090900080908000007
:10573000080911090808081151090908090911097E
:1057400008090809090808080808080908080808D5
:105750000808080808080851091111090951090920
:105760000909091111090909091111090909111179
:105770001211090911111109091111090909111150
:105780001108081112121209090909090909090960
:10579000090911090911090911121211110909093F
:1057A000090911110812121109110911121212110D
:1057B0000912121209090809090908080911120930
:1057C000080809111209080808090909080809093F
:1057D0000909080808090808080809090808080844
:1057E00009080808080808120908090808121B080F
:1057F000080808121B0808080812120808080812EE
:1058000012080808081209080808081109080808F9
:10581000080908080808080808000B1F16080800EF
:10582000161F140808091F161608080B1F161F0854
:10583000080B1F1F16080814161F27080814162720
:105840003708081427376F0A141F1F1F1414161F58
:105850001F160B1F271616141F27271F141627168F
:105860001F1F16161F2716161F1F1F371F16272745
:10587000276F6F161F27270A140A00090A14140A33
:105880000000001F160A0A0A0027160B1616142716
:1058900016141616161F14141F1F1F1616161F1681
:1058A000161F161416161409000009090000090035
:1058B0000A0B0A090A0A0914140A0A140A0A141417
:1058C0000B16140A1414141616140B1414161614AA
:1058D0000B1414141F1F0B080808080808000808F8
:1058E0000808080900080808080B00080808081438
:1058F00001080808081409080808080B0A0808081D
:10590000080B0B080808080808495109120808493B
:105910005109120809095109120808095109120808
:105920000909510911080009510912080009510912
:10593000520809095151525252525B5B5B52525B01
:105940005B5B5B52525B5B5B5B525B5B5B5B5B5BC2
:105950005B5B5B5B5B5B5B5B5B5B5B5B5B5B5B5B97
:105960005B5B5B5B5B5B5B5B5B5B5B1B235B5B5BFF
:105970005B5A235B5B5B5B5B235B5B5B5B5B235B20
:105980005B5B5B5B5B5B5B5B52521B5B5B525B5BC2
:105990001B525A5B52525B5208080808081208084A
:1059A0000808081208080808081208080808081B50
:1059B00009080808082311080808082351080808DE
:1059C000082312080808080809111212080809110A
:1059D00012120808091111121208090912121208EC
:1059E0000911111112080951111111080849091161
:1059F00011080809111212080800FF000008080821
:105A0000F6A4FF08080808F6F61212080808521152
:105A100011111108081112121111110909090909AE
:105A200009121112121212A4FFA400A452000000C5
:105A3000A4FF52A4FFA4FFA412F6FFF6A45212087A
:105A4000080811111111111211121209090909097D
:105A5000091212121212121212121212121212122F
:105A60001212121212121212121212121212121117
:105A70001111111111121212121212090909090938
:105A80000911111109090912121111090912121231
:105A900012120912121212121112121212121211F1
:105AA000111112111112111211110909090909110B
:105AB0005109090952511209080800080809090981
:105AC00009090909111211121212121212121211DD
:105AD00012121212120909090911111109090909F1
:105AE000095B5B5A5B5209000809090909090909A0
:105AF00011090912110909080812110908080812E8
:105B000011110808081111120908081109090908DA
:105B10000809090909080808080808080808080801
:105B200008080808080808080808080808080808F5
:105B300008080808080808080809090808080808E3
:105B400008080808080808090911121212080912A1
:105B50001212120911111212120911111212120944
:105B60001111121212090912121111090909090958
:105B70000808080808080812121208080812121269
:105B800008080812121208080812121B0808085107
:105B90001B1B090808110909080808080808080853
:105BA000080808080909090808080808080911125E
:105BB000080808091B1B120808511B1B1B080811A9
:105BC0001B1B1B0808111B1B1B0808091B1B1B08A0
:105BD00008121B1B1B1B090808162737BF080814CF
:105BE0001FBFFF08081416BFFF0808141677FF0828
:105BF00008141637770808141637370808141627BC
:105C00002708081416271FFFB71627271FFFF61FA0
:105C1000271F27FFB716271F37FF6F1F271F37774D
:105C2000271F272737371F2727276F271F272727B4
:105C3000372737272727371F1614162727373727E1
:105C4000161F2727273716162737B7BF6F1427BF0A
:105C5000FFFF6F1427FFFFFF6F1627FFFFFF6F1671
:105C60002777FF771F1F271F14161F1F14271616CD
:105C70001F1F141F161F1F1F1627161F1F1F162753
:105C800016271F1F16271F1F1F1F1F271627271F17
:105C90001F271627271F1F0B0A080808080B0A08CA
:105CA0000808080A0A080808080A0A080808080B69
:105CB0000A080808080B0A08080808140A0808084F
:105CC000080B0A08080808080009515112080009C1
:105CD000515112080809515251080809515A110826
:105CE0000808525A11080808525951000800095270
:105CF000520808080809095B5B5B5B5B525B5B5BF6
:105D0000525B525B5252525B525B5B5B525B5B522B
:105D10005B5B525252525B5B525B5B125B5B5B5B49
:105D20005B125B5B5B5B5B5B5B5B5B52525B525B27
:105D300052525B5B5B525B5B5B52525B5B5B5B5BE0
:105D40005B5B5B5B5B5A5B5B5B5B5B5B5B5B5B5BA4
:105D50005B5B5B5B5B525B235208080808235209BC
:105D60000808085B1B090808085B1B110808081BCA
:105D700023510808085B23510808085B2312080810
:105D8000085B231208080808080912525208000983
:105D9000091212080851125252000808091252083A
:105DA00008080912520008000912520808080912CE
:105DB0005208000809125212521212121212121133
:105DC00011110952525252525252525252525212BE
:105DD00052525252525252525252525212525252E3
:105DE0005252525252525212121212525209110966
:105DF0000911095252525212125252525252121256
:105E000052521212125252521212125212121252B2
:105E1000121212525252125252525252520909093D
:105E200009111112121212121152525252521152DF
:105E3000525252521152521252520952525252520C
:105E4000115252525212125212515A115B09515AA6
:105E500052125B095A5A515B5B5251115B5B5B5AA0
:105E600051125B5B5B5151525B5B5B515152525B18
:105E70005B51515252525B5B5B5B5B52125B5B5BF3
:105E80005B5B095B5B5B5B5B1B5B5B5B5B5B235B2C
:105E90005B5B5B5B235B5B5B5B5B235B5B5B5B5BC2
:105EA000235B5B5B5B1B23525252110808111112DA
:105EB0000908080912120908081B125209080823C8
:105EC000125209080823115209080823115209081F
:105ED000082312520908080808080952520808083D
:105EE0000952520808080912520808080909090845
:105EF0000808080808080808080808080808080822
:105F000008000808080808121B1B23231212121B82
:105F100023231B121B23232323121B1B23090912D8
:105F20001B23230808121B1B230808121B2323080A
:105F300008121B1B23080808080808080808080896
:105F400008080808080808080808080808080808D1
:105F500008080808000808080808080808080008D1
:105F60000008080808000808080B27371608081456
:105F700016373708081416777700080A16BF77080F
:105F800008012737270008011627160800001416F5
:105F9000160008000B16166FBF271FB777BFBF1F6D
:105FA00027BFBFFFF61F6FFFFFFFB727FFFFFFBF32
:105FB000BFBFFFFFFF6FFFFFFF77BF1FFFFF772709
:105FC0006F16FF6F1F161F3737371F272727271F0B
:105FD000272727271F1F1F2727771F6F272727FF01
:105FE0006FB7772727FFBFBF6F2727FFFF771F27D1
:105FF0002777FF6F272727271F271F1F1F271627F2
:106000001F1F1F27161F1F1F16271F1F1F1F161FAB
:1060100016161F1F142716161616161F14141616FA
:10602000141F16141414140B0A080808080B0A0885
:10603000080808140A080808080B0A080808080BCA
:106040000A080808080A09080808080B09080808C7
:10605000080B000808080808000808510908080883
:1060600008115100000808515A080808095A590037
:106070000008515A520800080952590008080952EC
:1060800052000000000000115B5B5B5B5B09525B30
:106090005B5B5B5152525B5B5B515B5B5B5B5B5180
:1060A0005B5B525B5251525B52525B51125B5252DC
:1060B0005B0000000000005B5B5B5B5B5B5B5B5B52
:1060C0005B5B5B5B5B5B5B5B5B5B5B5B5B5B5B5B20
:1060D000525B5B5B5B5B5B5B5B5B5B5B5B5B5B5B19
:1060E0005B0000000000005B23120808085B23121D
:1060F0000808085B23520808085B23520908081B9C
:106100001B1B0808085B231B0908081B5B520908B6
:10611000080000000000000808080808080808082F
:1061200008080808080908080808080808080808EE
:1061300008080808080808080808080808080808DF
:1061400008000000000000080808001252080808B3
:106150000809520800080809120808080809120866
:1061600008080808090808080808080808080808AE
:1061700008000000000000125212525252525252B5
:10618000525252125212525212525252521212126F
:10619000121212090909090909080808080808085B
:1061A00008000000000000521252521252521252C5
:1061B000121252125212120911125212090809092E
:1061C000090908080808080808080808080808084D
:1061D00008000000000000525212521212125252D5
:1061E00052121252525252521212121252121209D8
:1061F000080909090908080808080808080808081B
:10620000000000000000005251525B525B525112DC
:10621000525B52515152525B5B5152525B5B5B522B
:1062200051525B5B5B5251525B5B5B5151525B5B0A
:106230005B0000000000005B5B5B5B1B235B5B5B48
:106240005B5B235B5B5B5B1B235B5B5B5B5B235B86
:106250005B5B5B5B235B5B5B5B5B235B525B5B5B07
:1062600023000000000000231252090808231252E4
:10627000090808231112090808231109080808232E
:10628000110808080823120908080823120808083A
:1062900008000000000000080808080808080808AE
:1062A0000808080808080808080808080811080865
:1062B000080808521108080808525B0808084952E3
:1062C0005100000000000008080808080808080835
:1062D000080808080808080808080808080808093D
:1062E00009090912095252525212111111111212B6
:1062F0005200000000000008080808080800000814
:1063000008080808080800080808080008080851D4
:1063100008080808085208080808081208080808A9
:1063200008000000000000111B1B230808111B1BA4
:10633000230808111B1B230808091B1B230808112D
:10634000521B23080812521B230808111B1B230889
:1063500008000000000000080808000800080808FD
:1063600008080008080800080808080808080008C5
:10637000080808080808080808080808080808089D
:1063800008000000000000080000011416080008C2
:10639000000A1600080000000A08080008080008A3
:1063A000000800000808080808080008080808088D
:1063B00008000000000000165C1F1F1616141416BB
:1063C0001F1F160B0B16161616090A1416161600A2
:1063D00000090B1414080800080008080808080839
:1063E0000800000000000027776F1F1F1F161F1FE7
:1063F0001F1F1F1414161F1F1F0B14161616160B23
:106400000A141614140800080008080008080808F0
:10641000000000000000001F1414141414161414BB
:1064200014140A160B14140B00140A140B09000B95
:106430000A0A0100080808080808080800080808EF
:10644000080000000000000A00080808080008080A
:1064500008080800080808080808080808080808C4
:1064600008080808080808080808080808080808AC
:1064700008000000000000070707070707070707D5
:10648000070707383838383838383838383838C88F
:10649000C8C8C8C8C8C8C8C8C8C8C8FFFFFFFFFF69
:1064A000FFFFFFFFFFFFFF160F01020301010101C4
:1064B0000101010101040506070101010108090AA2
:1064C0000B0C010D0E0F10111213141516171801D5
:1064D0000101191A1B1C1D1E1F2021222324252601
:1064E0002728292A2B2C2D2E2F30313233343536C4
:1064F0003738393A3B3C3D3E3F40414243444545B5
:1065000045464748494A4B4C4D4E4F5051393952F8
:1065100053545545454545565758595A5B5C5D5E41
:106520005F60393939616245454545454563646574
:10653000666768696A6B6C6D6E6F7071454545453D
:1065400045454572737475767778797A7B7C7D7E64
:106550007F454545454545454580818283848586FF
:106560004545454587888945454545454545458ACD
:106570008B8C8D8E8F9091459245934545944545E2
:10658000454595969798999A8A9B9C9D9E9FA04574
:10659000A1A2A3A4A5A6A7A8A9AA8AABACADAEAF99
:1065A000B0B1B2B3B4B5B6B7B8B9BABBBCBDBEBF73
:1065B000C0C1C2C3C48AC5C6C7C8C9CACBCCCDCEA8
:1065C000CF8AD0D1D2D3D4D5D6D7D88AD9DADBDC0A
:1065D000DDDEDF8A8AE0E1E2E3E4E5E6E7E8E9EA36
:1065E000EBECEDEEEFF0F1F2F3F4F5F6F7F8F9FA83
:1065F000FB000000000000000000000000000000A0
:10660000000000000000000000000000000000008A
:10661000000000000000000000000000000000007A
:10662000000000FF00000000FFFFFF000000FFFF70
:10663000FF00000000FF0000000000FF000000005D
:1066400000000000000000FF00000000000000004B
:1066500000FFFF00FFFF00FFFF00FFFF00FF000043
:10666000FF0000000000000000000000000000002B
:10667000000000000000000000000000000000001A
:106680000000000000000000FF00FF0000FFFFFF0F
:10669000FFFF0000FF00FF000000FF00FF0000FF01
:1066A000FFFFFFFF0000FF00FF00000000000000F0
:1066B0000000FF0000000000FFFFFF0000FF0000DF
:1066C00000000000FFFF000000000000FF0000FFCE
:1066D000FFFF0000000000FF0000000000000000BD
:1066E00000FFFF0000FF00FFFF0000FF00000000B0
:1066F000FF00000000FF00000000FF00000000FF9E
:106700000000FFFF00FF0000FFFF0000000000008E
:106710000000FF00000000FF00FF000000FF00FF7E
:1067200000000000FF00000000FF00FF00FF00FF6E
:106730000000FF000000FFFF00FF0000000000005D
:106740000000FFFF00000000FFFF00000000FF004E
:106750000000000000000000000000000000000039
:106760000000000000000000000000000000000029
:10677000000000FF00000000FF0000000000FF001C
:1067800000000000FF0000000000FF00000000000B
:10679000FF000000000000FF0000000000000000FB
:1067A0000000FF000000000000FF0000000000FFEC
:1067B0000000000000FF0000000000FF00000000DB
:1067C00000FF00000000FF000000000000000000CB
:1067D0000000000000000000FF00FF000000FFFFBD
:1067E000FF0000FFFFFFFFFF0000FFFFFF000000B2
:1067F000FF00FF000000000000000000000000009B
:10680000000000000000000000FF0000000000FF8A
:10681000000000FFFFFFFFFF000000FF000000007E
:1068200000FF000000000000000000000000000069
:106830000000000000000000000000000000000058
:106840000000000000000000000000000000000048
:10685000FFFF00000000FFFF00000000FF0000003D
:106860000000000000000000000000000000000028
:10687000000000FFFFFFFFFF00000000000000001D
:106880000000000000000000000000000000000008
:1068900000000000000000000000000000000000F8
:1068A00000000000000000000000000000000000E8
:1068B000FFFF00000000FFFF0000000000000000DC
:1068C0000000000000000000000000FF00000000C9
:1068D000FF00000000FF00000000FF00000000FFBC
:1068E00000000000000000000000000000000000A8
:1068F00000002F2F2F00002F0000002F002F00007E
:106900002F2F002F002F002F002F2F00002F002FE0
:106910000000002F00002F2F2F00000000000000BB
:106920000000002F000000002F2F00000000002FAB
:1069300000000000002F00000000002F00000000F9
:10694000002F000000002F2F2F000000000000008B
:1069500000002F2F2F00002F0000002F000000004C
:10696000002F0000002F2F0000002F000000002F3C
:1069700000000000002F2F2F2F2F0000000000002C
:1069800000002F2F2F00002F0000002F000000001C
:10699000002F00002F2F2F0000000000002F002FDD
:1069A0000000002F00002F2F2F000000000000002B
:1069B000000000002F000000002F2F0000002F001B
:1069C0002F00002F00002F00002F2F2F2F2F00004F
:1069D00000002F00000000002F0000000000000059
:1069E000002F2F2F2F2F002F00000000002F00005E
:1069F0000000002F2F2F2F0000000000002F002F7D
:106A00000000002F00002F2F2F00000000000000CA
:106A10000000002F2F0000002F000000002F0000BA
:106A20000000002F2F2F2F00002F0000002F002F1D
:106A30000000002F00002F2F2F000000000000009A
:106A4000002F2F2F2F2F00000000002F000000002C
:106A50002F000000002F000000002F0000000000A9
:106A60002F00000000002F000000000000000000C8
:106A700000002F2F2F00002F0000002F002F0000FC
:106A8000002F00002F2F2F00002F0000002F002FBD
:106A90000000002F00002F2F2F000000000000003A
:106AA00000002F2F2F00002F0000002F002F0000CC
:106AB000002F00002F2F2F2F00000000002F0000BC
:106AC00000002F0000002F2F000000000000000039
:106AD0000000000000000000000000000000FFFFB8
:106AE00000000000FFFF00000000000000000000A8
:106AF000FFFF00000000FFFF00000000000000009A
:106B00000000000000000000000000000000FFFF87
:106B100000000000FFFF0000000000000000000077
:106B2000FFFF00000000FFFF00000000FF0000006A
:106B30000000000000FF00000000FF00000000FF58
:106B400000000000FF000000000000FF0000000047
:106B50000000FF000000000000FF00000000000037
:106B600000000000000000000000000000FFFFFF28
:106B7000FFFF00000000000000000000000000FF18
:106B8000FFFFFFFF00000000000000000000000009
:106B90000000FF000000000000FF000000000000F7
:106BA000FF000000000000FF00000000FF000000E8
:106BB00000FF00000000FF000000000000000000D7
:106BC0000000FFFFFF0000FF000000FF00000000CA
:106BD00000FF000000FFFF00000000FF00000000B9
:106BE00000000000000000FF0000000000000000A6
:106BF0000000FFFFFF0000FF000000FF00FF00FF9C
:106C0000FFFF00FF00FF00FF00FF00FFFFFF00FF8E
:106C1000000000000000FFFFFF0000000000000077
:106C20000000FFFFFF0000FF000000FF00FF00006A
:106C300000FF00FF000000FF00FFFFFFFFFF00FF5D
:106C4000000000FF00FF000000FF00000000000047
:106C500000FFFFFFFF0000FF000000FF00FF00003B
:106C600000FF00FFFFFFFF0000FF000000FF00FF2C
:106C7000000000FF00FFFFFFFF0000000000000019
:106C80000000FFFFFF0000FF000000FF00FF00000A
:106C9000000000FF0000000000FF0000000000FFF7
:106CA000000000FF0000FFFFFF00000000000000E8
:106CB00000FFFFFFFF0000FF000000FF00FF0000DB
:106CC00000FF00FF000000FF00FF000000FF00FFCA
:106CD000000000FF00FFFFFFFF00000000000000B9
:106CE00000FFFFFFFFFF00FF0000000000FF0000AB
:106CF000000000FFFFFFFF0000FF0000000000FF9A
:106D00000000000000FFFFFFFFFF00000000000088
:106D100000FFFFFFFFFF00FF0000000000FF00007A
:106D2000000000FFFFFFFF0000FF0000000000FF69
:106D30000000000000FF0000000000000000000054
:106D40000000FFFFFF0000FF000000FF00FF000049
:106D5000000000FF00FFFFFF00FF000000FF00FF3A
:106D6000000000FF0000FFFFFFFF00000000000028
:106D700000FF000000FF00FF000000FF00FF000018
:106D800000FF00FFFFFFFFFF00FF000000FF00FF0C
:106D9000000000FF00FF000000FF000000000000F6
:106DA0000000FFFFFF00000000FF0000000000FFE8
:106DB0000000000000FF0000000000FF00000000D5
:106DC00000FF00000000FFFFFF00000000000000C7
:106DD0000000000000FF0000000000FF00000000B5
:106DE00000FF0000000000FF00FF000000FF00FFA8
:106DF000000000FF0000FFFFFF0000000000000097
:106E000000FF000000FF00FF0000FF0000FF00FF88
:106E1000000000FFFF00000000FF00FF000000FF77
:106E20000000FF0000FF000000FF00000000000065
:106E300000FF0000000000FF0000000000FF000055
:106E4000000000FF0000000000FF0000000000FF45
:106E50000000000000FFFFFFFFFF00000000000037
:106E600000FF000000FF00FFFF00FFFF00FF00FF2A
:106E700000FF00FF000000FF00FF000000FF00FF18
:106E8000000000FF00FF000000FF00000000000005
:106E900000FF000000FF00FFFF0000FF00FF00FFF9
:106EA00000FF00FF0000FFFF00FF000000FF00FFE9
:106EB000000000FF00FF000000FF000000000000D5
:106EC0000000FFFFFF0000FF000000FF00FF0000C8
:106ED00000FF00FF000000FF00FF000000FF00FFB8
:106EE000000000FF0000FFFFFF00000000000000A6
:106EF00000FFFFFFFF0000FF000000FF00FF000099
:106F000000FF00FFFFFFFF0000FF0000000000FF88
:106F10000000000000FF0000000000000000000072
:106F20000000FFFFFF0000FF000000FF00FF000067
:106F300000FF00FF000000FF00FF00FF00FF00FF58
:106F40000000FF000000FFFF00FF00000000000045
:106F500000FFFFFFFF0000FF000000FF00FF000038
:106F600000FF00FFFFFFFF0000FF0000FF0000FF29
:106F7000000000FF00FF000000FF00000000000014
:106F80000000FFFFFF0000FF000000FF00FF000007
:106F900000000000FFFFFF000000000000FF00FFF6
:106FA000000000FF0000FFFFFF00000000000000E5
:106FB00000FFFFFFFFFF000000FF0000000000FFD8
:106FC0000000000000FF0000000000FF00000000C3
:106FD00000FF0000000000FF0000000000000000B3
:106FE00000FF000000FF00FF000000FF00FF0000A6
:106FF00000FF00FF000000FF00FF000000FF00FF97
:10700000000000FF0000FFFFFF0000000000000084
:1070100000FF000000FF00FF000000FF00FF000075
:1070200000FF00FF000000FF00FF000000FF000065
:10703000FF00FF00000000FF000000000000000053
:1070400000FF000000FF00FF000000FF00FF00FF46
:1070500000FF00FF00FF00FF00FF00FF00FF00FF38
:1070600000FF00FF0000FF00FF0000000000000024
:1070700000FF000000FF00FF000000FF0000FF0015
:10708000FF00000000FF00000000FF00FF0000FF05
:10709000000000FF00FF000000FF000000000000F3
:1070A00000FF000000FF00FF000000FF00FF0000E5
:1070B00000FF0000FF00FF00000000FF00000000D4
:1070C00000FF0000000000FF0000000000000000C2
:1070D00000FFFFFFFF0000000000FF00000000FFB6
:1070E00000000000FF00000000FF0000000000FFA3
:1070F0000000000000FFFFFFFF0000000000000094
:10710000000000FFFF000000FF0000000000FF0083
:10711000000000FFFF0000000000FF000000000072
:10712000FF000000000000FFFF0000000000000062
:10713000000000FFFF000000FF0000FF00FF00FF55
:10714000FF00FFFF00FF0000FFFF00FFFF00FF0048
:10715000FF0000FF000000FFFF0000000000000033
:107160000000FFFF000000000000FF000000000022
:10717000FF0000000000FFFF00000000FF00000013
:107180000000FF000000FFFF000000000000000002
:1071900000FEFEFEFEFEFEFEFEFEFEFEFEFEFEFE0D
:1071A000FEFEFEFEFEFEFEFEFEFEFEFEFEFEFEFEFF
:1071B000FEFEFEFEFEFEFEFEFEFEFEFEFEFEFEFEEF
:1071C000FE5EAFAFAFAFB7A61516161616A615160C
:1071D000161616A61516161616A61516161616A6A1
:1071E0001516161616A61516161616A61516161622
:1071F000165C0CAFAFAF560B651E1615090B651E5E
:107200001615090B651E1615090B5C0A1615090BD8
:107210000B010001550BA5B7AFAE490B651E161546
:1072200009A61516161616A61516161616000B160E
:1072300016160CB7530016160CA666AE000049A62B
:107240001516AFAF52A6151616154A140000000009
:107250005E0B651E1615090B651E161509535F1585
:10726000161509535F1516150967151616150966C3
:1072700015161615096715161609085C0000000199
:1072800055AFAFAFAFAFAF15161616150A151616D8
:1072900016150A00000000000015160A151616152E
:1072A000160A15161615160A151616000000000007
:1072B00000AFAFAFAFAFAE161616161509161616FD
:1072C00016150900000000000816150A16165516B6
:1072D000150A16165516150A161655000000000058
:1072E0000815161616150A15161616150A15161669
:1072F00016150A00000000000015160A15161615CE
:10730000160A15161615160A1516160000000000A6
:10731000001616161615091616161615091616163F
:1073200016150900000000000816150A1616551655
:10733000150A16165516150A1616550000000000F7
:1073400008FEFE0000FEFEFE005F0400FE005FFF80
:1073500007040000070707040000060706040000F2
:107360000406060400FE00040400FEFEFE0000FE0B
:10737000FEFEFE0000FEFEFE00EA9900FE00EAFFAF
:10738000E2490000E2E2E249000099E29949000086
:107390004999994900FE00494900FEFEFE0000FEA1
:1073A000FEFEFE0000FEFEFE007D2100FE007DFFD1
:1073B000311900003131311900002131211900004B
:1073C0001921211900FE00191900FEFEFE0000FE21
:1073D000FEFEFE0000FEFEFE00F78600FE00F7FF48
:1073E000C74C0000C7C7C74C000086C7864C0000CA
:1073F0004C86864C00FE004C4C00FEFEFE0000FE5B
:10740000FEE3E3E3E3E3E3E3E3E3E3E3E3E3E3E331
:10741000E3E3E3E3E3E3E3E3E3E3E3E3E3E3E3E33C
:10742000E3E3E3E3E3E3E3E3E3E3E3E3E3E3E3E32C
:10743000E30804111213141516171518191A1B1C3A
:107440001D1E1F15151515201515231515151524A9
:1074500015FEFEFEFEFEFEFEFEFEFEFEFEFEFEFE35
:10746000FEFEFEFEFEFEFEFEFEFEFEFEFEFEFEFE3C
:10747000FEFEFEFEFEFEFEFEFEFEFEFEFEFEFEFE2C
:10748000FE3810FEFE38103810FEFE38103810FEA0
:10749000FE38103838383838103810FEFE381038BA
:1074A00010FEFE38103810FEFE3810FEFEFEFEFE06
:1074B000FEFEFE3810FEFEFE38103810FE3810FEBC
:1074C000FE38103838383838103810FEFE3810388A
:1074D00010FEFE38103810FEFE3810FEFEFEFEFED6
:1074E000FE3838383810FE3810FEFE38103810FEDE
:1074F000FE38103838383810FE3810FEFEFEFE38E0
:1075000010FEFEFEFE3810FEFEFEFEFEFEFEFEFE3D
:10751000FE3810FEFE38103810FEFE38103810FE0F
:10752000FE3810FE38103810FEFEFE3810FEFEFE4B
:10753000FE3810FEFEFEFE3810FEFEFEFEFEFEFED3
:10754000FE3810FEFEFEFE3810FEFEFEFE3810FE77
:10755000FEFEFE3810FEFEFEFE3810FEFEFEFE3879
:1075600010FEFEFEFE383838383810FEFEFEFEFEF5
:10757000FEFE38383810FE3810FEFE38103810FE87
:10758000FE38103810FEFE38103810FEFE38103865
:1075900010FEFE3810FE38383810FEFEFEFEFEFEED
:1075A000FE3810FEFE38103810FEFE38103810FE7F
:1075B000FE38103810FEFE381038103810381038E9
:1075C00038103838103810FEFE3810FEFEFEFEFE71
:1075D000FE3838383838103810FEFEFEFE3810FEFF
:1075E000FEFEFE38383810FEFE3810FEFEFEFE3875
:1075F00010FEFEFEFE383838383810FEFEFEFEFE65
:10760000FE3810FEFE3810383810FE3810381038AA
:107610001038103810FE3838103810FEFE38103888
:1076200010FEFE38103810FEFE3810FEFEFEFEFE84
:10763000FEFFFFFFFF02FEFEFEFEFEBF02FEFEFE9D
:10764000FE3F02FE27272702FE1702FEFEFEFE1661
:1076500002FEFEFEFE060606060602FEFEFEFEFE1A
:10766000FEFEFFFFFF02FEBF02FEFEBF023F02FE64
:107670003F3F02270227022702171702FE170216B2
:1076800002FEFE1602FE06060602FEFEFEFEFEFEDE
:10769000FEFEFFFFFF02FEBF02FEFEBF023F02FE34
:1076A000FE3F02FE27272702FE1702FEFE170216E4
:1076B00002FEFE1602FE06060602FEFEFEFEFEFEAE
:1076C000FEFEADFFADFEFEADFEFFFEADFEFF07FF11
:1076D00007FFFEADFFFFFFADFEFEFFFEFFFEFEFE5D
:1076E000FEFEFEFEFEFEADFFADFEFEFEFEFEFEFE5B
:1076F000FEFEFEFEFEFEFEFEFEFEFEFEFEFEFEFEAA
:1077000016FEFEFEFE1627FEFEFE161F2716FEFEC6
:10771000161F2716FEFE161F1FFEFEFEFE1616FE85
:10772000FEFEFEFEFEFEFEFEFEFEFEFEFEFEFE1661
:10773000FEFEFEFEFE1616FEFEFEFE271FFEFEFEEF
:1077400016772716FEFE16271F16FEFEFE1616FEDD
:10775000FEFEFEFEFEFEFEFEFEFEFEFEFEFEFEFE49
:1077600016FEFEFEFE1627FEFEFE1F277716FEFE05
:1077700016772716FEFEFE27160EFEFEFEFE16FEEE
:10778000FEFEFE00FEFEFEFEFE00FEFEFEFEFE0013
:1077900000FEFEFEFE000000FEFE0000000000FEF7
:1077A0000000000000FE00000000000000000000DB
:1077B00000FEFEFEFEFEFEFEFEFEFEFEFEFEFEFEE7
:1077C000FE00FEFEFEFEFE00FEFEFEFEFE000000CF
:1077D00000FEFE00000000000000000000000007A6
:1077E00000FEFEFEFEFEFEFEFEFEFEFEFEFE00FEB5
:1077F000FEFEFEFE00FEFEFEFE0000FEFEFEFE00A1
:1078000000FEFE0000000000000000070000000075
:1078100000FEFEFE00FEFEFEFEFE00FEFEFEFE0080
:1078200000FEFEFE000000FEFE0000000000FE0064
:1078300000000000FE0000000000FE00000000004C
:1078400000FEFEFEFEFEFEFEFEFEFEFEFEFEFEFE56
:10785000FEFEFEFEFEFEFEFEFEFEFEFEFEFEFEFE48
:10786000FEFEFEFEFEFEFEFEFEFEFEFEFEFEFEFE38
:10787000FEFEFEFEFEFEFEFEFEFEFEFEFEFEFEFE28
:10788000FE00FEFEFEFEFE00FEFEFEFEFE0000FE10
:10789000FEFEFE0000FEFE00000000FE00000007ED
:1078A00000FEFEFEFEFEFEFEFEFEFEFEFEFE00FEF4
:1078B000FEFEFEFE00FEFEFEFE0000FEFEFEFE00E0
:1078C00000FEFEFEFE00000000FEFE0700000000BD
:1078D000FE000000000000000000000000000000AA
:1078E00000FEFE00000000FEFE0000FE00FEFE00A6
:1078F000FEFEFEFEFE00FEFEFEFEFE00FEFEFEFEA4
:10790000FE00FEFE00000000FEFEFE000000FEFE87
:10791000FE0000FEFEFEFE0000FEFEFEFEFE00FE7D
:10792000FEFEFEFEFEFEFEFEFEFEFEFEFEFEFEFE77
:10793000FE000000FEFE000000FEFEFE000000FE55
:10794000FEFE000000FEFEFEFE00FEFEFEFEFEFE4F
:10795000FEFEFEFEFEFEFEFEFEFEFEFEFEFEFEFE47
:10796000FE000000000000000000000000FEFE001D
:10797000000000FEFE00000000FEFE00FE0000FE13
:10798000FEFEFEFE00FEFEFEFEFE00FEFEFEFEFE13
:1079900000FEFEFEFEFEFEFEFEFEFEFE00FEFEFE03
:1079A000FEFE00FEFEFEFE0000FEFEFE000000FEEB
:1079B000FEFE000000FEFE00000000FEFE000000D3
:1079C00000000000000000000000FE00000000FEBB
:1079D000FE000000FEFEFE000000FEFEFEFE0000B7
:1079E000FEFEFEFEFE00FEFEFEFEFE00FEFEFEFEB3
:1079F000FE0000000000000000FE0000000000FE8D
:107A0000FE00000000FEFEFE0000FEFEFEFE00FE88
:107A1000FEFEFEFE00FEFEFEFEFE00FEFEFEFEFE82
:107A200000FEFEFEFEFEFE00FEFEFEFEFE00FEFE70
:107A3000FEFEFE0000FEFEFEFE000000FEFEFE005A
:107A40000000FEFEFE00000000FEFE00000000FE42
:107A5000FEFE0000000000FE0000000000FE00002E
:107A60000000FE00000000FEFE00000000FEFE0020
:107A7000000000FEFE00000000FEFE00000000FE10
:107A8000FE00FEFEFEFEFE00FEFEFEFEFE00FEFE10
:107A9000FEFEFEFEFEFEFEFEFEFEFEFEFEFEFEFE06
:107AA000FEFEFEFEFEFEFEFEFEFEFEFEFEFEFEFEF6
:107AB000FEFEFEFEFEFE00FEFEFEFEFE00FEFEFEE2
:107AC000FEFE00FEFEFEFEFEFEFEFEFEFEFEFEFED4
:107AD000FEFEFEFEFEFEFEFEFEFEFEFEFEFEFEFEC6
:107AE000FE0000000000FE0000000000FEFE00009E
:107AF0000000FEFEFE00000000FEFE00000000FE92
:107B0000FE00000000FEFE00000000FEFE0000007F
:107B1000000000FE00FEFE0000FEFEFEFE00FEFE77
:107B2000FEFEFEFEFEFEFEFEFEFEFEFEFEFEFEFE75
:107B3000FEFEFEFEFEFEFEFEFEFEFEFEFEFEFEFE65
:107B4000FEFEFE00FE0000FEFEFEFE0000FEFEFE4B
:107B5000FEFE00FEFEFEFEFEFEFEFEFEFEFEFEFE43
:107B6000FEFEFEFEFEFEFEFEFEFEFEFEFEFEFEFE35
:107B7000FEFEFEFEFEFEFEFEFEFEFEFEFEFEFEFE25
:107B8000FEFEFEFEFEFEFEFEFEFEFEFEFEFEFEFE15
:107B9000FEFEFEFEFEFEFEFEFEFEFEFEFEFEFEFE05
:107BA000FEFEADFFADFEFEADFEFFFEADFEFF07FF2C
:107BB00007FFFEADFFFFFFADFEFEFFFEFFFEFEFE78
:107BC000FEFEFEFEFEFEADFFADFEFEFEFEFEFEFE76
:107BD000FEFEADFFADFEFEADFEFFFEADFEFF05FFFE
:107BE00005FFFEADFFFFFFADFEFEFFFEFFFEFEFE4A
:107BF000FEFEFEFEFEFEFEFEFEFEFEFEADFFADFE46
:107C0000FEFEADFFADFEFEADFEFFFEADFEFF03FFCF
:107C100003FFFEADFFFFFFADFEFEFFFEFFFEFEFE1B
:107C2000FEFEFEFEFEFEADFFADFEFEFEFEFEFEFE15
:107C3000FEFEADFFADFEFEADFEFFFEADFEFF05FF9D
:107C400005FFFEADFFFFFFADFEFEFFFEFFFEFEFEE9
:107C5000FEFEFEFEFEFEFEFEFEFEFEFEADFFADFEE5
:107C6000FE0000005252520000520000000000527C
:107C70000700070000520000000000520000000052
:107C80000000520000FFA4A4A4A4A4FFFFA40000CD
:107C9000A40000000000005200000000005200009C
:107CA000000000A40000000000A40000000000A4E8
:107CB0005200000000FFA400000000FFA40000002C
:107CC000000000005252520000520000000000521A
:107CD00007000700005200000000005200000000F2
:107CE0000000520000FFA4A4FFFFA4FFFFFF00005C
:107CF000A4FFA4A400A4FFA4A4A4A4FFFFA4520072
:107D0000A4A4A452000000A45200000000520000ED
:107D10000000000000000000000000000000000063
:107D200000FFA400000000FFA452000000FFA4A474
:107D3000000000FFFFA4520000A4FFA45200005264
:107D4000A4A4A452000052A4A4A400000000525213
:107D500052FFFFFF00A4FFFFFFA4A4FFFFA45200F7
:107D6000A4FFA452000000A45252000000A452003C
:107D700000000052000000000000000000000000B1
:107D800000FFA400000000FFA452000000FFFFA4B9
:107D9000000000FFFFFF520000FFFFFF520000A4A1
:107DA000A4FFA4520000A4A4FFA400000052525259
:107DB00052FEFEFEFEFEFEFEFEFEFEFEFEFEFEFE8F
:107DC000FEFEFEFEFEFEFEFEFEFEFEFEFEFEFEFED3
:107DD000FEFEFEFEFEFEFEFEFEFEFEFEFEFEFEFEC3
:107DE000FEFEFE06FEFEFEFE000700FEFEFEFE009C
:107DF000FEFEFEFEFEFEFEFEFEFEFEFEFEFEFEFEA3
:107E0000FEFEFEFEFEFEFEFEFEFEFEFEFEFEFEFE92
:107E1000FEFEFE06FEFEFEFE0607FEFEFEFE050759
:107E200000FEFEFE000700FEFEFEFE00FEFEFEFE61
:107E3000FEFEFEFEFEFEFEFEFEFEFEFEFEFEFEFE62
:107E4000FEFEFE05FEFEFEFE060705FEFEFE060722
:107E500007FEFEFE050600FEFEFE000500FEFEFE1D
:107E6000FE00FEFEFEFEFEFEFEFEFEFEFEFEFEFE30
:107E7000FEFEFE06FEFEFEFE050707FEFEFE0607F0
:107E800006FEFEFE070705FEFEFE060700FEFEFEDE
:107E9000050600FEFEFE0000FEFEFEFEFEFEFEFEED
:107EA000FEFEFE05FEFEFEFEFE06FEFEFEFE0507D3
:107EB00005FEFEFE060705FEFEFE050706FEFEFEAB
:107EC000060705FEFEFE050600FEFEFE0000FEFEA5
:107ED000FEFEFE05FEFEFEFEFE06FEFEFEFEFE07AA
:107EE00005FEFEFE050706FEFEFE060705FEFEFE7B
:107EF000050700FEFEFE000500FEFEFEFE00FEFE83
:107F0000FE00000000000000000000005200000021
:107F10000000520000000000A40000000000A400C7
:107F200000000052A400000000A4FF00000000A414
:107F3000FF525252000000000000520000070007EC
:107F4000520000000000520000000000520000003B
:107F50000052000000A4FFFFA4A4FFA40000FFFF44
:107F6000FF525252000000000000520000070007BC
:107F7000520000000000520000000000520000000B
:107F80000052000000A4A4A4A4A4FFA40000A4FF25
:107F9000FF00000000A4FF00000052A4FF0000004A
:107FA000A4FFFF000052FFFFFF000052FFFFFF0091
:107FB00052A4FFA4A400A4FFA4A400525252520051
:107FC00000FFA400FFFFFFFFFFA4A4FFFFA4FFA486
:107FD0000052A452A40000005252A400000052001B
:107FE000520000000000000000000000000000003F
:107FF0000000000000A4FF00000052A4FF000000E9
:10800000A4A4FF000052A4FFFF000052A4FFFF0041
:1080100052A4A4A45200A4A4A4520052525200009C
:1080200000FFA400A4A4FFFFFFA4A4A4A4A4A4A4EC
:108030000052A452A40000005200520000000000B0
:108040000000000000000000000000000000000030
:108050000000000000000000000000000000000020
:108060000000000000000000000000000000000010
:108070000000000000000000000000000000000000
:108080000000FEFEFEFEFE00FEFEFEFEFE00FEFE08
:10809000FEFEFE00FEFEFEFEFE00FEFEFEFEFE00FA
:1080A000FEFEFEFEFE00FEFEFEFEFE00FEFEFEFEEC
:1080B000FE0000FEFEFEFE0000FEFEFEFE0000FED4
:1080C000FEFEFE0000FEFEFEFE0000FEFEFEFE00C6
:1080D00000FEFEFEFE0000FEFEFEFE0000FEFEFEB6
:1080E000FE000000FEFEFE000000FEFEFE0000009E
:1080F000FEFEFE000000FEFEFE000000FEFEFE0092
:108100000000FEFEFE000000FEFEFE000000FEFE7F
:10811000FE00000000FEFE00000000FEFE00000069
:1081200000FEFE00000000FEFE00000000FEFE005B
:10813000000000FEFE00000000FEFE00000000FE49
:10814000FE0000000000FE0000000000FE00000035
:108150000000FE0000000000FE0000000000FE0025
:1081600000000000FE0000000000FE000000000013
:10817000FEFEFEFEFEFE00FEFEFEFEFE00FEFEFE1B
:10818000FEFE00FEFEFEFEFE00FEFEFEFEFE00FE09
:10819000FEFEFEFE00FEFEFEFEFE00FEFEFEFEFEFB
:1081A00000FEFEFEFE0000FEFEFEFE0000FEFEFEE5
:1081B000FE0000FEFEFEFE0000FEFEFEFE0000FED3
:1081C000FEFEFE0000FEFEFEFE0000FEFEFEFE00C5
:1081D00000FEFEFE000000FEFEFE000000FEFEFEB1
:1081E000000000FEFEFE000000FEFEFE000000FE9D
:1081F000FEFE000000FEFEFE000000FEFEFE00008F
:1082000000FEFE00000000FEFE00000000FEFE007A
:10821000000000FEFE00000000FEFE00000000FE68
:10822000FE00000000FEFE00000000FEFE00000058
:1082300000FE0000000000FE0000000000FE000044
:10824000000000FE0000000000FE0000000000FE34
:108250000000000000FE0000000000FE0000000022
:10826000000000000000000000000000000000000E
:10827000000000FEFEFEFEFEFEFEFEFEFEFEFEFE18
:10828000FEFEFEFEFEFEFEFEFEFEFEFEFEFEFEFE0E
:10829000FE000000000000000000000000FEFEFEE6
:1082A000FEFEFEFEFEFEFEFEFEFEFEFEFEFEFEFEEE
:1082B000FEFEFEFEFEFEFEFEFEFEFEFEFEFEFEFEDE
:1082C000FE000000000000FEFEFEFEFEFEFEFEFEC2
:1082D000FEFEFEFEFEFEFEFEFEFEFEFEFEFEFEFEBE
:1082E000FEFEFEFEFEFEFEFEFEFEFEFEFEFEFEFEAE
:1082F000FEFEFEFE2020FEFE27201827FE271F1F61
:108300001F1F27271F001F001F371F001F001F1FD1
:108310001F1F1F1F1E1F1F0000271EFE1F1F1E1EC8
:10832000FE47474747474747474747474747474726
:1083300047474747474747474747474747474747CD
:1083400047474747474747474747474747474747BD
:10835000473838383838383838383838383838388E
:10836000383838383838383838383838383838388D
:10837000383838383838383838383838383838387D
:1083800038FEFEFEFEFEFEFEFEFEFEFE00FEFEFED1
:10839000FEFEFEFEFEFE00FEFEFEFEFEFEFEFEFEFB
:1083A000FEFEFEFEFEFEFEFEFE00FEFEFEFEFEFEEB
:1083B000FEFEFE00FEFE00FEFEFEFEFE00FEFEFED7
:1083C000FEFEFEFEFEFE0000FEFEFEFEFEFEFEFEC9
:1083D00000FEFEFEFEFEFEFEFE0000FEFEFEFEFEB7
:1083E00000FE0000FE0000FEFEFEFEFE00FEFEFEA1
:1083F000FEFEFE00FEFE0000FEFEFEFEFE0000FE93
:108400000000FEFEFEFEFEFE000000FE00FEFE007E
:1084100000FE0000000000FEFE00FE0000FE00FE68
:10842000FEFE0000FE000000FEFEFEFE000000005A
:108430000000FE0000FEFEFE000000FE0000FE0048
:1084400000FE000000000000FE00FE0000FE00FE36
:10845000000000000000000000FEFE000000000020
:108460000000FE000000FE00000000FE0000000012
:108470000000000000000000FE00000000FE00FE02
:10848000000000000000000000FE000000000000EE
:10849000000000000000FE00000000F0F0F0F0F02E
:1084A000F0FEFE00FEFEFEFEFEFEFEFEFE00FEFEF6
:1084B000FE00FEFEFEFEFEFEFEFEFE00FEFEFEFED8
:1084C000FEFEFEFEFE00FEFEFE00FEFEFEFEFEFEC8
:1084D000FE00FE00FE00FEFEFEFEFEFEFE00FE00B2
:1084E000FE00FEFEFEFEFEFEFE00FE00FE00FEFEA4
:1084F000FEFEFEFEFE00FE00FE00FEFE00FEFEFE94
:10850000FE00FE00FE00FEFE00FEFEFE0000FE007D
:10851000FE00FEFE00FE00FE0000FE00FE00FEFE6D
:1085200000FE00FE0000FE00FE00FEFE00FE00FE5B
:10853000FE0000000000FEFE000000FE0000000043
:10854000000000FE00FE00FE000000000000FEFE35
:1085500000FE00FE00000000000000FE00FE00FE25
:10856000000000000000000000FE0000000000000D
:1085700000000000000000FE0000000000000000FD
:1085800000FE00000000000000000000000000FEEF
:1085900000000000000000000000000000000000DB
:1085A00000000000000000000000000000000000CB
:1085B00000000000000000000000000000000000BB
:1085C0000000000000000003030303030303030390
:1085D0000404050304040405050405050505060651
:1085E0000606060606070606060606070606070727
:1085F000070000000000000300000000000401006C
:108600000000000504000000000504000000000652
:10861000050000000006050000000006050000003F
:108620000000000000000000030303030301040432
:1086300004050504050606050504060605050501ED
:1086400005050506060005060606060005060606DB
:1086500006000000000000030301030303050403F8
:1086600004040405040504050505050405050506BF
:1086700005040405060605040405060605040305AD
:1086800006000000000000030303030303040404C6
:108690000405050506060606050506060605050683
:1086A000060606060606060606060506060606046D
:1086B0000300000000000004040404040405050590
:1086C000050505050606060606060606060606064E
:1086D0000606060606060606070707040606070737
:1086E0000700000000000004040404010105050562
:1086F0000502020606060504050606060605060628
:10870000060606050607060606050606050606040D
:108710000600000000000004040303030205050531
:1087200004030305060505050506060606060606F6
:1087300006060606060606060606060607070706D6
:108740000600000000000002020303030403040407
:1087500004040506060505050506060505050606C5
:1087600006060606060606060606060606060607A8
:1087700007000000000000040404010104050505D1
:1087800002020405050503030506060504040506A3
:108790000605040405060606040406070606060484
:1087A00004000000000000040403030303050504A3
:1087B0000405050505050505050606060606060663
:1087C0000606060606060606060606060607070647
:1087D0000600000000000003030303030405040473
:1087E0000505050505050506050606060606050632
:1087F000060606060606060606060606060506061A
:108800000600000000000004000000000004010059
:10881000000000050400000000060501000000063D
:108820000504000000060505010000060605040118
:108830000000000000000000000000000000000038
:108840000001020000000302030000010303030013
:1088500000030303040001030304040103030304EE
:1088600005000000000000020203030303030303EA
:1088700004040403040405050504040505060504B1
:10888000050506060605050606060605060606068D
:1088900007000000000000000000000000020100CE
:1088A00000000005050400000006060501000006A2
:1088B0000605040000070606050100060706060572
:1088C000010000000000000000000303030000019D
:1088D000030304000003030505000004030506006C
:1088E0000103040406010104050506010101050652
:1088F0000500000000000003030303000005050657
:108900000501000506060604000505060605000526
:108910000606060500050706060501070606060504
:108920000100000000000000000000000000000046
:10893000000001000000000003000000000103002F
:10894000000000040300000002040301000404030B
:1089500003000000000000030202030304030303FA
:10896000030304030303040405030B0B04040503BE
:108970000B0B0405060B0B040405060B0B04050585
:10898000060606070707070707070707070707077A
:108990000707070707070707060707070707060769
:1089A000060507070606060406070606030406066C
:1089B0000606050000000006050000000006050090
:1089C0000000000501000000000500000000000597
:1089D000000000000005000000000005000000008D
:1089E000000004060607060001050607070000054B
:1089F0000607070000050607060000050607060033
:108A00000005060706000005060706000005060724
:108A10000606050302050606050201020506050114
:108A2000010105050101010105050101010105051E
:108A30000101010505050101000404050100000014
:108A400000060606050303060606060303060606D9
:108A500005020303020501010202010400010101F4
:108A60000000000001000000000001000000000004
:108A70000503060607070705060707070606060794
:108A80000707060506070706060506070706050584
:108A90000607060501050607060500060707060581
:108AA000000605060502060603050101020602048A
:108AB00000010102000000000100000000000000B1
:108AC00000000000000000000000000000000000A6
:108AD0000006070707060606060707060605060737
:108AE0000706050506070706050506070706050527
:108AF0000607060501050607060500050607060523
:108B00000006050606060603020205060402010029
:108B10000405020100000000010000000000000048
:108B20000000000000000000000000000000000045
:108B300000070706060404060706060404060606E0
:108B400006040402060606030401050605020300E6
:108B500005050201020005050001010000000000FA
:108B600001060606070706060607070707060607A3
:108B7000070707060607070707060607070706058C
:108B80000607070606050607070605050607060584
:108B90000106060506060506060405050306060386
:108BA00005040106050200000106050000000002A0
:108BB00000000000000000000000000000000000B5
:108BC000000505050402010405050403020305046C
:108BD0000304030104030304040103030304040066
:108BE0000303030404010303030404020303030453
:108BF0000402030304050503030405050603040535
:108C00000506060304050506050405050605050415
:108C10000506050302050506050201050606050110
:108C200000060606070706060607070607060607E4
:108C300006060706070606050606060606030602DA
:108C40000505020205000404010004000000000004
:108C500000070706060501070706070605070707B9
:108C600007060506060707060506060707060502A6
:108C700004060707060102060607060001050607A7
:108C800006010101050606010100010506010000BB
:108C900000050600000000010501000000000505B8
:108CA00000000000010500000000000500000000B9
:108CB0000006060606050206060606050207070662
:108CC000060502060706060505060606060505054D
:108CD000060606060505060707060501050607063A
:108CE0000501010403030B02020303030B02020349
:108CF0000303030203030303040304030304040440
:108D00000403030405040403040405040404050522
:108D1000050B040405060504040505060304040503
:108D200006050304050506050205050505040005FD
:108D3000050201000005050100000005010000001A
:108D400000050103060606000101050606000001F4
:108D500005060600000005060600000105060600DF
:108D600000050606050000050606050001050606C5
:108D700005050000000000050000000000050000DF
:108D800000000005000000000005000000000001D8
:108D900000000000000000000000000000000000D3
:108DA000000000050607060000050607060000058E
:108DB0000607060000050606050000050606050074
:108DC0000005060605000005060605000005060666
:108DD000050500000000000500000000000500007F
:108DE0000000000100000000000000000000000082
:108DF0000000000000000000000000000000000073
:108E00000000000000000500000000000500000058
:108E10000000050000000000050000000001050042
:108E20000000000506000000000506000000000527
:108E300006060707060500060706050100060706E1
:108E400005000006060501000006060500000007F3
:108E500006050000000706050000000605010000E9
:108E60000000000000000000000000000000000002
:108E700000000000000000000000000000000000F2
:108E800000000000000000000000000000000000E2
:108E9000000506070605010105060706050005068B
:108EA000070706000506070707000506070707006E
:108EB000010506070700000506070600000506066F
:108EC0000300000000000001010505050003020683
:108ED0000606020606060706060707070707060630
:108EE0000606070707050505060706010001030634
:108EF000060000000000000000000000000000006C
:108F00000000000500000000000501000000000650
:108F1000050000000006050000000002000000003F
:108F200000050607060500050607060500050607F5
:108F300006050001050606050100050606060200F5
:108F400005060706060005060707060005060707CB
:108F50000700000000000000000000000100000009
:108F600000000200000000040401000102050602E6
:108F70000505060606040606070706060707060691
:108F800006030303020305030402010205040401AE
:108F900001010505010101010505010101010505A9
:108FA00001010101050501010101050501010101A1
:108FB0000505060605000005060501000006060574
:108FC0000000000606050000000606050000000679
:108FD0000501000000060500000000060500000075
:108FE0000000000000000000000000000000000081
:108FF0000000000000000000000000000000000071
:109000000000000000000000000000000000000060
:10901000000000050607060000050607060000051B
:1090200006070600000506070600000506070600FD
:109030000001050606000000050606000000010507
:10904000060500000000000500000000000500000B
:109050000000000500000000000500000000000501
:1090600000000000000500000000000500000000F6
:1090700000000506070606000506060606000506AA
:109080000607070005030607070004020606070097
:1090900000010206060000000105060000000005B0
:1090A0000605050606060606050606060607050663
:1090B0000606060706060606040706060606040751
:1090C000070606040307070606030207070605024C
:1090D0000105000000000005000000000005000080
:1090E000000000050000000000050100000000066F
:1090F000050000000005050000000001050000005B
:109100000001010506060501010506060501010528
:10911000060605010105060605010105060605010D
:1091200001050606050001050606050000050607FF
:109130000600000000000000000000000000000029
:10914000000000000000000000000000000000001F
:109150000000000000010000000000050000000009
:1091600000000005060605000005060605000005CE
:1091700006060500000506050100000506050000BD
:1091800000050605000000050605000000050605AF
:1091900000000000000000000000000000000000CF
:1091A00000000000000000000000000000000000BF
:1091B00000000000000000000000000000000000AF
:1091C0000000000001050600000005060700000081
:1091D000050607000000050606000001050606005A
:1091E0000005060605000005060605000005060642
:1091F0000506050000000006050000000006050049
:109200000000000501000000000500000000000152
:10921000000000000000000000000000000000004E
:10922000000000000000000000000000000000003E
:10923000000000000000000000000000000000002E
:10924000000000000000000000000000000000001E
:1092500000000105060501000506060500000506DB
:1092600006050000010506050000000506050000D2
:1092700000050605000000050605000000050605BE
:1092800000000000010505000000000505000000C9
:1092900000050500000000050100000000040000BA
:1092A00000000000000000000000000000000000BE
:1092B00000010000000000000000000000000000AD
:1092C000000000000000000000000000000000009E
:1092D000000000000000000000000000000000008E
:1092E0000000050607070700050607070700050633
:1092F000070706000506070706000506070605001E
:109300000506070605000506070605000105060611
:109310000507060605060607060201020606050001
:109320000001050200000000010100000000000033
:10933000000000000000000000000000000000002D
:1093400001050101010105060501010105060502EE
:1093500001020505060502020205060502020305D3
:1093600006060503030506060503020506060502B3
:1093700002060500000000060500000000060500CA
:1093800000000006050000000005050000000006C2
:1093900005000000000505010000000205050000B1
:1093A00000000000000506000000000506000000A7
:1093B000000506000000000505000000000505008E
:1093C0000000000505000000000505000000000584
:1093D0000505000000000005000000000005000079
:1093E000000000010000000000000000000000007C
:1093F000000000000000000000000000000000006D
:109400000000000000050600000000050600000046
:10941000000506000000000506000000000506002B
:10942000000000050600000001050600000005061A
:1094300007070706050100070606010000070606E4
:1094400001000007070605000007070605010007E1
:1094500005070605000705070605000605060605BB
:1094600000000400000000000000000000000000F8
:1094700000000000000000000000000000000000EC
:1094800000000000000000000000000000000000DC
:1094900000000005060706000001050607000000A1
:1094A0000506070000000105060000000005060093
:1094B00000000001050000000000050000000000A1
:1094C0000005010000000006050000000006050080
:1094D0000000000605010000010606030101020666
:1094E0000606050505060606060606020606060623
:1094F0000600010506050000050606050001050633
:10950000060500050606050100060606050000061C
:109510000606040000060605040000060504030014
:10952000000000000000000000000000000000003B
:10953000000000000000000000000000000000002B
:10954000000000000000000000000000000000001B
:1095500000000105060605000506060501000506D2
:1095600006050100050606050200050606060300BD
:10957000050607060500050606060600050606069A
:1095800006000000000000000000000000010000D4
:1095900000000001010404010402020505030405A2
:1095A000050605050406060505040306050504036E
:1095B00003000000000000000000000000000000A8
:1095C0000000000404000000000403000000000389
:1095D0000100000000020000000000010000000087
:1095E0000000000506050100000105060500000059
:1095F000050605000000050605000000050606003A
:10960000000005060600000005060600000005062D
:109610000600000000000000000000000000000044
:10962000000000010000000000030100000000062F
:1096300005050504050606060505060606060505D4
:109640000500000000000000000000000000000015
:109650000000000000000000000000000000000505
:1096600004000000000504000000000200000000EB
:1096700000000005060605000005060605000005B9
:10968000060605000005060606000005060606009B
:10969000000506060600000506060600000506068B
:1096A00006000000000002010000000405010100A6
:1096B0000205050301040506050403050605050664
:1096C0000505050505060606050403060605050449
:1096D000030506050402010606050401010504044C
:1096E000030100050403010000040302000000035D
:1096F000030100000003020000000003010000005D
:10970000000205050100000105060500000105062F
:10971000050100000105060500000005060602001F
:1097200000050606060000040606060000050604FD
:109730000600000000000000000000000000000023
:109740000000000000000000000000000000000514
:1097500000000000000602010001020606050505E2
:1097600005000000010505000000050605000001D8
:1097700005060500000506060500020606050505A6
:1097800006060201000506050100000606040000A9
:1097900000000000000000000000000000000000C9
:1097A00000000000000000000000000000000000B9
:1097B00000000000000000000000000000000000A9
:1097C0000000000005060700000005060600000175
:1097D000050606000005060606000005060605004B
:1097E000000506050100000506050000000505014D
:1097F000000604060605000603040605000502032C
:109800000605010201020506050100010506050025
:109810000000010506000000000506000000000130
:109820000500000000000000000000000000000033
:109830000000000000000000000100000000000522
:10984000000000000005000000000005000000000E
:109850000000000000000000000000000000000008
:1098600000000000000000000000000000000000F8
:1098700000000000000000000000000000000000E8
:1098800000000505060606000002050505000000AB
:1098900004040400000000000000000000000000BC
:1098A00000000000000000000000000000000000B8
:1098B0000005040403000002030302000001010389
:1098C0000200000000010200000000000200000091
:1098D0000000000000000000000000000000000088
:1098E0000000000000000000000000000000000078
:1098F0000000000000000000000000000000000068
:109900000000000000000000000000000000000057
:109910000000050506060600040606060500040507
:109920000605040004050504020004050404010002
:109930000404020000000403000000000000000016
:1099400000050504030302050403030200030303E7
:1099500002000002030100000000020000000000FD
:1099600000000000000000000000000000000000F7
:1099700000000000000000000000000000000000E7
:1099800000000000000000000000000000000000D7
:1099900000000000000000000000000000000000C7
:1099A000000000000405060000000105060000009C
:1099B0000004050000000004030000000004010092
:1099C0000000000000000000000000000000000097
:1099D000000505040404030505030503030404034B
:1099E000040303030303020303030302010303014C
:1099F0000201000000000200000000000000000062
:109A00000001000000000000000000000000000055
:109A10000000000000000000000000000000000046
:109A20000000000000000000000000000000000036
:109A300000000005060505000005050302000004FE
:109A40000502010000010401010000000401000002
:109A500000000400000000000400000000000000FE
:109A600000050505040303020404050303010303C1
:109A700004030300010302030100000201030000CC
:109A800000000000000000000000000000000000D6
:109A900000030000000000010000000000000000C2
:109AA00000000000000000000000000000000000B6
:109AB00000000000000000000000000000000000A6
:109AC000000000050502040000040100000000047D
:109AD0000000000000000000000000000000000086
:109AE0000000000000000000000000000000000076
:109AF0000005060606050601020506060500000427
:109B0000050404000000020403000000000302003A
:109B10000000000000000000000000000000000045
:109B20000006050400000005040100000004030015
:109B30000000000200000000000000000000000023
:109B40000000000000000000000000000000000015
:109B50000000000000000000000000000000000005
:109B600000000000000000000000000000000000F5
:109B700000000000000000000000000000000000E5
:109B800000000105050000000505010000000505B5
:109B900000000000050500000000040400000000B3
:109BA00000000000000000000000000000000000B5
:109BB000000000000000050000000000050000009B
:109BC000000005000000000001000000000000008F
:109BD0000000000000000000000000000000000085
:109BE0000005000000000005000000000005000066
:109BF000000000050000000000040000000000005C
:109C00000000000000000000000000000000000054
:109C1000000000FF03000000BF03BF03003F03007C
:109C2000003F033737373737032703000027031F69
:109C30000300001F030703000007030000000000EB
:109C400000FFFFFFFF0300BF030000BF033F03004F
:109C5000003F033737373703002703000027031F70
:109C60000300001F030707070703000000000000B0
:109C70000000FFFFFF0300BF030000BF033F03001E
:109C80000000003703000000002703000000001F51
:109C90000300001F03000707070300000000000087
:109CA00000FFFFFFFF0300BF030000BF033F0300EF
:109CB000003F033703000037032703000027031F7B
:109CC0000300001F03070707070300000000000050
:109CD00000FFFFFFFFFF03BF03000000003F030082
:109CE0000000003737373703002703000000001F4C
:109CF000030000000007070707070300000000003B
:109D000000FFFFFFFFFF03BF03000000003F030051
:109D10000000003737373703002703000000001F1B
:109D20000300000000070300000000000000000026
:109D30000000FFFFFF0300BF030000BF033F03005D
:109D40000000003703003737032703000027031FF5
:109D50000300001F030007070703000000000000C6
:109D600000FF030000FF03BF030000BF033F030029
:109D7000003F033737373737032703000027031F18
:109D80000300001F0307030000070300000000009A
:109D900000FFFFFFFFFF030000BF03000000003FC4
:109DA000030000000037030000000027030000004C
:109DB000001F03000007070707070300000000005B
:109DC0000000FFFFFFFF0300000000BF03000000D2
:109DD000003F030000000037030000000027031FBE
:109DE0000300001F03000707070300000000000036
:109DF00000FF030000FF03BF0300BF03003F033F5A
:109E00000300003737030000002703270300001F6B
:109E100003001F0300070300000703000000000009
:109E200000FF0300000000BF03000000003F03002C
:109E30000000003703000000002703000000001F9F
:109E400003000000000707070707030000000000E9
:109E500000FF030000FF03BFBF03BFBF033F033F7B
:109E6000033F033703000037032703000027031FC6
:109E70000300001F030703000007030000000000A9
:109E800000FF030000FF03BFBF0300BF033F033F0A
:109E9000033F033703003737032703000027031F5F
:109EA0000300001F03070300000703000000000079
:109EB0000000FFFFFF0300BF030000BF033F0300DC
:109EC000003F033703000037032703000027031F69
:109ED0000300001F03000707070300000000000045
:109EE00000FFFFFFFF0300BF030000BF033F0300AD
:109EF000003F033737373703002703000000001FF8
:109F00000300000000070300000000000000000044
:109F10000000FFFFFF0300BF030000BF033F03007B
:109F2000003F033703000037032703270327031FDE
:109F300003001F1F030007070703000000000000C5
:109F400000FFFFFFFF0300BF030000BF033F03004C
:109F5000003F033737373703002703000027031F6D
:109F60000300001F030703000007030000000000B8
:109F70000000FFFFFF0300BF030000BF033F03001B
:109F80000000000037373703000000000027031FE0
:109F90000300001F03000707070300000000000084
:109FA00000FFFFFFFFFF030000BF03000000003FB2
:109FB000030000000037030000000027030000003A
:109FC000001F030000000007030000000000000065
:109FD00000FF030000FF03BF030000BF033F0300B7
:109FE000003F033703000037032703000027031F48
:109FF0000300001F03000707070300000000000024
:10A0000000FF030000FF03BF030000BF033F030086
:10A01000003F033703000037032703000027030036
:10A020001F031F03000000070300000000000000E2
:10A0300000FF030000FF03BF030000BF033F030056
:10A04000003F033703000037032703270327031FBD
:10A050001F031F1F03070300000703000000000089
:10A0600000FF030000FF03BF030000BF03003F0326
:10A070003F03000000370300000027032703001FF1
:10A080000300001F03070300000703000000000097
:10A0900000FF030000FF03BF030000BF03003F03F6
:10A0A0003F0300000037030000000027030000000A
:10A0B000001F030000000007030000000000000074
:10A0C00000FFFFFFFFFF0300000000BF03000000D0
:10A0D0003F03000000370300000027030000001FBB
:10A0E0000300000000070707070703000000000047
:10A0F00000000000202000002720182700271F1F35
:10A100001F1F27271F001F001F371F001F001F1FB3
:10A110001F1F1F1F1E1F1F0000271E001F1F1E1EA8
:10A12000000000000000000000000000000000002F
:10A13000000000000000000000000000000000001F
:10A14000000000000000000000000000000000000F
:10A15000000000FF5B000000FF5BFF5B00FF5B0097
:10A1600000FF5BFFFFFFFFFF5BFF5B0000FF5BFF8C
:10A170005B0000FF5BFF5B0000FF5B000000000076
:10A1800000FFFFFFFF5B00FF5B0000FF5BFF5B006A
:10A1900000FF5BFFFFFFFF5B00FF5B0000FF5BFF5B
:10A1A0005B0000FF5BFFFFFFFF5B000000000000A3
:10A1B0000000FFFFFF5B00FF5B0000FF5BFF5B0039
:10A1C000000000FF5B00000000FF5B00000000FFDC
:10A1D0005B0000FF5B00FFFFFF5B00000000000072
:10A1E00000FFFFFFFF5B00FF5B0000FF5BFF5B000A
:10A1F00000FF5BFF5B0000FF5BFF5B0000FF5BFF9E
:10A200005B0000FF5BFFFFFFFF5B00000000000042
:10A2100000FFFFFFFFFF5BFF5B00000000FF5B0034
:10A22000000000FFFFFFFF5B00FF5B00000000FF7E
:10A230005B00000000FFFFFFFFFF5B00000000006D
:10A2400000FFFFFFFFFF5BFF5B00000000FF5B0004
:10A25000000000FFFFFFFF5B00FF5B00000000FF4E
:10A260005B00000000FF5B00000000000000000039
:10A270000000FFFFFF5B00FF5B0000FF5BFF5B0078
:10A28000000000FF5B00FFFF5BFF5B0000FF5BFF68
:10A290005B0000FF5B00FFFFFF5B000000000000B1
:10A2A00000FF5B0000FF5BFF5B0000FF5BFF5B00EC
:10A2B00000FF5BFFFFFFFFFF5BFF5B0000FF5BFF3B
:10A2C0005B0000FF5BFF5B0000FF5B000000000025
:10A2D00000FFFFFFFFFF5B0000FF5B00000000FFCF
:10A2E0005B00000000FF5B00000000FF5B0000005F
:10A2F00000FF5B0000FFFFFFFFFF5B0000000000AE
:10A300000000FFFFFFFF5B00000000FF5B0000009C
:10A3100000FF5B00000000FF5B00000000FF5BFF30
:10A320005B0000FF5B00FFFFFF5B00000000000020
:10A3300000FF5B0000FF5BFF5B00FF5B00FF5BFF5C
:10A340005B0000FFFF5B000000FF5BFF5B0000FFA6
:10A350005B00FF5B00FF5B0000FF5B000000000094
:10A3600000FF5B00000000FF5B00000000FF5B00DF
:10A37000000000FF5B00000000FF5B00000000FF2A
:10A380005B00000000FFFFFFFFFF5B00000000001C
:10A3900000FF5B0000FF5BFFFF5BFFFF5BFF5BFFFE
:10A3A0005BFF5BFF5B0000FF5BFF5B0000FF5BFF91
:10A3B0005B0000FF5BFF5B0000FF5B000000000034
:10A3C00000FF5B0000FF5BFFFF5B00FF5BFF5BFFCD
:10A3D0005BFF5BFF5B00FFFF5BFF5B0000FF5BFF62
:10A3E0005B0000FF5BFF5B0000FF5B000000000004
:10A3F0000000FFFFFF5B00FF5B0000FF5BFF5B00F7
:10A4000000FF5BFF5B0000FF5BFF5B0000FF5BFF8B
:10A410005B0000FF5B00FFFFFF5B0000000000002F
:10A4200000FFFFFFFF5B00FF5B0000FF5BFF5B00C7
:10A4300000FF5BFFFFFFFF5B00FF5B00000000FF12
:10A440005B00000000FF5B00000000000000000057
:10A450000000FFFFFF5B00FF5B0000FF5BFF5B0096
:10A4600000FF5BFF5B0000FF5BFF5BFF5BFF5BFFD1
:10A470005B00FFFF5B00FFFFFF5B000000000000D0
:10A4800000FFFFFFFF5B00FF5B0000FF5BFF5B0067
:10A4900000FF5BFFFFFFFF5B00FF5B0000FF5BFF58
:10A4A0005B0000FF5BFF5B0000FF5B000000000043
:10A4B0000000FFFFFF5B00FF5B0000FF5BFF5B0036
:10A4C00000000000FFFFFF5B0000000000FF5BFFDB
:10A4D0005B0000FF5B00FFFFFF5B0000000000006F
:10A4E00000FFFFFFFFFF5B0000FF5B00000000FFBD
:10A4F0005B00000000FF5B00000000FF5B0000004D
:10A5000000FF5B00000000FF5B0000000000000097
:10A5100000FF5B0000FF5BFF5B0000FF5BFF5B0079
:10A5200000FF5BFF5B0000FF5BFF5B0000FF5BFF6A
:10A530005B0000FF5B00FFFFFF5B0000000000000E
:10A5400000FF5B0000FF5BFF5B0000FF5BFF5B0049
:10A5500000FF5BFF5B0000FF5BFF5B0000FF5B0039
:10A56000FF5BFF5B000000FF5B00000000000000DD
:10A5700000FF5B0000FF5BFF5B0000FF5BFF5B0019
:10A5800000FF5BFF5B0000FF5BFF5BFF5BFF5BFFB0
:10A59000FF5BFFFF5BFF5B0000FF5B000000000054
:10A5A00000FF5B0000FF5BFF5B0000FF5B00FF5BE9
:10A5B000FF5B000000FF5B000000FF5BFF5B00FF34
:10A5C0005B0000FF5BFF5B0000FF5B000000000022
:10A5D00000FF5B0000FF5BFF5B0000FF5B00FF5BB9
:10A5E000FF5B000000FF5B00000000FF5B0000005D
:10A5F00000FF5B00000000FF5B00000000000000A7
:10A6000000FFFFFFFFFF5B00000000FF5B0000009A
:10A61000FF5B000000FF5B000000FF5B000000FF2D
:10A620005B00000000FFFFFFFFFF5B000000000079
:10A630000000000000000000FFFF5B000000FFFFC3
:10A640005B000000000000000000FFFF5B00000056
:10A65000FFFF5B00000000000000000000000000A1
:10A6600000000000000000000000000000000000EA
:10A6700000000000000000000000000000000000DA
:10A68000FFFF5B000000FFFF5B0000000000000018
:10A690000000FFFF5B000000FFFF5B000000FFFF0A
:10A6A0005B000000FF5B00000000000000000000F5
:10A6B000FFFF5B000000FFFF5B00000000000000E8
:10A6C0000000FFFF5B000000FFFF5B000000FF5B7E
:10A6D000000000000000000000000000000000007A
:10A6E000000000000000000000000000000000006A
:10A6F00000000000202000002720182700271F1F2F
:10A700001F1F27271F001F001F371F001F001F1FAD
:10A710001F1F1F1F1E1F1F0000271E001F1F1E1EA2
:10A720000028010102030405060708090A0B0C0DA5
:10A730000E0F101112131415161718191A1B1C1DC1
:10A740001E1F20010203040506FEFEFEFEFEFEFEA5
:10A75000FEFEFEFEFEFEFEFEFEFEFEFEFEFEFEFE19
:10A76000FEFEFEFEFEFEFEFEFEFEFEFEFEFEFEFE09
:10A77000FEFEFEFEFEFEFEFEFEFEFEFEFEFEFEFEF9
:10A78000FEFEFEFEFEFEFEFEFEFE08FEFEFEFE08D5
:10A7900018FEFEFEFE0818FEFEFEFEFE08FEFEFE91
:10A7A000FEFEFEFEFEFEFEFEFEFEFE1808FEFEFEA5
:10A7B00018081808FE1808FE1808FE08FE1808FEFB
:10A7C000FEFEFE091808FEFEFE081808FEFEFE0842
:10A7D0001808FE080A140A0A09FEFEFEFEFEFEFE26
:10A7E000FEFEFEFEFEFEFEFEFEFEFEFEFEFEFEFE89
:10A7F000FEFEFEFEFEFEFEFEFEFEFEFEFEFEFEFE79
:10A80000091808FEFE08180808FEFEFEFEFE00FEFF
:10A81000FEFEFEFE0AFEFEFEFE001EFEFEFEFE0A1E
:10A8200027FEFEFEFE1D27FEFEFE091F27FEFEFE82
:10A83000132727FEFEFE15272713151E140A0B1FCC
:10A840001D1F15140B271D1E15150A271E27151D64
:10A850000B1F1E1F151F0B1F131D141F141E001E80
:10A86000130A1513001F14001401FE1808FEFE0140
:10A87000FE1800FEFE011808FEFEFE0A001800FE8B
:10A88000FE0A011808FEFE0A011808FEFE0B0A0067
:10A8900000FEFE0A0A00FEFEFEFEFEFE1E2727FE4A
:10A8A000FE0127271FFEFE0B27271DFEFE1427276C
:10A8B00013FEFE15272727FE001E270B1D0001276C
:10A8C0001F091D000A270914270A001F14000A0087
:10A8D000001F14000000001E1400000000151400EA
:10A8E00000271E1E1D0B092727271F27141F271FA0
:10A8F0001F27141F27271E271D0A0B00FEFEFE0A16
:10A900000B00FEFEFE090B0900FEFE090B0900FE0E
:10A91000FE010B0A01FEFE010B0A00FEFE0A0B0AF5
:10A9200000FEFE000B0B00FEFE000B2709132700A4
:10A9300014271F091E00141F270A0A00141E1F1EB9
:10A940000000141E1F1F1400141E1E1E1E00141DC6
:10A950001E1527000B151E141F1F27271E1E1D1F47
:10A96000271F1E1F15001F1E1E1F150014011E018C
:10A9700014000A00090001000000000000010A00A4
:10A980000A00001514011E010A0B000B00FEFE094F
:10A99000000A00FEFE00000A00FEFE000101FEFEAD
:10A9A000FE000101FEFEFE010A01FEFEFE0B01009B
:10A9B000FEFEFE0B0100FEFEFE000A1415141FFE33
:10A9C000090B0B0B1FFE000A0A0A15FEFE0101010E
:10A9D00014FEFEFE000014FEFEFEFE000AFEFEFE59
:10A9E000FEFE00FEFEFEFEFEFE141F1F1E140A14D5
:10A9F0001E1E1E0B0A14151E150B090B1415140A26
:10AA0000010B13150B09000B0B0B0A0100000109C8
:10AA10000100FEFEFEFEFEFEFE0A01FEFEFEFE013F
:10AA200000FEFEFEFE01FEFEFEFEFE01FEFEFEFE3E
:10AA3000FE00FEFEFEFEFEFEFEFEFEFEFEFEFEFE34
:10AA4000FEFEFEFEFEFEFEFEFE0A001F14000A00D1
:10AA5000001F14000000071E14070000001514005A
:10AA600000271E1E1D0B092727271F27141F271F1E
:10AA70001F27141F27271E271D0A001F14000A0066
:10AA8000001F14000000061E14060000001514002C
:10AA900000271E1E1D0B092727271F27141F271FEE
:10AAA0001F27141F27271E271D0A001F14000A0036
:10AAB000001F14000000041E140400000015140000
:10AAC00000271E1E1D0B092727271F27141F271FBE
:10AAD0001F27141F27271E271D0A001F14000A0006
:10AAE000001F14000000031E1403000000151400D2
:10AAF00000271E1E1D0B092727271F27141F271F8E
:10AB00001F27141F27271E271D0A001F14000A00D5
:10AB1000001F14000000011E1401000000151400A5
:10AB200000271E1E1D0B092727271F27141F271F5D
:10AB30001F27141F27271E271D4841505059204802
:10AB4000414C4C4F5745454E210000000102030384
:10AB50000400000102050506070808090000000AB4
:10AB60000B0B0C000027282928272829282720201C
:10AB700020202020202020202020202020202020D5
:10AB80002020202020005F205F205F20435245448A
:10AB9000495453205F205F205F0050524F4752417D
:10ABA0004D4D494E475B0047524150484943535B26
:10ABB00000434C415920434F5747494C4C004D5599
:10ABC000534943414C2053434F52455B00424A4F47
:10ABD000524E204C594E4E4500415544494F20415C
:10ABE0005353495354414E43455B00414C45432028
:10ABF000424F5552515545004752454554494E47DD
:10AC0000535B0055484848485C5C5C2054484552BA
:10AC1000455E53004E4F424F445920454C5345200A
:10AC2000494E2054484500555A45424F58205343F9
:10AC3000454E45205945545D5D5D00544543484EA1
:10AC400049515545535B00564552544943414C20A8
:10AC50005343524F4C4C494E4700414C5445524E81
:10AC60004154494E47205350524954455300464F92
:10AC70005220455854454E44454420475245595367
:10AC8000005350524954455320464F522044495492
:10AC90004845520057495045204F4E204D41494E9E
:10ACA000205449544C450053505249544553204672
:10ACB0004F52205445585400574954482053494E48
:10ACC00045204F464653455420544F0041564F4966
:10ACD00044204C494E45204C494D495453004D5554
:10ACE0004C5449504C452054494C452053455453ED
:10ACF0000053484152454420464F4E5420414E4453
:10AD000000535052495445204752415048494353FB
:10AD10000020202020202054484520454E445C003F
:10AD20002020202020205F205F205F202020202066
:10AD30002000FFFE00010260626567696C6E70733F
:10AD400075777A7C7E80838587898B8D8F919395AB
:10AD500097999B9D9FA0A2A4A6A7A9AAACADAEB0AF
:10AD6000B1B2B4B5B6B7B8B9BABABBBCBDBDBEBE58
:10AD7000BFBFBFC0C0C0C0C0C0C0C0C0BFBFBFBEDB
:10AD8000BEBDBDBCBBBABAB9B8B7B6B5B4B2B1B046
:10AD9000AEADACAAA9A7A6A4A2A09F9D9B9997958A
:10ADA00093918F8D8B89878583807E7C7A7775736D
:10ADB000706E6C69676562605E5B59575452504DA6
:10ADC0004B49464442403D3B39373533312F2D2BDB
:10ADD0002927252321201E1C1A19171614131210B7
:10ADE0000F0E0C0B0A0908070606050403030202EE
:10ADF000010101000000000000000000010101024B
:10AE0000020303040506060708090A0B0C0E0F10BF
:10AE10001213141617191A1C1E2021232527292B5B
:10AE20002D2F31333537393B3D40424446494B4D58
:10AE300050525457595B5E80868C92989EA5AAB05A
:10AE4000B6BCC1C6CBD0D5DADEE2E6EAEDF0F3F56A
:10AE5000F8FAFBFDFEFEFFFFFFFEFEFDFBFAF8F534
:10AE6000F3F0EDEAE6E2DEDAD5D0CBC6C1BCB6B08F
:10AE7000AAA59E98928C868079736D67615A554F0A
:10AE800049433E39342F2A25211D1915120F0C0A6A
:10AE90000705040201010000000101020405070A80
:10AEA0000C0F1215191D21252A2F34393E43494F05
:10AEB000555A61676D73797F868C92989EA5AAB06A
:10AEC000B6BCC1C6CBD0D5DADEE2E6EAEDF0F3F5EA
:10AED000F8FAFBFDFEFEFFFFFFFEFEFDFBFAF8F5B4
:10AEE000F3F0EDEAE6E2DEDAD5D0CBC6C1BCB6B00F
:10AEF000AAA59E98928C868079736D67615A554F8A
:10AF000049433E39342F2A25211D1915120F0C0AE9
:10AF10000705040201010000000101020405070AFF
:10AF20000C0F1215191D21252A2F34393E43494F84
:10AF3000555A61676D73790000000000000101013E
:10AF400002020203030404050506070708090A0BA9
:10AF50000B0C0D0E0F1011121415161718191B1CBF
:10AF60001D1F202123242527282A2B2D2E30313365
:10AF7000343637393A3C3D3F4142444547484A4BD5
:10AF80004D4E505153545657595A5B5D5E5F616246
:10AF90006365666768696A6C6D6E6F7071727373F2
:10AFA00074757677777879797A7A7B7B7C7C7C7D0F
:10AFB0007D7D7E7E7E7E7E7E7E7E7E7E7E7D7D7DB6
:10AFC0007C7C7C7B7B7A7A797978777776757473F9
:10AFD000737271706F6E6D6C6A69686766656362C3
:10AFE000615F5E5D5B5A595756545351504E4D4BFD
:10AFF0004A4847454442413F3D3C3A39373634336D
:10B0000031302E2D2B2A282725242321201F1D1CDB
:10B010001B1918171615141211100F0E0D0C0B0B0F
:10B020000A090807070605050404030302020201D2
:10B03000010100000000000000000000010101010A
:10B04000020202030304040506060708090A0A0BA4
:10B050000C0D0E0F10111214151617181A1B1C1EAA
:10B060001F212223252628292B2C2E30313334363C
:10B0700038393B3C3E4041434546484A4B4D4E5093
:10B0800052535556585A5B5D5E60616364656768EC
:10B090006A6B6C6E6F7071727475767778797A7B83
:10B0A0007C7C7D7E7F808081828283838484848592
:10B0B0008585858686868686868686878585858536
:10B0C000848484838382828180807F7E7D7C7C7B7C
:10B0D0007A7978777675747271706F6E6C6B6A6856
:10B0E0006765646361605E5D5B5A585655535250A4
:10B0F0004E4D4B4A4846454341403E3C3B3938362D
:10B10000343331302E2C2B292826252322211F1EB3
:10B110001C1B1A18171615141211100F0E0D0C0BFC
:10B120000A0A0908070606050404030302020201CD
:10B130000101010000000018191A1C1D1E1F20210A
:10B1400022232425262728292A2B2B2C2D2D2E2E71
:10B150002F2F2F3030303030303030302F2F2F2EF7
:10B160002E2D2D2C2B2B2A2928272625242322215E
:10B17000201F1E1D1C1A1918171614131211100F58
:10B180000E0D0C0B0A09080706050504030302024D
:10B1900001010100000000000000000001010102A7
:10B1A000020303040505060708090A0B0C0D0E0F20
:10B1B0001011121314161718191A1C1D1E1F202106
:10B1C00022232425262728292A2B2B2C2D2D2E2EF1
:10B1D0002F2F2F3030303030303030302F2F2F2E77
:10B1E0002E2D2D2C2B2B2A292827262524232221DE
:10B1F000201F1E1D1C1A1918171614131211100FD8
:10B200000E0D0C0B0A0908070605050403030202CC
:10B210000101010000000000000000000101010226
:10B22000020303040505060708090A0B0C0D0E0F9F
:10B230001011121314161714060102030405060751
:10B2400008090A0B0C0D0E0F101112131415161706
:10B2500018191A1B1C1D1E1F2021222324252627F6
:10B2600028292A2B2C2D2E2F3031323334353637E6
:10B2700038393A3B3C3D3E3F4041424344454647D6
:10B2800048494A004B4C4D4E4F505152535455561D
:10B290005758595A5B5C5D5E5F60616263646566C6
:10B2A0006768696A6B6C6D6E6F707172737475CA62
:10B2B000C7C4C1BEBBB7B4B1ADAAA8A39F9C9895A3
:10B2C000918E8A8784807D7A7774716F6C6A6765E6
:10B2D00063615F5D5C5A59585756555454535353E4
:10B2E000535354545556565758595B5C5D5F6062D2
:10B2F000646567696B6D6E70727476787A7B7D7F3A
:10B30000808283858687898A8B8B8C8D8D8E8E8EAD
:10B310008E8E8D8D8C8C8B8A8987868483817F7DB0
:10B320007B787673706E6B6865625E5B5854510211
:10B3300003101B2237343F41464E555A686A730644
:10B340001E10270A09140A1C240D2B130C220906AF
:10B3500094059605B4053C0300014C0514090B083F
:10B360007C090C088504000206090D080002060984
:10B370000E087B0206090F087C02060910088402E9
:10B3800006091108860210051E0300051E040002AE
:10B390001E0707069403000164052804000528031E
:10B3A0000005280400050F0264050F0300051401C1
:10B3B00058040005140300090A087C0909088E01D5
:10B3C0000609080886010609070883010609060818
:10B3D0008301060905087801060904087F011005A4
:10B3E0001E0400053C0204090308000206090408C3
:10B3F00000020609050800020609060800020609FF
:10B4000007080002060908080002060909080002E8
:10B4100006090A08000206090B08000206090C08C2
:10B42000000206090D08000206090E0800020609BE
:10B430000F080002060910080002060911080002A0
:10B440000C03000514010C091108830106091008FA
:10B45000830106090F08800106090E087E0106090E
:10B460000D088E0106090C08860106090B087A01F1
:10B4700006090A08000106090908900106090808DA
:10B480007801060907088301060906087A010609FA
:10B49000050800010609040890010609030879015E
:10B4A0003C0400050A030001320A010707001124C9
:10B4B0001FBECFEFD0E1DEBFCDBF14BE88E10FB617
:10B4C000F89480936000109260000FBE11E0A0E03D
:10B4D000B1E0E2E4FCEF02C005900D92AE31B1079D
:10B4E000D9F71CE0AEE1B1E001C01D92AA37B10767
:10B4F000E1F70E942A6A0E94CD600E9495610E9435
:10B500005C720C941F7E0C94000061606B6079602B
:10B510008F5FE05BE8EDC8950000EA95E1F7C0E2D7
:10B52000D1E0002400C000C0CABDDBBD2091800571
:10B530002770022F220F220F220F7091BF09720F66
:10B54000672F262E677026942694269410E2219E5B
:10B55000C00DD11DC0938105D0938205EE24A0E2D9
:10B56000B5E000242011ED012011F72E2011962EB8
:10B57000201166272011E39420E8201B00EDA02E67
:10B58000A3E1B6E041D000C000C03D01A3EBB9E0AB
:10B590000EEF14E0ED91FD9101930193019301935E
:10B5A000019301931A95B1F7D301AA9401F1739510
:10B5B000639500C0683021F008E00A95F1F7E2CF0A
:10B5C0006627A0960AB41BB42090810530908205AE
:10B5D00023950BF4E1010BF4692D0BF47F2D0BF493
:10B5E000EE2444247030E40409F4E001CBCF05E0FC
:10B5F0000A95F1F700000E945260E1E0E093C20971
:10B60000E2E0E0933600089528980E946D6A2F9337
:10B610001E01C090BB09D090BC0980E323E036E056
:10B6200099270D91102F0F71129516951770C3E57C
:10B63000D9E0029FC00DD11D4880F6010A81089F04
:10B64000E00DF11D139FE00DF11DC3E8D5E0C40D21
:10B65000D91FC093B309D093B409059009920590FE
:10B66000099205900992059009920590099205901A
:10B6700009920D91102F0F71129516951770C3E551
:10B68000D9E0029FC00DD11D4880F6010A81089FB4
:10B69000E00DF11D139FE00DF11DC3E8D5E0C40DD1
:10B6A000C093B509D91F289AD093B609059009927D
:10B6B00005900992059009920590099205900992CA
:10B6C000059009920D91102F0F7112951695177014
:10B6D000C3E5D9E0029FC00DD11D4880F6010A8163
:10B6E000089FE00DF11D139FE00DF11DC3E8D5E0AB
:10B6F000C40DD91FC093B709D093B809059009921A
:10B700000590099205900992059009920590099279
:10B71000059009920D91102F0F71129516951770C3
:10B72000C3E5D9E0029FC00DD11D4880F6010A8112
:10B73000089FE00DF11D139FE00DF11DC3E8D5E05A
:10B74000C40DD91FC093B909D093BA0905900992C5
:10B750000590099205900992059009920590099229
:10B7600005900992E101E091C109EA95E093C109D0
:10B770003D01DE013C2F307E1EEFC9E8D5E0409050
:10B78000C4095090C50926E0629FC001E2E1F5EBD3
:10B7900088240000000000000000880C1124E80D3F
:10B7A000F11D05901490F00186944C9120E3429F86
:10B7B000A395AF71A32B040C151C080E191E099438
:10B7C000F001C895C895C895C8950591D990D11232
:10B7D0000D2D08B94C910591D990D1120D2D08B9B4
:10B7E000429F0591D990D1120D2D08B9040C151C5A
:10B7F0000591D990D1120D2D08B9080E191E059189
:10B80000D990D1120D2D08B9A395AF710591D9909A
:10B81000D1120D2D08B9A32BF0010591D990D112A9
:10B820000D2D08B94C910591D990D1120D2D08B963
:10B83000429F0591D990D1120D2D08B9040C151C09
:10B840000591D990D1120D2D08B9080E191E059138
:10B85000D990D1120D2D08B9A395AF710591D9904A
:10B86000D1120D2D08B9A32BF0010591D990D11259
:10B870000D2D08B94C910591D990D1120D2D08B913
:10B88000429F0591D990D1120D2D08B9040C151CB9
:10B890000591D990D1120D2D08B9080E191E0591E8
:10B8A000D990D1120D2D08B9A395AF710591D990FA
:10B8B000D1120D2D08B9A32BF0010591D990D11209
:10B8C0000D2D08B94C910591D990D1120D2D08B9C3
:10B8D000429F0591D990D1120D2D08B9040C151C69
:10B8E0000591D990D1120D2D08B9080E191E059198
:10B8F000D990D1120D2D08B9A395AF710591D990AA
:10B90000D1120D2D08B9A32BF0010591D990D112B8
:10B910000D2D08B94C910591D990D1120D2D08B972
:10B92000429F0591D990D1120D2D08B9040C151C18
:10B930000591D990D1120D2D08B9080E191E059147
:10B94000D990D1120D2D08B9A395AF710591D99059
:10B95000D1120D2D08B9A32BF0010591D990D11268
:10B960000D2D08B94C910591D990D1120D2D08B922
:10B97000429F0591D990D1120D2D08B9040C151CC8
:10B980000591D990D1120D2D08B9080E191E0591F7
:10B99000D990D1120D2D08B9A395AF710591D99009
:10B9A000D1120D2D08B9A32BF0010591D990D11218
:10B9B0000D2D08B94C910591D990D1120D2D08B9D2
:10B9C000429F0591D990D1120D2D08B9040C151C78
:10B9D0000591D990D1120D2D08B9080E191E0591A7
:10B9E000D990D1120D2D08B9A395AF710591D990B9
:10B9F000D1120D2D08B9A32BF0010591D990D112C8
:10BA00000D2D08B94C910591D990D1120D2D08B981
:10BA1000429F0591D990D1120D2D08B9040C151C27
:10BA20000591D990D1120D2D08B9080E191E059156
:10BA3000D990D1120D2D08B9A395AF710591D99068
:10BA4000D1120D2D08B9A32BF0010591D990D11277
:10BA50000D2D08B94C910591D990D1120D2D08B931
:10BA6000429F0591D990D1120D2D08B9040C151CD7
:10BA70000591D990D1120D2D08B9080E191E059106
:10BA8000D990D1120D2D08B9A395AF710591D99018
:10BA9000D1120D2D08B9A32BF0010591D990D11227
:10BAA0000D2D08B94C910591D990D1120D2D08B9E1
:10BAB000429F0591D990D1120D2D08B9040C151C87
:10BAC0000591D990D1120D2D08B9080E191E0591B6
:10BAD000D990D1120D2D08B9A395AF710591D990C8
:10BAE000D1120D2D08B9A32BF0010591D990D112D7
:10BAF0000D2D08B94C910591D990D1120D2D08B991
:10BB0000429F0591D990D1120D2D08B9040C151C36
:10BB10000591D990D1120D2D08B9080E191E059165
:10BB2000D990D1120D2D08B9A395AF710591D99077
:10BB3000D1120D2D08B9A32BF0010591D990D11286
:10BB40000D2D08B94C910591D990D1120D2D08B940
:10BB5000429F0591D990D1120D2D08B9040C151CE6
:10BB60000591D990D1120D2D08B9080E191E059115
:10BB7000D990D1120D2D08B9A395AF710591D99027
:10BB8000D1120D2D08B9A32BF0010591D990D11236
:10BB90000D2D08B94C910591D990D1120D2D08B9F0
:10BBA000429F0591D990D1120D2D08B9040C151C96
:10BBB0000591D990D1120D2D08B9080E191E0591C5
:10BBC000D990D1120D2D08B9A395AF710591D990D7
:10BBD000D1120D2D08B9A32BF0010591D990D112E6
:10BBE0000D2D08B94C910591D990D1120D2D08B9A0
:10BBF000429F0591D990D1120D2D08B9040C151C46
:10BC00000591D990D1120D2D08B9080E191E059174
:10BC1000D990D1120D2D08B9A395AF710591D99086
:10BC2000D1120D2D08B9A32BF0010591D990D11295
:10BC30000D2D08B94C910591D990D1120D2D08B94F
:10BC4000429F0591D990D1120D2D08B9040C151CF5
:10BC50000591D990D1120D2D08B9080E191E059124
:10BC6000D990D1120D2D08B9A395AF710591D99036
:10BC7000D1120D2D08B9A32BF0010591D990D11245
:10BC80000D2D08B94C910591D990D1120D2D08B9FF
:10BC9000429F0591D990D1120D2D08B9040C151CA5
:10BCA0000591D990D1120D2D08B9080E191E0591D4
:10BCB000D990D1120D2D08B9A395AF710591D990E6
:10BCC000D1120D2D08B9A32BF0010591D990D112F5
:10BCD0000D2D08B94C910591D990D1120D2D08B9AF
:10BCE000429F0591D990D1120D2D08B9040C151C55
:10BCF0000591D990D1120D2D08B9080E191E059184
:10BD0000D990D1120D2D08B9A395AF710591D99095
:10BD1000D1120D2D08B9A32BF0010591D990D112A4
:10BD20000D2D08B94C910591D990D1120D2D08B95E
:10BD3000429F0591D990D1120D2D08B9040C151C04
:10BD40000591D990D1120D2D08B9080E191E059133
:10BD5000D990D1120D2D08B9A395AF710591D99045
:10BD6000D1120D2D08B9A32BF0010591D990D11254
:10BD70000D2D08B94C910591D990D1120D2D08B90E
:10BD8000429F0591D990D1120D2D08B9040C151CB4
:10BD90000591D990D1120D2D08B9080E191E0591E3
:10BDA000D990D1120D2D08B9A395AF710591D990F5
:10BDB000D1120D2D08B9A32BF0010591D990D11204
:10BDC0000D2D08B94C910591D990D1120D2D08B9BE
:10BDD000429F0591D990D1120D2D08B9040C151C64
:10BDE0000591D990D1120D2D08B9080E191E059193
:10BDF000D990D1120D2D08B9A395AF710591D990A5
:10BE0000D1120D2D08B9A32BF0010591D990D112B3
:10BE10000D2D08B94C910591D990D1120D2D08B96D
:10BE2000429F0591D990D1120D2D08B9040C151C13
:10BE30000591D990D1120D2D08B9080E191E059142
:10BE4000D990D1120D2D08B9A395AF710591D99054
:10BE5000D1120D2D08B9A32BF0010591D990D11263
:10BE60000D2D08B94C910591D990D1120D2D08B91D
:10BE7000429F0591D990D1120D2D08B9040C151CC3
:10BE80000591D990D1120D2D08B9080E191E0591F2
:10BE9000D990D1120D2D08B9A395AF710591D99004
:10BEA000D1120D2D08B9A32BF0012F910000000035
:10BEB0000027E101D30108B90895CC03CC03CC03DA
:10BEC000CC03CC03CC03CC03CC03CC03CC03CC03FA
:10BED000CC03CC03CC03CC03CC03CC03CC03CC03EA
:10BEE000CC03CC03CC03CC03CC03CC03CC03CC03DA
:10BEF000CC03CC03CC03CC03CC03CC03CC03CC03CA
:10BF0000CC03CC03CC03CC03CC03CC03CC03CC03B9
:10BF1000CC03CC03CC03CC03CC03CC03CC032898B8
:10BF20000E94816AE7E1EA95F1F7289A05D1E0E0FD
:10BF3000F6E0E8D0E0FF43D0E0FF02C00E9447698E
:10BF40000895129A0C94A45F0C94A65F129844274B
:10BF50005527662777278CE00C94AE5F0C94B05F72
:10BF60000C94B25F0C94B45F0C94B65F0C94B85F01
:10BF7000440F551F00994160660F771F019961605A
:10BF8000139A0C94C35F0C94C55F13980C94C85F0C
:10BF90000C94CA5F0C94CC5F0C94CE5F8A9541F7E9
:10BFA00040955095609570955F707F704093CB0978
:10BFB0005093CC096093CD097093CE090895EF9307
:10BFC000E091C109E43EE0F5E431D0F12F923F92D7
:10BFD0004F925F926F927F928F929F92AF92BF9299
:10BFE000CF92DF92EF92FF920F931F932F933F9385
:10BFF0004F935F936F937F938F939F93AF93BF9371
:10C00000CF93DF930E948A5ADF91CF91BF91AF9176
:10C010009F918F917F916F915F914F913F912F9160
:10C020001F910F91FF90EF90DF90CF90BF90AF9056
:10C030009F908F907F906F905F904F903F902F9048
:10C04000EF910895FF93EF93EFB7EF93E0918400A2
:10C05000EE50E13000F0E23000F0E33000F0E43088
:10C0600000F0E53000F0E63000F0E73000F0E830B6
:10C0700000F0E93000F005D0EF91EFBFEF91FF91B4
:10C0800018950F921F92EAE0F5EB0090C009000CA2
:10C090001124E00DF11D05901490F00109951F90F9
:10C0A0000F90089528980E94816AE5E1EA95F1F7DA
:10C0B000E091C109EA95E093C109289A00000000C7
:10C0C000089528980E94AA6A289A0000E1E0F6E004
:10C0D00019D02BD0089528980E94AA6AE0EB00009E
:10C0E000EA95E9F700000000289AF6E0E2E00AD0BD
:10C0F000089528980E94AA6A289A0000E3E0FCEFBD
:10C1000001D008950090C1090A9410905F0011FCBD
:10C110000F2E0092C1090090C00911FC0E2E009252
:10C12000C009E0E011FCE1E00895E3E0E09389005C
:10C13000EDE8E09388000895E7E0E0938900EBE103
:10C14000E09388000895E0E6F4E0A0E2B1E066271D
:10C150006D933197E9F7112408959927772720E205
:10C16000629F080E191EA0E2B1E0A00DB11D4C9314
:10C17000112408950895992720E2629F080E191E40
:10C18000A0E2B1E0A00DB11D5091CA09450F4C933A
:10C19000112408958093CA090895F8944427409380
:10C1A0008100409345004FEF47B944B940E84AB990
:10C1B00041E04C7F4C6041B91298139800E0009325
:10C1C000C00906E00093C1094093850040938400B4
:10C1D00043E0409389004DE84093880049E0409354
:10C1E000810042E040936F0042E44093440040E00D
:10C1F0004093470041E000004093450043E84093EE
:10C20000B00040E04093B30041E04093B10041E012
:10C2100045B97894112440E9A3E8B5E00EEF0D93F9
:10C220004A95E9F740E04093800508958093C80956
:10C230009093C90908958093C4099093C5090895FE
:10C240008093C6099093C70908958091C209089503
:10C2500011241092C2090895882329F48091CB09F2
:10C260009091CC0908958091CD099091CE090895BF
:10C2700080E891E08093610090936100089580E8E8
:10C2800090E0809361009093610008958093BB09D2
:10C290009093BC09089580938005089528E088E173
:10C2A00090E00FB6F894A895809360000FBE20939D
:10C2B00060000895882329F48091CB099091CC09DE
:10C2C00004C08091CD099091CE099093E1098093AB
:10C2D000E0094091E0095091E1094F3F510519F102
:10C2E000CA018070937080509340E9F4CA0188704D
:10C2F000987088509840B9F48091CB099091CC09FE
:10C30000892B31F08091CD099091CE09892BA1F72D
:10C3100028E088E190E00FB6F894A895809360003B
:10C320000FBE20936000CA0108950F931F9384E30A
:10C3300098E00E942E6200E710E0C8010E941B6195
:10C34000C8010E9416610E94A3608FE090E00E94E5
:10C350007D6841E06FEF80E00E946A6500EC17E0C5
:10C36000A8016CE088E00E94306883E090E00E94C1
:10C370007D6844EF57E06CE088E00E94306882E01E
:10C3800090E00E947D68A8016CE088E00E9430681F
:10C3900088E290E00E947D680E94A36084E190E0C2
:10C3A0000E947D681F910F91089590E025E130E093
:10C3B000829FF001839FF00D929FF00D1124EC5E9F
:10C3C000F34F618708956093080C089590E025E18C
:10C3D00030E0829FF001839FF00D929FF00D1124B9
:10C3E000EC5EF34F12861182089590E025E130E073
:10C3F000829FF001839FF00D929FF00D1124EC5E5F
:10C40000F34F81E0828B089590E025E130E0829F38
:10C41000F001839FF00D929FF00D1124EC5EF34F1D
:10C420006087089590E025E130E0829FF001839FCE
:10C43000F00D929FF00D1124EC5EF34F648308958C
:10C4400090E025E130E0829FF001839FF00D929F04
:10C45000F00D1124EC5EF34F6583089590936B0CFF
:10C4600080936A0C1092E209E4E1FCE021E08FEF96
:10C4700098E12083178286831386808711829583B3
:10C4800075963CE0E836F307A1F708951092150C75
:10C4900010922A0C10923F0C1092540C019690931B
:10C4A000740C8093730C9093130C8093120C9093E4
:10C4B000770C8093760C1092720C1092710C109283
:10C4C000690C1092680C10926C0C81E08093E20968
:10C4D00010926F0C10926E0C08958091120C909136
:10C4E000130C0E944662089580911D0C87FD03C0C5
:10C4F0008AEF80931D0C8091320C87FD03C08AEF78
:10C500008093320C8091470C87FD03C08AEF8093A3
:10C51000470C80915C0C87FD03C08AEF80935C0C14
:10C520001092E209089581E08093E2090895DC0108
:10C53000ED91FC911197AF014F5F5F4F11965C93A6
:10C540004E93E4912E2F30E0E7FF13C02F77307029
:10C550003695322F222737952795FA014F5F5F4F87
:10C56000E4918E2F8F77280F311DE7FDF1CF4D938A
:10C570005C93C901089508950F931F93CF93DF93A0
:10C58000182F062FEA01833049F481E091E090935F
:10C590000A0C8093090C2093080C10C0622F0E9493
:10C5A0001F69812F90E0FC01EE0FFF1FE80FF91FBC
:10C5B000EE0FFF1FEB50F44FD283C183212F30E0E9
:10C5C00085E190E0289FF001299FF00D389FF00D44
:10C5D0001124EC5EF34F81E082870783DF91CF91D6
:10C5E0001F910F9108950E941F690895EF92FF9285
:10C5F0000F931F93CF93DF93182F062FF42EE22E65
:10C60000C82FD0E085E190E0C89FF001C99FF00DF0
:10C61000D89FF00D1124EC5EF34F8285882321F022
:10C620008181882309F077C0EE2091F485E190E0C4
:10C63000C89FF001C99FF00DD89FF00D1124EC5E4A
:10C64000F34F128A8185882309F065C0178263C081
:10C65000133059F481E091E090930A0C8093090C17
:10C6600081E08093080C0F2D08C060E0812F0E94AC
:10C670001F696F2D812F0E9400690F3799F485E1A2
:10C6800090E0C89FF001C99FF00DD89FF00D1124D4
:10C69000EC5EF34F80916E0C86878FE69CE0948B66
:10C6A000838B20C0802F90E0880F991FE0916A0C47
:10C6B000F0916B0CE80FF91F259134912F5F3F4FDC
:10C6C000F901449185E190E0C89FF001C99FF00D08
:10C6D000D89FF00D1124EC5EF34F46872F5F3F4F3C
:10C6E000348B238B85E190E0C89FF001C99FF00D4A
:10C6F000D89FF00D1124EC5EF34F17861186038747
:10C7000011828FEF8087E782F282108A81E0828730
:10C71000128A118A1482DF91CF911F910F91FF909D
:10C72000EF900895CF92DF92FF920F931F93CF93D4
:10C73000DF93ECE1FCE08181282F332727FD309542
:10C740008081280F311D2F3F310519F014F02FEF94
:10C7500030E0C90137FF02C080E090E08083759629
:10C760004CE0E037F40739F78091E209882309F0BB
:10C77000CBC0E7C0E091730CF091740C9F012F5F68
:10C780003F4F3093740C2093730C44914F3F69F5E5
:10C79000A9014F5F5F4F5093740C4093730CF901E4
:10C7A00084918F3219F41092E209BCC0863009F0EE
:10C7B0009CC0FA013196CF0101969093740C80933E
:10C7C000730CE491E33529F49093770C8093760C05
:10C7D0008CC0E53409F089C08091760C9091770C7B
:10C7E0009093740C8093730C80C047FF02C04093F9
:10C7F0006C0C542F5F70842F90E0807F9070803B92
:10C800009105B9F0803C9105B9F08039910559F551
:10C81000C9010196F9014491523011F44093700C12
:10C8200001969093740C8093730C0197FC012491F2
:10C8300034C02E5F3F4F48C02F5F3F4F3093740C82
:10C840002093730C21503040F9012491852F90E002
:10C850008C9FF0018D9FF00D9C9FF00D1124EC5EDC
:10C86000F34F238742C080916C0C582F5F7090E08B
:10C87000807F9070803B910529F1803C910549F1C2
:10C880008039910591F52F5F3F4F3093740C2093C1
:10C89000730C21503040F9012491852F90E08C9F3A
:10C8A000D0018D9FB00D9C9FB00D1124AC5EB34F95
:10C8B0008C918823D1F0220F1B966C91852F0E94BA
:10C8C000F66213C02F5F3F4F3093740C2093730CAC
:10C8D0000CC0852F90E08C9FF0018D9FF00D9C9FE8
:10C8E000F00D1124EC5EF34F438783E79CE00E9438
:10C8F0009762969587959093720C8093710C109225
:10C90000690C1092680C02C0C5E1D0E06091680C1F
:10C910007091690C8091710C9091720C6817790775
:10C9200009F428CF6F5F7F4F7093690C6093680C98
:10C9300080916E0C90916F0C019690936F0C809388
:10C940006E0C05EF1BE0C5E1DCE0FF248FEFC82E85
:10C95000D12C8989882309F05EC08A899B89892B1B
:10C9600009F456C09E858D85981708F04CC050C0BC
:10C970008A852A893B898F37E9F4D9018D91BB8B50
:10C98000AA8B8F3F01F1F90161811196BB8BAA8BB4
:10C99000E82FF0E0EE0FFF1FE050FF4F0190F08115
:10C9A000E02D8F2D0995EA89FB8981918D87FB8B7D
:10C9B000EA8B28C0A9014F5F5F4F5B8B4A8BF9015F
:10C9C00084918F3F21F418821B8A1A8A21C04F5FFD
:10C9D0005F4F5B8B4A8B41505040FA016491E82FC6
:10C9E000F0E0EE0FFF1FE050FF4F0190F081E02DCF
:10C9F0008F2D0995EA89FB893196FB8BEA8B31975C
:10CA0000E491ED871E869E858D85981709F4B0CF39
:10CA10008E858F5F8E878985882319F420E030E02A
:10CA200047C08F858F3F11F08F5F8F879E8199233D
:10CA3000C9F12F812223B1F18D81882399F1899F3A
:10CA4000C001112480509F4F892F992730E0AC01FD
:10CA5000429FC001439F900D529F900D1124805022
:10CA60009F4F292F33278B818823F1F0EA81F0E053
:10CA7000E050FA42E491E058E89FC0011124805050
:10CA80009F4F892F9927F601E81BF90BE29FC00100
:10CA9000E39F900DF29F900D112480509F4F292FFE
:10CAA000332702C020E030E08A819C81890F8A838D
:10CAB000F8012083F3940A5F1F4F6596F4E0FF1698
:10CAC00009F047CFDF91CF911F910F91FF90DF9039
:10CAD000CF9008951F93CF93DF93582F90E0880F46
:10CAE000991F20916A0C30916B0C280F391FF901A6
:10CAF00085919491DC011196FC018491813011F4AF
:10CB000013E01DC080912A0C8823B1F08091350C70
:10CB1000851711F4442381F480913F0C882371F030
:10CB200080914A0C851711F4442341F49091390CFB
:10CB300080914E0C891710F411E001C012E0212FF2
:10CB400030E0FD01449185E190E0289FE001299FBC
:10CB5000D00D389FD00D1124CC5ED34F4E87119647
:10CB6000BC8BAB8B1F8680E58A836F838FEF8887B2
:10CB700019861A8A188A21E02A87198A5C872983EC
:10CB80001C82133049F481E091E090930A0C809369
:10CB9000090C2093080C08C060E5812F0E940069F1
:10CBA0006989812F0E941F69DF91CF911F9108959C
:10CBB000FF920F931F93082FF62E0E94006910E03A
:10CBC00085E190E0089FF001099FF00D189FF00D9E
:10CBD0001124EC5EF34FF2821F910F91FF900895A4
:10CBE000962F482F50E025E130E0429FF001439F0F
:10CBF000F00D529FF00D1124EC5EF34F6281691B22
:10CC000062830E9400690895482F50E025E130E0DA
:10CC1000429FF001439FF00D529FF00D1124EC5EF6
:10CC2000F34F9281690F62830E94006908951F93F8
:10CC3000CF93DF93FA01549131961491C52FD0E030
:10CC40009F012F5F3F4F70E095E0660F771F9A9529
:10CC5000E1F7680F711D40E00BC084918D939F5FD9
:10CC600031969517D0F34F5F2C0F3D1F605E7F4FBD
:10CC7000411730F4DB01A05EBE4FF90190E0F1CF27
:10CC8000DF91CF911F910895803C88F4282F30E0E8
:10CC9000220F331FC9018A5C974FFC018491295CE4
:10CCA000374FF90194918093BE099093BD09609329
:10CCB000BF090895CF92DF92EF92FF921F93CF9317
:10CCC000DF938091800587FF0AC090E08F7090709D
:10CCD000009729F00196880F880F880F01C088E01F
:10CCE000E3E1F6E01082118212821382349699E019
:10CCF000E335F907B9F7C6E5D9E061E0C82EDD24D0
:10CD000019819881812F8150873D08F055C0992362
:10CD100009F452C09A3808F04FC0712F785040E0A3
:10CD200050E0E12EFF24942F9A012E0D3F1D2C156B
:10CD30003D05E4F1283D3105CCF5272F30E0D90140
:10CD4000AA0FBB1FAA0FBB1FAD5EB94F8C918823E2
:10CD500031F49295990F907E960F9C9327C011966F
:10CD60008C911197882339F49295990F907E960FA4
:10CD700011969C931BC0F901EE0FFF1FEE0FFF1FD2
:10CD8000EB5EF94F8081882331F49295990F907E64
:10CD9000960F90830BC013968C911397882331F4D0
:10CDA0009295990F907E960F13969C934F5F5F4FCD
:10CDB0007F5F711709F0B7CF6F5F2396603209F07C
:10CDC0009FCFDF91CF911F91FF90EF90DF90CF9099
:10CDD00008958F929F92AF92BF92CF92DF92EF927F
:10CDE000FF920F931F93CF93DF93882E962E5A01B5
:10CDF0006901F02E00E010E080EEF80E0CC04F2D1F
:10CE00006E2D882D8C0F0E94BB602196CA15DB0504
:10CE1000B4F30F5F1F4F0C151D052CF4C0E0D0E0DC
:10CE2000E02EE90CF3CFDF91CF911F910F91FF908E
:10CE3000EF90DF90CF90BF90AF909F908F9008952C
:10CE400040520E94BB600895FF920F931F93CF93AF
:10CE5000DF938C01F62EEA01FE01449121964423D2
:10CE600049F0802F0F5F1F4F4F7740526F2D0E9468
:10CE7000BB60F2CFDF91CF911F910F91FF9008958A
:10CE8000FF920F931F93182F062FF42E42954F7089
:10CE90004A3010F4405F01C0495E602F812F0E942C
:10CEA000BB604F2D4F70812F8F5F4A3010F4405F71
:10CEB00001C0495E602F0E94BB601F910F91FF90DF
:10CEC0000895FF920F931F93F82E162F042F452FCE
:10CED0000E944067402F612F8F2D8E5F0E94406718
:10CEE0001F910F91FF900895EF92FF920F931F9360
:10CEF000F62E042F182FF8E0EF2EE80E07FF02C0E1
:10CF000041E101C040E16F2D812F0E94BB601F5F96
:10CF10001E1511F0000FF2CF1F910F91FF90EF90AF
:10CF20000895FF920F931F93CF93DF93F62E042F54
:10CF3000EC0110E0002311F4112339F4802F6AE092
:10CF40000E94597D905F492F01C040E06F2D8C2FCA
:10CF50000E94BB601F5F2197133031F0802F6AE081
:10CF60000E94597D082FE6CFDF91CF911F910F913D
:10CF7000FF900895CF92DF92EF92FF920F931F934D
:10CF8000CF93DF93C62E79018A01EC01DD24E114F1
:10CF9000F1040105110511F4DD2059F4C801B701B0
:10CFA0002AE030E040E050E00E94787D462F405F6C
:10CFB00001C040E06C2D8C2F0E94BB60D394219760
:10CFC00086E0D81669F0C801B7012AE030E040E0F9
:10CFD00050E00E94787DC901DA017C018D01D7CF34
:10CFE000DF91CF911F910F91FF90EF90DF90CF9045
:10CFF00008957F928F929F92AF92BF92CF92DF92CD
:10D00000EF92FF920F931F93CF93DF93782E862E8C
:10D010005A016901780100E010E00CC0A701692DF8
:10D02000872D8C0F0E94AD602196CA15DB05B4F3E5
:10D030000F5F1F4F0C151D052CF4C0E0D0E0902EA3
:10D04000980CF3CFDF91CF911F910F91FF90EF904C
:10D05000DF90CF90BF90AF909F908F907F9008957A
:10D060007F928F929F92AF92BF92CF92DF92EF9278
:10D07000FF920F931F93CF93DF93782E862EEA01B2
:10D08000FA01C590D490FA013296A590B49000E0D0
:10D0900016C0FC01EE0DFF1D3296EE0FFF1FEC0FC8
:10D0A000FD1F45915491692D812F870D0E94AD6020
:10D0B0001F5F812F90E08C159D055CF30F5F802F23
:10D0C00090E08A159B055CF48C9D70018D9DF00CA1
:10D0D0009C9DF00C112410E0902E980CEACFDF916B
:10D0E000CF911F910F91FF90EF90DF90CF90BF9065
:10D0F000AF909F908F907F9008950F931F93CF9341
:10D10000DF938C01C0E0D0E007C00E942561882336
:10D11000E1F30E9428612196C017D107B4F3DF9193
:10D12000CF911F910F9108950000000000000000B2
:10D1300000000000000000000000000000000000EF
:10D1400000000000000000000000000000000000DF
:10D1500000000000000000000000000000000000CF
:10D1600000000000000000000000000000000000BF
:10D1700000000000000000000000000000000000AF
:10D18000000000000000000000000000000000009F
:10D19000000000000000000000000000000000008F
:10D1A000000000000000000000000000000000007F
:10D1B000000000000000000000000000000000006F
:10D1C000000000000000000000000000000000005F
:10D1D000000000000000000000000000000000004F
:10D1E000000000000000000000000000000000003F
:10D1F000000000000000000000000000000000002F
:10D2000099277727833008F00895E0E0F0EE660F65
:10D21000771FE60FF71FA591B491E5EFFBE026E03D
:10D22000289FE00DF11DA183B283112408959091F0
:10D23000080C9170880F892B8093080C089599270A
:10D240007727E5EFFBE026E0289FE00DF11D6E3F1C
:10D2500031F46091080C6E7F6093080C0BC06F3F37
:10D2600031F46091080C6E6F6093080C03C076ED8A
:10D27000760F75831124089599277727E5EFFBE052
:10D2800026E0289FE00DF11D6083112408952F935F
:10D290003F934F935F936F937F938F939F93AF933E
:10D2A000BF93789411240E945A660E94A15F0E9445
:10D2B00092632F923F924F925F926F927F928F92E2
:10D2C0009F92AF92BF92CF92DF92EF92FF920F9315
:10D2D0001F93CF93DF930090F20B002019F4A6EE7A
:10D2E000B9E002C0ABEEBAE001E000260092F20B1A
:10D2F00002E00093F30B2090F60B3090F70B409078
:10D30000F90B5090FA0B6090F80B1091F50B7090A0
:10D31000FC0B8090FD0B9090FE0BA090FF0BB0904B
:10D32000000C2091FB0BC090020CD090030CE090FD
:10D33000050CF090060C0091040C3091010C5091FA
:10D34000070C6091090C70910A0C80910B0C9FEFF7
:10D35000620C431CF2014491410300240008C12DDA
:10D36000D02D970CA81CF50144914203002400081D
:10D37000C10DD01D0C0DED1CF70144914303002499
:10D380000008C10DD01D8A956AF44091080C842FC5
:10D390008695062E0694062600FA7695679576F908
:10D3A00040FF66F940E860FD4FE7450300240008B0
:10D3B000C10DD01DD595C7950024C038D0050CF0FF
:10D3C000CFE70A94C038D0050CF4C0E8CD939A9505
:10D3D00009F0BECF4091F30B4A954093F30B96E0D2
:10D3E00009F0B6CF6092F80B4092F90B9092FE0BC9
:10D3F000A092FF0B0093040CE092050C6093090CC3
:10D4000070930A0C80930B0CDF91CF911F910F91B9
:10D41000FF90EF90DF90CF90BF90AF909F908F9054
:10D420007F906F905F904F903F902F9099278091C1
:10D43000C00977276091C10911240E94BB62BF9186
:10D44000AF919F918F917F916F915F914F913F919C
:10D450002F910895A6EEB9E08AE092E000E00D93E6
:10D460000197E9F7A6EEB9E0A093F00BB093F10BAA
:10D4700000270093F20B66ED6093FA0B6093000CAB
:10D480006093060C61E06093090C60930A0C61E004
:10D490006093080C66276093F50B6093FB0B609319
:10D4A000010C6093070C6093F60B6093F70B60938D
:10D4B000F80B6093F90B6093FC0B6093FD0B60938A
:10D4C000FE0B6093FF0B6093020C6093030C609360
:10D4D000040C6093050C11240895E091F00BF09179
:10D4E000F10B019100580093B3000BE0E03FF0070F
:10D4F00006EE19E008F0F801E093F00BF093F10B61
:10D5000008950C94836A0C94856A0F931F932ABD27
:10D51000E091F00BF091F10B019100580093B300F2
:10D520000BE0E03FF00710F40000000010F0E6EE22
:10D53000F9E0E093F00BF093F10BC895C895C8950E
:10D54000C895C895C8950000000000002AB51F9135
:10D550000F9108950000E091C109E0FFD6CFE1E10D
:10D56000EA95F1F7000000000895000000000000B7
:10D5700000000000000000000000000000000000AB
:10D58000000000000000000000000000000000009B
:10D59000000000000000000000000000000000008B
:10D5A000000000000000000000000000000000007B
:10D5B000000000000000000000000000000000006B
:10D5C000000000000000000000000000000000005B
:10D5D000000000000000000000000000000000004B
:10D5E000000000000000000000000000000000003B
:10D5F000000000000000000000000000000000002B
:10D60000000306090C101316191C1F2225282B2EA7
:10D61000313336393C3F414447494C4E51535558BC
:10D620005A5C5E60626466686A6B6D6F7071737479
:10D63000757678797A7A7B7C7D7D7E7E7E7F7F7F32
:10D640007F7F7F7F7E7E7E7D7D7C7B7A7A79787618
:10D6500075747371706F6D6B6A68666462605E5C2E
:10D660005A585553514E4C494744413F3C39363343
:10D67000312E2B2825221F1C191613100C09060306
:10D6800000FDFAF7F4F0EDEAE7E4E1DEDBD8D5D20D
:10D69000CFCDCAC7C4C1BFBCB9B7B4B2AFADABA8D8
:10D6A000A6A4A2A09E9C9A9896959391908F8D8CFB
:10D6B0008B8A888786868584838382828281818122
:10D6C0008181818182828283838485868687888A1C
:10D6D0008B8C8D8F9091939596989A9C9EA0A2A4E6
:10D6E000A6A8ABADAFB2B4B7B9BCBFC1C4C7CACDB1
:10D6F000CFD2D5D8DBDEE1E4E7EAEDF0F4F7FAFDCE
:10D70000808182838485868788898A8B8C8D8E8FA1
:10D71000909192939495969798999A9B9C9D9E9F91
:10D72000A0A1A2A3A4A5A6A7A8A9AAABACADAEAF81
:10D73000B0B1B2B3B4B5B6B7B8B9BABBBCBDBEBF71
:10D74000C0C1C2C3C4C5C6C7C8C9CACBCCCDCECF61
:10D75000D0D1D2D3D4D5D6D7D8D9DADBDCDDDEDF51
:10D76000E0E1E2E3E4E5E6E7E8E9EAEBECEDEEEF41
:10D77000F0F1F2F3F4F5F6F7F8F9FAFBFCFDFEFF31
:10D78000000102030405060708090A0B0C0D0E0F21
:10D79000101112131415161718191A1B1C1D1E1F11
:10D7A000202122232425262728292A2B2C2D2E2F01
:10D7B000303132333435363738393A3B3C3D3E3FF1
:10D7C000404142434445464748494A4B4C4D4E4FE1
:10D7D000505152535455565758595A5B5C5D5E5FD1
:10D7E000606162636465666768696A6B6C6D6E6FC1
:10D7F000707172737475767778797A7B7C7D7E7FB1
:10D8000000020406080A0C0E10121416181A1C1E28
:10D8100020222426282A2C2E30323436383A3C3E18
:10D8200040424446484A4C4E50525456585A5C5E08
:10D8300060626466686A6C6E70727476787A7C7EF8
:10D840007F7D7B79777573716F6D6B6967656361D8
:10D850005F5D5B59575553514F4D4B4947454341C8
:10D860003F3D3B39373533312F2D2B2927252321B8
:10D870001F1D1B19171513110F0D0B0907050301A8
:10D88000FFFDFBF9F7F5F3F1EFEDEBE9E7E5E3E198
:10D89000DFDDDBD9D7D5D3D1CFCDCBC9C7C5C3C188
:10D8A000BFBDBBB9B7B5B3B1AFADABA9A7A5A3A178
:10D8B0009F9D9B99979593918F8D8B898785838168
:10D8C00080828486888A8C8E90929496989A9C9E68
:10D8D000A0A2A4A6A8AAACAEB0B2B4B6B8BABCBE58
:10D8E000C0C2C4C6C8CACCCED0D2D4D6D8DADCDE48
:10D8F000E0E2E4E6E8EAECEEF0F2F4F6F8FAFCFE38
:10D900007F7F7F7F7F7F7F7F7F7F7F7F7F7F7F7F27
:10D910007F7F7F7F7F7F7F7F7F7F7F7F7F7F7F7F17
:10D920007F7F7F7F7F7F7F7F7F7F7F7F7F7F7F7F07
:10D930007F7F7F7F7F7F7F7F7F7F7F7F7F7F7F7FF7
:10DC00000309131E28313A40464C5054585B5E615C
:10DC1000636567696B6C6E6F70717273747576771C
:10DC2000777879797A7A7B7B7C7C7C7D7D7D7E7E42
:10DC30007E7E7F7F7F7F7F7F7F7F7F7F7F7F7F7FF6
:10DC40007F7F7F7F7F7F7F7F7F7F7F7F7F7E7E7EE7
:10DC50007E7D7D7D7C7C7C7B7B7A7A797978777719
:10DC6000767574737271706F6E6C6B6967656361E2
:10DC70005E5B5854504C46403A31281E130903004D
:10DC8000C6CCD5DBDFE3E5E7E9EAEBECEDEEEFEF61
:10DC9000F0F0F0F1F1F1F1F2F2F2F2F2F2F2F2F36D
:10DCA000F3F3F3F3F3F3F3F3F3F3F3F3F3F3F3F344
:10DCB000F3F3F3F3F3F3F3F3F3F3F3F3F3F3F3F334
:10DCC000F3F3F3F3F3F3F3F3F3F3F3F3F3F3F3F324
:10DCD000F3F3F3F3F3F3F3F3F3F3F3F3F3F3F3F314
:10DCE000F2F2F2F2F2F2F2F2F1F1F1F1F0F0F0EF21
:10DCF000EFEEEDECEBEAE9E7E5E3DFDBD5CCC600E0
:10DD000000283D42302D2C2B2C2D2E2F3032333538
:10DD100037393B3D3F414345484A4C4E5053555798
:10DD2000595B5D5F61636567696B6C6E707173747D
:10DD3000757778797A7B7C7D7D7E7E7F7F7F7F7F24
:10DD40007F7F7F7F7F7F7E7E7D7D7C7B7A7978770A
:10DD500075747371706E6C6B69676563615F5D5B31
:10DD600059575553504E4C4A484543413F3D3B3926
:10DD700037353332302F2E2D2C2B2C2D30423D2891
:10DD800000E9E5FED4D7D7D7D6D4D2D0CECCCAC8F6
:10DD9000C6C3C1BFBDBAB8B6B4B1AFADABA9A7A534
:10DDA000A3A19F9E9C9A999795949391908F8D8C07
:10DDB0008B8A898888878685858484848383838306
:10DDC0008383838383848484858586878888898AFE
:10DDD0008B8C8D8F909193949597999A9C9E9FA1EF
:10DDE000A3A5A7A9ABADAFB1B4B6B8BABDBFC1C307
:10DDF000C6C8CACCCED0D2D4D6D7D7D7D4FEE5E9C0
:10DE0000F9F8F9F5EBE1DDDEE0E2E4E5E6E5E4E290
:10DE1000DED9D2CAC1B7ACA299918A8683818080AB
:10DE20008182838586888A8C8D8F90929395969730
:10DE300098999A9B9B9C9D9D9D9E9E9E9F9F9F9F18
:10DE40009F9F9F9E9E9E9D9D9D9C9B9B9A99989710
:10DE500096959392908F8D8C8A8886858382818017
:10DE6000808183868A9199A2ACB7C1CAD2D9DEE2F9
:10DE7000E4E5E6E5E4E2E0DEDDE1EBF5F9F8F90002
:10DE80000708070B151F2322201E1C1B1A1B1C1E14
:10DE900022272E363F49545E676F767A7E7F7F7FDA
:10DEA0007F7E7D7B7A7876747371706E6D6B6A6934
:10DEB000686766656564646363626262616161612B
:10DEC0006161616262626363636465656667686914
:10DED0006A6B6D6E7071737476787A7B7D7E7F7FEE
:10DEE0007F7F7E7A766F675E54493F362E27221EEB
:10DEF0001C1B1A1B1C1E2022231F150B07080700C2
:10DF00001F313D444E5354565A5F64696E7476799E
:10DF10007C7F7F7F7F7F7F7F7F7F7F7F7F7F7F7F14
:10DF20007F7F7F7F7F7F7F7F7F7F7F7F7F7F7F7F01
:10DF30007F7F7F7F7F7F7F7F7F7F7F7F7F7F7F7FF1
:10DF40007F7F7F7F7F7F7F7F7F7F7F7F7F7F7F7FE1
:10DF50007F7F7F7F7F7F7F7F7F7F7F7F7F7F7F7FD1
:10DF60007F7F7F7F7F7F7F7F7F7F7F7F7F7F7F7FC1
:10DF70007F7F7F7F7F7F7F7F7F7F7F7C7871684C13
:10DF80002C1C120C0A0B0A05FDF3E9DFD4CAC0B73A
:10DF9000AEA69E97918B86858280808080808080CF
:10DFA0008080808080808080808080808080808071
:10DFB0008080808080808080808080808080808061
:10DFC0008080808080808080808080808080808051
:10DFD0008080808080808080808080808080808041
:10DFE0008080808080808080808080808080808031
:10DFF000808080808087919DACC4CBD4DDF2FAFA1A
:10E0000022002400260028002B002D0030003300C1
:10E01000360039003D004000440048004C005100EB
:10E0200056005B00600066006C00730079008100A0
:10E03000880090009900A200AC00B600C100CC009E
:10E04000D800E500F3000101100121013201440173
:10E0500057016C0181019801B001CA01E50102027A
:10E060002102410264028802AE02D7020303300398
:10E0700061039403CB03050442048304C704100521
:10E080005D05AF0505066106C20629079607090862
:10E09000830805098E09200ABA0A5D0B0A0CC10C17
:10E0A000840D510E2B0F121007110A121D1340146C
:10E0B0007415BA1614188319071BA31C571E2420A5
:10E0C0000E22142439267F28E82A752D293006339C
:10E0D0000F364539AD3C49401B442848734CFE502F
:10E0E000CF55EA5A51600C661D6C8B725A7992803A
:10E0F00037885090E598FDA19FABD3B5A3C0000031
:10E100002F923F924F925F926F927F928F929F9247
:10E11000AF92BF92CF92DF92EF92FF920F931F9335
:10E12000DF93CF9300D000D0CDB7DEB7662E742E2C
:10E1300081118AE0E82FF0E006E0202E260C862DE3
:10E14000845F898312E1412E460CB8E03B2E370CE8
:10E15000A0E15A2E570C972D985E9A83222309F03E
:10E16000A8C0CF0102964C01880C991C880E991EFC
:10E17000A3E5B9E08A0E9B1E81E1D40112968C932F
:10E18000CF0103965C01AA0CBB1CA80EB91E83E547
:10E1900099E0A80EB91E82E1D50112968C93CF01A9
:10E1A00004966C01CC0CDD1CC80ED91E83E599E0E9
:10E1B000C80ED91E83E1D60112968C93CF01059625
:10E1C0007C01EE0CFF1CE80EF91E83E599E0E80ED9
:10E1D000F91E84E1D70112968C93CF0106968C012B
:10E1E000000F111F080F191F0D5A164F88E1D80193
:10E1F00012968C93CF010796BC01660F771F680FAC
:10E20000791F6D5A764F89E1DB0112968C93CF010D
:10E210000896AC01440F551F480F591F4D5A564FD1
:10E220008AE1DA0112968C93CF0109969C01220FA4
:10E23000331F280F391F2D5A364F8BE1D901129603
:10E240008C93CF010A96DC01AA0FBB1FA80FB91F40
:10E25000AD5AB64F86E2782E12967C921297CF0175
:10E260000B96FC01EE0FFF1FE80FF91FED5AF64F5A
:10E27000FC83EB837282F4016082F5012082898144
:10E28000F6018083F7014082F8016082FB01208261
:10E29000FA018083F90140826C92EB81FC8140821B
:10E2A000F4013182F5013182F6013182F7013182C8
:10E2B000A9C0CF0102964C01880C991C880E991EAA
:10E2C00083E599E0880E991E84E2D40112968C931E
:10E2D000CF0103965C01AA0CBB1CA80EB91E83E5F6
:10E2E00099E0A80EB91E86E1D50112968C93CF0154
:10E2F00004966C01CC0CDD1CC80ED91E83E599E098
:10E30000C80ED91E87E1D60112968C93CF010596CF
:10E310007C01EE0CFF1CE80EF91E83E599E0E80E87
:10E32000F91E85E2D70112968C93CF0106968C01D7
:10E33000000F111F080F191F0D5A164F8CE1D8013D
:10E3400012968C93CF010796BC01660F771F680F5A
:10E35000791F6D5A764F8DE1DB0112968C93CF01B8
:10E360000896AC01440F551F480F591F4D5A564F80
:10E370008EE1DA0112968C93CF0109969C01220F4F
:10E38000331F280F391F2D5A364F8FE1D9011296AE
:10E390008C93CF010A96DC01AA0FBB1FA80FB91FEF
:10E3A000AD5AB64F80E212968C931297CF010B961E
:10E3B000FC01EE0FFF1FE80FF91FED5AF64FFC832B
:10E3C000EB8383E28283F4016082F50120828981FC
:10E3D000F6018083F7014082F8016082FB01208210
:10E3E000FA018083F90140826C92EB81FC814082CA
:10E3F000872D805EF4018183F5013182F60131823F
:10E40000F7018183F8015182FB015182FA015182A7
:10E41000F9015182FA811196FC93EA81AB81BC81AA
:10E420001196EC930F900F900F900F90CF91DF917A
:10E430001F910F91FF90EF90DF90CF90BF90AF9022
:10E440009F908F907F906F905F904F903F902F9014
:10E450000895DB01FA0125E0AA0FBB1F2A95E1F719
:10E46000A80FB91FA05EBE4F8491882349F0803267
:10E4700011F480E002C08F7780548D933196F4CFF1
:10E480000895CF93DF9380E00E945A61EC0191FFE1
:10E4900005C080E00E945A61892BD9F760910E0C6B
:10E4A00080910D0C0E944466D093110CC093100C07
:10E4B00080E0DF91CF9108952F923F924F925F922B
:10E4C0006F927F928F929F92AF92BF92CF92DF9284
:10E4D000EF92FF920F931F93DF93CF93CDB7DEB7E9
:10E4E000ED970FB6F894DEBF0FBECDBF8CEF81B9AC
:10E4F00089E994E30E942E6286EB99E00E944662CD
:10E5000053E5452E59E0552EF2018AEF8083818331
:10E510001282339629E0E33BF207C1F781E090E0F5
:10E520000E947D6881E594E70E94466187ED94E34F
:10E530000E941B618EEF0E94CA600E94A36010922D
:10E54000180180E80E944B61CE0101969BAF8AAF13
:10E55000FC0180E08193885F8035E1F7EAEBF2EB24
:10E56000E491E055E0930E0C6E2F80910D0C0E940B
:10E57000446681E995E80E941B6147E352EB65E040
:10E5800081E00E94176686E78093730287E7809395
:10E590007402109255090E94497D0E94497DE3E56D
:10E5A000F9E085EF8083339699E0E33BF907D1F7F3
:10E5B00010920E0C0E94497D0E94497D8DE280934D
:10E5C000560981E78093570988E290E00E947D68B0
:10E5D0009BE29093560981E38093590990935C09DB
:10E5E00080935F098AE08093570980935A0982E1FA
:10E5F00080935D09809360098EE18093620984E6CF
:10E600008093630984E38093640925E030E0A2E30A
:10E6100019C0FB018491845FF8018083FA01849121
:10E62000885DF8018183A2839F5F6F5F7F4F0D5FDD
:10E630001F4F4F5F5F4F993061F72C5F3F4F253180
:10E64000310589F0C9010597BC01615D7C448901F0
:10E65000000F111F020F131F0D5A164FAC01415C22
:10E660005C4495E0D6CF00E010E08BE0C82ED12CC2
:10E67000CC0EDD1EBBE1EB2EF12CEC0EFD1E0E943C
:10E68000497DF601E00FF11F69E170E00E94657DB0
:10E690008083F701E00FF11F10820F5F1F4F0031E1
:10E6A000110569F7ABE0FA2E05E710E081E090E094
:10E6B0000E947D68EF2DF0E0E155FD44E491E055C6
:10E6C000E0930E0C6E2F80910D0C0E944466F39423
:10E6D0000150104059F780E48093A3098093A60964
:10E6E0008093A9098093AC091092790C1092780C50
:10E6F0001DAAF6E9CF2EE6E9DE2E662477248824CB
:10E700009924F1E0FAABF9AB1CA6AA24BB247BE167
:10E71000272E312C2C0E3D1E9E01255D3F4F3FAB19
:10E720002EAB81E090E00E947D688091780C909102
:10E73000790C01969093790C8093780C3AA931303A
:10E7400089F4F301ED56FC444491C30101969C0108
:10E750002D563C44F90124913C010894611C711C24
:10E76000042F122FF9A9F13089F4F401E15BFC4484
:10E770004491C40101969C01215B3C44F901249120
:10E780004C010894811C911CE42EF22EFCA5F13062
:10E7900009F0DFC00894A11CB11C2CEDA216B10435
:10E7A00009F0D7C081E090E00E947D6806E519E09D
:10E7B00088ECF80180830D5F1F4FF9E0033B1F07D2
:10E7C000C1F781E090E00E947D68D801D897E7E525
:10E7D000F9E080E38083828B8C9352968C935297DE
:10E7E0003396885F13968036A9F787EB80939F094D
:10E7F0008093A2098093A5098093A8096DEBE62E6A
:10E8000061E0F62E5DEFA52E51E0B52E4DE3C42E4E
:10E8100042E0D42E10E037E5732E28E5822E99E5EC
:10E82000992E0AE583E090E00E947D68812F845F45
:10E83000809356098093590980935C0980935F09FE
:10E84000809362098093650980939E09912F9A5F56
:10E850009093680990936B0990936E099093710956
:10E8600090937409909377099093A10910937A0972
:10E8700010937D09109380091093830910938609E2
:10E88000109389091093A409825180938C09809375
:10E890008F098093920980939509809398098093BA
:10E8A0009B098093A7097092580970925B09709236
:10E8B0005E097092610970926409709267097092A2
:10E8C000A00980926A0980926D09809270098092F5
:10E8D000730980927609809279098092A3099092B7
:10E8E0007C0990927F09909282099092850990927A
:10E8F000880990928B099092A60900938E09009343
:10E900009109009394090093970900939A09009341
:10E910009D090093A909F701108210A2F501108248
:10E9200010A2F601108210A220E232E0E20EF31EE5
:10E93000F701108221EE3DEFE20EF31E0894A11CB8
:10E94000B11C0894C11CD11C9A3B09F4A5C1192F14
:10E9500069CF053031F1063060F40230E1F0033068
:10E9600018F4013089F515C0033079F0043061F5F1
:10E9700014C00830D9F0093018F4063029F514C055
:10E980000930E9F00A3001F51EC031E03AAB18AAAF
:10E990001FC0CA9406C0C39404C081E08AAB88AB90
:10E9A00017C0115099F010C0C12E10C02EA5E22F33
:10E9B000F0E0E052FC4F108331E03AAB09C01EA7F3
:10E9C00081E08AAB05C01CA71AAA02C091E09AABED
:10E9D000E4E0EE16F9F0EE1548F0F2E0EF16C1F0C3
:10E9E000FE1580F021E0E21669F510C036E0E3166E
:10E9F000C1F0E31698F088E0E816B9F099E0E9165E
:10EA000009F51CC0E1E0E9AB1FA620C0DA9406C0FE
:10EA1000D39404C0F1E0F9ABFFA718C0FA94A1F0B9
:10EA200011C0D12E21E029AB11C03DA5E32FF0E0AC
:10EA3000E052FC4FF08281E089AB08C0FDA691E076
:10EA400099AB04C019AA02C0E1E0E9ABFDA9FF5FE0
:10EA5000FDABC09256098C2D8A5F80935909C092F4
:10EA60005C0980935F09C092A7098093AA09D0929C
:10EA700095098D2D8A5F80939809D0929B09809388
:10EA80009E09D092A1098093A4098F2F90E0FC01E8
:10EA9000E95CFE44E491E695E6952E2F28552093F7
:10EAA000570920935A09285F20935D092093600934
:10EAB000E854E093A809E093AB09805C9F4F907005
:10EAC000895C9E44FC01849186958695282F285563
:10EAD0002093960920939909285F20939C092093FD
:10EAE0009F0988548093A2098093A5098091780C8E
:10EAF0009091790C8F709070029709F5DE011B964A
:10EB000044E659E091018C9118161CF481508C93C5
:10EB10000EC0FA0180818F5F8083883340F088E3E4
:10EB20008083F9018081882311F481E0808311962C
:10EB30004D5F5F4F2F5F3F4FA215B30521F7C10116
:10EB40004FE353EBA3E6B9E0FC012081121634F544
:10EB5000322F3F5F3083FA012491E32FFF27E7FD37
:10EB6000F095E95CF045E491E20FE85DEC93E23862
:10EB7000A8F0FCA5FF2349F4285D2C9323E311960C
:10EB80002C931197FC01108209C0FAEFFC9323E348
:10EB900011962C9311972EEFFC01208301964F5F65
:10EBA0005F4F1396EEA9FFA98E179F0769F6809114
:10EBB000780C80FD1BC0FFA5F13059F429E32093A8
:10EBC00097093AE330939A098EE380939D098FE386
:10EBD0000AC08BE2809397099CE290939A0980E3A4
:10EBE00080939D0981E38093A0091AC0EFA5E130CD
:10EBF00059F4F9E3F09397092AE320939A098CE3F7
:10EC000080939D098DE3EFCF3BE2309397098CE22F
:10EC100080939A099EE290939D09EFE2E093A00908
:10EC20008091780C80FD1BC0F8A9F13059F429E3DC
:10EC3000209358093AE330935B098EE380935E0991
:10EC40008FE30AC08BE2809358099CE290935B09A2
:10EC500080E380935E0981E3809361091AC0E8A98B
:10EC6000E13059F4F9E3F09358092AE320935B0962
:10EC70008CE380935E098DE3EFCF3BE2309358093C
:10EC80008CE280935B099EE290935E09EFE2E09351
:10EC900061090E94417245CDE3E5F9E08AEF808386
:10ECA00081831282339629E0E33BF207C1F781E0CA
:10ECB00090E00E947D6881E594E70E94466187EDBF
:10ECC00094E30E941B618EEF0E94CA600E94A360C1
:10ECD0001092180180E80E944B61FE01319680E09D
:10ECE0008193885F8035E1F747EA54E665E080E08C
:10ECF0000E9417668CEF809394038DEF80939503A9
:10ED000081E090E00E947D68109255090E94497D43
:10ED10008C010E94497D7C01E3E5F9E085EF808369
:10ED2000339639E0E33BF307D1F72AE43BEADF010E
:10ED30005C97F90184918C932F5F3F4F1396FBEA08
:10ED400023353F07B1F7E5E9F9E0DE01119698E2D6
:10ED500090838D9181833396995F9E36C9F7C80160
:10ED600065E070E00E94657D782EC70165E070E087
:10ED70000E94657D882E10920E0C0E94497D0E9493
:10ED8000497D8DE28093560981E78093570910925F
:10ED9000790C1092780CBB241BA6992484E9A82E28
:10EDA0001CAA04E91BAACC242224239433243394E0
:10EDB000DD2410E06624EE24FF249E01255F3F4FF2
:10EDC00039AF28AFCE010A969DAF8CAF81E090E0BD
:10EDD0000E947D688091780C9091790C01969093B7
:10EDE000790C8093780C9BA59F5F9BA7892F8F73CD
:10EDF0008A3019F40894E11CF11CE2E2EE16F104E9
:10EE00000CF490C0F8E2EF16F1040CF487C081E036
:10EE100090E00E947D688AEF80935609E6E5F9E06C
:10EE200028EC2083339639E0E33BF307C9F781E010
:10EE300090E00E947D6881E890E80E944661E6E5E6
:10EE4000F9E080E3818398E09083885F3396883A85
:10EE5000C9F7E3E8F9E080E390E881839083885F75
:10EE60003396883AD1F705EBE02EF12C04E81AE846
:10EE7000B12EB5E5CB2EB1E0DB2E4BC080833396AF
:10EE8000A3E88A2EA9E09A2E8E169F06B9F7F40100
:10EE90000083339629E0E03BF207D1F710E00EC083
:10EEA000108385A7339639E0E538F307C9F781E089
:10EEB00090E00E947D681F5F153029F0E8E5F9E0D9
:10EEC000812F8B5FEDCFF601EE19FF09E05EFE4F5B
:10EED00085ED93E08E199F09805E9E4F1082B0965B
:10EEE000E817F907D9F7F701E05EFE4FC701805632
:10EEF0009C4F1082B096E817F907D9F781E090E0AF
:10EF00000E947D680894E108F1080650023409F473
:10EF1000A1C18B2D801BE6E5F9E0B0CF7724739477
:10EF2000882483948CE3981689F5662079F5D39428
:10EF300092E09D15C0F425E63BEAA5E9B9E0E8ECCE
:10EF4000EC93F901849112968C93129713962F5F8C
:10EF50003F4FF9E0A03BBF0791F79924CC24DD2473
:10EF60006624639413C089E0D89E90011124265B27
:10EF70003445A7E9B9E0F90184918C932F5F3F4FA5
:10EF80001396F9E0A23BBF07B1F799242BA52F3FB9
:10EF900009F4C394FE01319680818F5F819388AD1F
:10EFA00099ADE817F907C1F78091780C80FF5DC033
:10EFB0009E012F5F3F4FA5E9B9E079E26AE257E28F
:10EFC00048E2F901808190E0FC01E95CFE44E491B3
:10EFD000E2561196EC931197662009F43DC0F1E0DA
:10EFE000FC1574F1895C9045FC0184918A5F8C93D7
:10EFF0008091780C82FF30C0822FFAAD8F1B883051
:10F0000059F112968C911297883271F0893218F466
:10F01000873211F505C0893259F08A32E9F40CC003
:10F0200012964C93129718C012967C93129714C0A4
:10F0300012966C93129710C012965C9312970CC0A4
:10F04000895C9F44FC0184918A5F8C93863820F010
:10F05000F6E21296FC9312972F5F3F4F13968CADFA
:10F060009DAD2817390709F0ACCF92E09C154CF5FF
:10F07000EAE4FBEAA7E9B9E084918C933196139610
:10F080002BEAE335F207C1F7A5E9B9E09E012F5F4E
:10F090003F4F88E28C93F90191919F01E92FF0E0B5
:10F0A000E95CFE44E491E2561196EC9311971396B5
:10F0B000895F873679F780EF8093B009CC24DD240F
:10F0C00066248091780C9091790C059769F41092E0
:10F0D000790C1092780C0E94497D63E070E00E94E8
:10F0E000657D825F80935809B394F3E0BF1609F001
:10F0F00042C093942CA92F5F2CAB3BA93F5F3BAB45
:10F10000422F4170242F485D6A2D81E00E9480705B
:10F110004BA94170242F4D58602F80E00E948070D1
:10F12000672D6A0D080D643628F089E1E816F104B0
:10F130000CF464E6043628F099E1E916F1040CF4C5
:10F1400004E66C3828F0EAE1EE16F1040CF06CE805
:10F150000C3828F0FAE1EF16F1040CF00CE8A62EBA
:10F1600025E0621710F4E5E0AE2E063018F4BB245B
:10F1700005E001C0BB242A943A9412149CF00E942A
:10F18000497D6AE070E00E94657D7AE1272E280EB5
:10F190000E94497D65E070E00E94657DFC01EE5CA7
:10F1A000F245749013149CF00E94497D68E070E071
:10F1B0000E94657D6EE1362E380E0E94497D65E025
:10F1C00070E00E94657DFC01EE5CF24584900E9437
:10F1D000417280E00E945A619C0184FF0CC01F5F55
:10F1E000103208F01FE112541093EA031E5B7724DB
:10F1F00073948824839426FF0CC0812F90E0FC0137
:10F20000EE0FFF1FE80FF91FED5AF64F81818F5F58
:10F21000818327FF0CC0812F90E0FC01EE0FFF1FC0
:10F22000E80FF91FED5AF64F81818150818325FF48
:10F230000BC0115009F411E012541093EA031E5B45
:10F2400077247A9488248A9423FD1F5F33FFBECDF0
:10F250001150BCCD0E94A36089E497EA0E944661E8
:10F2600081E291EA0E941B6180E20E94CA608AEFFB
:10F27000F20180838183128223E030E0420E531E2C
:10F2800033EB431639E0530699F70E94A3601092BE
:10F29000180180E80E944B6110920E0C60E0809192
:10F2A0000D0C0E94446636E0309356099CED909315
:10F2B000570981E0809358092CE0209359099093D5
:10F2C0005A0982E080935B0942E140935C09909384
:10F2D0005D0983E080935E0930935F0994EE90931B
:10F2E000600984E080936109209362099093630927
:10F2F00085E0809364094093650990936609309393
:10F300006709309368099CEE9093690987E08093C0
:10F310006A0920936B0990936C0988E080936D09CA
:10F3200040936E0990936F0989E080937009309340
:10F33000710994EF909372098AE080937309209386
:10F340007409909375098BE080937609409377094F
:10F35000909378092093790930937A099CEF9093E0
:10F360007B098DE080937C0920937D0990937E0931
:10F370008EE080937F0986EB8093800990938109CA
:10F380008FE0809382091092790C1092780C00E043
:10F3900010E0EE24FF2482E090E00E947D688091DE
:10F3A000780C9091790C01969093790C8093780C5D
:10F3B0000894E11CF11C88E7E816F10454F4E7E531
:10F3C000F9E0808181508083339699E0E438F90731
:10F3D000C1F7C701855893408638910548F4E6E5A2
:10F3E000F9E080818F5F808333968E169F06C9F780
:10F3F000EBE1EE16E4E0FE0614F00C9400008091C0
:10F40000700C8F3F61F08FEF8093700C0E94497DEC
:10F4100065E070E00E94657D805F80936D090E94C9
:10F42000417280910E0C8F5F80930E0C0F5F08303D
:10F4300009F0DAC21F5F869586958695875E8F7183
:10F440008F5F90E035E0880F991F3A95E1F7EEE67F
:10F45000FBEADC01A05EBE4F2491222349F020325A
:10F4600011F420E002C02F7720542D933196F4CF71
:10F47000123819F400E010E0B7C21D3209F484C15B
:10F480001E32B8F5173109F4EFC01831C8F41B303B
:10F4900009F4A2C01C3050F4153009F479C01730BB
:10F4A00009F488C0113009F09EC260C0113109F41E
:10F4B000B7C0133109F4C6C01D3009F094C29EC014
:10F4C000133209F419C1143250F41D3109F4F0C09B
:10F4D000113209F4FFC0193109F085C2D7C01732C3
:10F4E00009F42EC11B3209F43DC1153209F07BC26B
:10F4F00015C11D3309F4D8C11E33C8F4153309F4FE
:10F500008BC1163350F4113309F462C1133309F47B
:10F5100071C11F3209F067C249C1193309F4A0C192
:10F520001B3309F4AFC1173309F05DC287C115342D
:10F5300009F402C2163450F4113409F4D9C1133459
:10F5400009F4E8C11F3309F04EC2C0C1193409F4EF
:10F5500017C21A3420F4173409F045C2FFC11B3416
:10F5600009F41FC2143609F03EC22CC2E6E8FBEAD9
:10F57000DC01AD5DBE4F8491882309F434C2803232
:10F5800011F480E002C08F7780548D933196F3CFD1
:10F59000EAE9FBEADC01AD5DBE4F8491882309F402
:10F5A00022C2803211F480E002C08F7780548D93A4
:10F5B0003196F3CFE1EBFBEADC01AB5DBE4F84910A
:10F5C000882309F410C2803211F480E002C08F77E2
:10F5D00080548D933196F3CFE7EAFBEADC01AD5D11
:10F5E000BE4F8491882309F4FEC1803211F480E07B
:10F5F00002C08F7780548D933196F3CFE1EBFBEA15
:10F60000DC01AB5DBE4F8491882309F4ECC18032EC
:10F6100011F480E002C08F7780548D933196F3CF40
:10F62000EEEBFBEADC01AD5DBE4F8491882309F46B
:10F63000DAC1803211F480E002C08F7780548D935C
:10F640003196F3CFEDECFBEADC01AB5DBE4F84916C
:10F65000882309F4C8C1803211F480E002C08F779A
:10F6600080548D933196F3CFE9EDFBEADC01AD5D7B
:10F67000BE4F8491882309F4B6C1803211F480E032
:10F6800002C08F7780548D933196F3CFEBEEFBEA77
:10F69000DC01AB5DBE4F8491882309F4A4C18032A4
:10F6A00011F480E002C08F7780548D933196F3CFB0
:10F6B000E0E2FDEADC01AD5DBE4F8491882309F4F0
:10F6C00092C1803211F480E002C08F7780548D9314
:10F6D0003196F3CFE8EFFBEADC01AD5DBE4F8491DC
:10F6E000882309F480C1803211F480E002C08F7752
:10F6F00080548D933196F3CFE3E0FCEADC01AD5DFD
:10F70000BE4F8491882309F46EC1803211F480E0E9
:10F7100002C08F7780548D933196F3CFE4E1FCEAF9
:10F72000DC01AD5DBE4F8491882309F45CC1803259
:10F7300011F480E002C08F7780548D933196F3CF1F
:10F74000E7E2FCEADC01AD5DBE4F8491882309F459
:10F750004AC1803211F480E002C08F7780548D93CB
:10F760003196F3CFEBE3FCEADC01AD5DBE4F849153
:10F77000882309F438C1803211F480E002C08F7709
:10F7800080548D933196F3CFE7E4FCEADC01AD5D64
:10F79000BE4F8491882309F426C1803211F480E0A1
:10F7A00002C08F7780548D933196F3CFE0E2FDEA6B
:10F7B000DC01AD5DBE4F8491882309F414C1803211
:10F7C00011F480E002C08F7780548D933196F3CF8F
:10F7D000EAE5FCEADC01AD5DBE4F8491882309F4C3
:10F7E00002C1803211F480E002C08F7780548D9383
:10F7F0003196F3CFEEE6FCEADC01AD5DBE4F8491BD
:10F80000882309F4F0C0803211F480E002C08F77C1
:10F8100080548D933196F3CFE0E2FDEADC01AD5DDB
:10F82000BE4F8491882309F4DEC0803211F480E059
:10F8300002C08F7780548D933196F3CFE1E8FCEAD4
:10F84000DC01AD5DBE4F8491882309F4CCC08032C9
:10F8500011F480E002C08F7780548D933196F3CFFE
:10F86000E4E9FCEADC01AD5DBE4F8491882309F434
:10F87000BAC0803211F480E002C08F7780548D933B
:10F880003196F3CFE0E2FDEADC01AD5DBE4F84913D
:10F89000882309F4A8C0803211F480E002C08F7779
:10F8A00080548D933196F3CFE7EAFCEADC01AD5D3D
:10F8B000BE4F8491882309F496C0803211F480E011
:10F8C00002C08F7780548D933196F3CFE8EBFCEA3A
:10F8D000DC01AD5DBE4F8491882309F484C0803281
:10F8E00011F480E002C08F7780548D933196F3CF6E
:10F8F000ECECFCEADC01AD5DBE4F8491882309F499
:10F9000072C0803211F480E002C08F7780548D93F2
:10F910003196F3CFE0E2FDEADC01AD5DBE4F8491AC
:10F92000882309F460C0803211F480E002C08F7730
:10F9300080548D933196F3CFEEEDFCEADC01AD5DA2
:10F94000BE4F8491882309F44EC0803211F480E0C8
:10F9500002C08F7780548D933196F3CFE0E2FDEAB9
:10F96000DC01AD5DBE4F8491882309F43CC0803238
:10F9700011F480E002C08F7780548D933196F3CFDD
:10F98000E1EFFCEADC01AD5DBE4F8491882359F1C3
:10F99000803211F480E002C08F7780548D933196CD
:10F9A000F4CFE1E0FDEADC01AD5DBE4F8491882338
:10F9B000D1F0803211F480E002C08F7780548D93B3
:10F9C0003196F4CFE1E1FDEADC01AD5DBE4F8491FB
:10F9D000882349F0803211F480E002C08F77805490
:10F9E0008D933196F4CF00E080E00E945A61D3CC31
:10F9F000A0E0B0E0EEEFFCE70C94F07DEC01A88015
:10FA0000B980CA80DB80A114B104C104D10441F4DF
:10FA100084E2A82E89EDB82E8BE5C82E87E0D82E7B
:10FA2000C601B5012DE133EF41E050E00E94CD7DEC
:10FA300027EA31E440E050E00E94AE7D7B018C017A
:10FA4000C601B5012DE133EF41E050E00E94CD7DCC
:10FA5000CA01B9012CEE34EF4FEF5FEF0E94AE7D8B
:10FA60006E0D7F1D801F911F97FF04C06150704075
:10FA700080409048688379838A839B839B013F778A
:10FA8000C901CDB7DEB7EAE00C940C7E0E94F87C89
:10FA9000089589E191E00E94F87C0895A0E0B0E02B
:10FAA0008093190190931A01A0931B01B0931C013C
:10FAB0000895991B79E004C0991F961708F0961BCA
:10FAC000881F7A95C9F78095089597FB092E072618
:10FAD0000AD077FD04D02ED006D000201AF47095FD
:10FAE00061957F4F0895F6F7909581959F4F089502
:10FAF000A1E21A2EAA1BBB1BFD010DC0AA1FBB1F32
:10FB0000EE1FFF1FA217B307E407F50720F0A21BA3
:10FB1000B30BE40BF50B661F771F881F991F1A9410
:10FB200069F760957095809590959B01AC01BD013A
:10FB3000CF010895AA1BBB1B51E107C0AA1FBB1F21
:10FB4000A617B70710F0A61BB70B881F991F5A9569
:10FB5000A9F780959095BC01CD010895629FD001D1
:10FB6000739FF001829FE00DF11D649FE00DF11D78
:10FB7000929FF00D839FF00D749FF00D659FF00D27
:10FB80009927729FB00DE11DF91F639FB00DE11D14
:10FB9000F91FBD01CF011124089597FB092E0526F9
:10FBA0000ED057FD04D0A4DF0AD0001C38F45095C5
:10FBB0004095309521953F4F4F4F5F4F0895F6F791
:10FBC00090958095709561957F4F8F4F9F4F0895C9
:10FBD0002F923F924F925F926F927F928F929F925D
:10FBE000AF92BF92CF92DF92EF92FF920F931F934B
:10FBF000CF93DF93CDB7DEB7CA1BDB0B0FB6F894FC
:10FC0000DEBF0FBECDBF09942A88398848885F843B
:10FC10006E847D848C849B84AA84B984C884DF80AC
:10FC2000EE80FD800C811B81AA81B981CE0FD11D90
:10FC30000FB6F894DEBF0FBECDBFED010895F89466
:02FC4000FFCFF4
:10FC4200D561E361F3620466F065E661F561046221
:0EFC5200D865126220623CC301010000000070
:00000001FF
